:020000040800F2
:10000000000008243D2E00083D2A00083F2A000871
:10001000412A0008432A0008452A00080000000081
:10002000000000000000000000000000472A000857
:10003000492A0008000000004B2A00084D2A000849
:100040008D2E00088D2E00088D2E00088D2E0008A4
:100050008D2E00088D2E00088D2E00088D2E000894
:100060008D2E00088D2E00088D2E00088D2E000884
:100070008D2E00088D2E00088D2E00088D2E000874
:100080008D2E00088D2E00088D2E00088D2E000864
:100090008D2E00088D2E00088D2E00088D2E000854
:1000A0008D2E00088D2E00088D2E00088D2E000844
:1000B0008D2E00088D2E00088D2E00088D2E000834
:1000C0008D2E00088D2E00088D2E00088D2E000824
:1000D0008D2E0008552A00088D2E0008652A00087C
:1000E0008D2E00088D2E0008000000008D2E0008C7
:1000F0008D2E00088D2E00088D2E00088D2E0008F4
:100100008D2E00088D2E00088D2E00088D2E0008E3
:100110008D2E00088D2E00088D2E00088D2E0008D3
:100120008D2E00088D2E00088D2E00088D2E0008C3
:100130008D2E00088D2E00088D2E00088D2E0008B3
:1001400000000000000000000000000000000000AF
:100150008D2E00088D2E00088D2E00088D2E000893
:100160008D2E00088D2E00088D2E00088D2E000883
:100170008D2E00088D2E00088D2E00088D2E000873
:100180008D2E00088D2E00088D2E00088D2E000863
:100190008D2E00088D2E00088D2E00088D2E000853
:1001A0008D2E00088D2E00088D2E00088D2E000843
:1001B0008D2E00088D2E00088D2E00088D2E000833
:1001C0008D2E00088D2E00088D2E00088D2E000823
:1001D0008D2E00088D2E00088D2E00088D2E000813
:1001E0008D2E00088D2E00088D2E00088D2E000803
:1001F0008D2E00088D2E00088D2E00088D2E0008F3
:100200008D2E00088D2E00088D2E00088D2E0008E2
:100210008D2E00088D2E00088D2E00088D2E0008D2
:100220008D2E00088D2E00088D2E00080000000085
:100230008D2E00088D2E0008000000008D2E000875
:100240008D2E00088D2E00088D2E00088D2E0008A2
:100250008D2E00088D2E00088D2E00088D2E000892
:100260008D2E00088D2E00088D2E00088D2E000882
:100270008D2E00088D2E00088D2E00080000000035
:100280008D2E00088D2E00088D2E00080000000025
:08029000000000008D2E0008A3
:1002C00010B5054C237833B9044B13B10448AFF390
:1002D00000800123237010BDCC0900240000000021
:1002E0001CE9000808B5034B1BB103490348AFF3F1
:1002F000008008BD00000000D00900241CE90008AF
:1003000081F0004102E000BF83F0004330B54FEAC6
:1003100041044FEA430594EA050F08BF90EA020F33
:100320001FBF54EA000C55EA020C7FEA645C7FEAC6
:10033000655C00F0E2804FEA5454D4EB5555B8BFE9
:100340006D420CDD2C4480EA020281EA030382EA5A
:10035000000083EA010180EA020281EA0303362DEC
:1003600088BF30BD11F0004F4FEA01314FF4801CBF
:100370004CEA113102D0404261EB410113F0004FD1
:100380004FEA03334CEA133302D0524263EB430388
:1003900094EA050F00F0A780A4F10104D5F1200E26
:1003A0000DDB02FA0EFC22FA05F2801841F1000181
:1003B00003FA0EF2801843FA05F359410EE0A5F155
:1003C00020050EF1200E012A03FA0EFC28BF4CF086
:1003D000020C43FA05F3C01851EBE37101F000453C
:1003E00007D54FF0000EDCF1000C7EEB00006EEB49
:1003F0000101B1F5801F1BD3B1F5001F0CD34908D3
:100400005FEA30004FEA3C0C04F101044FEA445229
:1004100012F5800F80F09A80BCF1004F08BF5FEAB0
:10042000500C50F1000041EB045141EA050130BD90
:100430005FEA4C0C404141EB0101013C28BFB1F5A2
:10044000801FE9D291F0000F04BF01460020B1FAED
:1004500081F308BF2033A3F10B03B3F120020CDAC0
:100460000C3208DD02F1140CC2F10C0201FA0CF09E
:1004700021FA02F10CE002F11402D8BFC2F1200C03
:1004800001FA02F120FA0CFCDCBF41EA0C019040B9
:10049000E41AA2BF01EB0451294330BD6FEA040402
:1004A0001F3C1CDA0C340EDC04F11404C4F12002ED
:1004B00020FA04F001FA02F340EA030021FA04F3FF
:1004C00045EA030130BDC4F10C04C4F1200220FA56
:1004D00002F001FA04F340EA0300294630BD21FA94
:1004E00004F0294630BD94F0000F83F4801306BF5A
:1004F00081F480110134013D4EE77FEA645C18BF4E
:100500007FEA655C29D094EA050F08BF90EA020FE4
:1005100005D054EA000C04BF1946104630BD91EADC
:10052000030F1EBF0021002030BD5FEA545C05D1DF
:100530004000494128BF41F0004130BD14F580041E
:100540003CBF01F5801130BD01F0004545F0FE4192
:1005500041F470014FF0000030BD7FEA645C1ABFC7
:10056000194610467FEA655C1CBF0B46024650EAFE
:10057000013406BF52EA033591EA030F41F400212A
:1005800030BD00BF90F0000F04BF0021704730B5B0
:100590004FF4806404F132044FF000054FF0000185
:1005A00050E700BF90F0000F04BF0021704730B546
:1005B0004FF4806404F1320410F0004548BF40421B
:1005C0004FF000013EE700BF42004FEAE2014FEA70
:1005D00031014FEA02701FBF12F07F4393F07F4F4B
:1005E00081F06051704732F07F4208BF704793F04E
:1005F0007F4F04BF41F40021704730B54FF4607461
:1006000001F0004521F000411CE700BF50EA010263
:1006100008BF704730B54FF000050AE050EA01020C
:1006200008BF704730B511F0004502D5404261EB7C
:1006300041014FF4806404F132045FEA915C3FF4BD
:10064000D8AE4FF003025FEADC0C18BF03325FEA5A
:10065000DC0C18BF033202EBDC02C2F1200300FA0B
:1006600003FC20FA02F001FA03FE40EA0E0021FA30
:1006700002F11444BDE600BF4FF0FF3C06E000BFAE
:100680004FF0010C02E000BF4FF0010C4DF804CD1B
:100690004FEA410C7FEA6C5C4FEA430C18BF7FEADB
:1006A0006C5C1BD001B050EA410C0CBF52EA430C09
:1006B00091EA030F02BF90EA020F0020704710F189
:1006C000000F91EA030F58BF994208BF90422CBF18
:1006D000D8176FEAE37040F0010070474FEA410C11
:1006E0007FEA6C5C02D150EA013C07D14FEA430C2F
:1006F0007FEA6C5CD6D152EA033CD3D05DF8040BA0
:10070000704700BF8446104662468C4619466346D1
:1007100000E000BF01B5FFF7B7FF002848BF10F1A8
:10072000000F01BD4DF808EDFFF7F4FF0CBF0120ED
:1007300000205DF808FB00BF4DF808EDFFF7EAFF69
:1007400034BF012000205DF808FB00BF4DF808ED24
:10075000FFF7E0FF94BF012000205DF808FB00BF19
:100760004DF808EDFFF7CEFF94BF012000205DF8A3
:1007700008FB00BF4DF808EDFFF7C4FF34BF0120B0
:1007800000205DF808FB00BF4FEA410C7FEA6C5C7B
:1007900002D150EA013C0AD14FEA430C7FEA6C5C7B
:1007A00002D152EA033C02D14FF0000070474FF0F3
:1007B000010070474FEA410212F5001215D211D51F
:1007C0006FF47873B3EB625212D94FEAC12343F04E
:1007D000004343EA505311F0004F23FA02F018BFD0
:1007E000404270474FF00000704750EA013005D199
:1007F00011F0004008BF6FF0004070474FF000005C
:10080000704700BF80F0004002E000BF81F000416F
:1008100042001FBF5FEA410392EA030F7FEA226CA6
:100820007FEA236C6AD04FEA1262D2EB1363C1BF36
:10083000D218414048404140B8BF5B42192B88BFA5
:10084000704710F0004F40F4000020F07F4018BFC8
:10085000404211F0004F41F4000121F07F4118BFE8
:10086000494292EA030F3FD0A2F1010241FA03FC90
:1008700010EB0C00C3F1200301FA03F100F0004378
:1008800002D5494260EB4000B0F5000F13D3B0F140
:10089000807F06D340084FEA310102F10102FE2AAF
:1008A00051D2B1F1004F40EBC25008BF20F001001F
:1008B00040EA03007047490040EB0000013A28BFBE
:1008C000B0F5000FEDD2B0FA80FCACF1080CB2EB41
:1008D0000C0200FA0CF0AABF00EBC25052421843BF
:1008E000BCBFD0401843704792F0000F81F4000164
:1008F00006BF80F400000132013BB5E74FEA410337
:100900007FEA226C18BF7FEA236C21D092EA030FA2
:1009100004D092F0000F08BF0846704790EA010F1C
:100920001CBF0020704712F07F4F04D1400028BF49
:1009300040F00040704712F100723CBF00F500002B
:10094000704700F0004343F0FE4040F40000704761
:100950007FEA226216BF08467FEA2363014642020D
:1009600006BF5FEA412390EA010F40F48000704720
:100970004FF0000304E000BF10F0004348BF4042C6
:100980005FEA000C08BF704743F0964301464FF002
:1009900000001CE050EA010208BF70474FF000035E
:1009A0000AE000BF50EA010208BF704711F000439F
:1009B00002D5404261EB41015FEA010C02BF84466F
:1009C0000146002043F0B64308BFA3F18053A3F5CE
:1009D0000003BCFA8CF2083AA3EBC25310DB01FA15
:1009E00002FC634400FA02FCC2F12002BCF1004F99
:1009F00020FA02F243EB020008BF20F0010070472A
:100A000002F1200201FA02FCC2F1200250EA4C007D
:100A100021FA02F243EB020008BF20EADC707047C3
:100A20004FF0FF0C1CEAD0521EBF1CEAD15392EAD1
:100A30000C0F93EA0C0F6FD01A4480EA010C4002AD
:100A400018BF5FEA41211ED04FF0006343EA501007
:100A500043EA5111A0FB01310CF00040B1F5000F49
:100A60003EBF490041EAD3715B0040EA010062F1F8
:100A70007F02FD2A1DD8B3F1004F40EBC25008BFE2
:100A800020F00100704790F0000F0CF0004C08BF00
:100A900049024CEA502040EA51207F3AC2BFD2F1CD
:100AA000FF0340EAC250704740F400004FF00003DB
:100AB000013A5DDC12F1190FDCBF00F00040704715
:100AC000C2F10002410021FA02F1C2F1200200FA53
:100AD00002FC5FEA310040F1000053EA4C0308BF1A
:100AE00020EADC70704792F0000F00F0004C02BF6B
:100AF000400010F4000F013AF9D040EA0C0093F0E6
:100B0000000F01F0004C02BF490011F4000F013B3F
:100B1000F9D041EA0C018FE70CEAD15392EA0C0FAD
:100B200018BF93EA0C0F0AD030F0004C18BF31F018
:100B3000004CD8D180EA010000F00040704790F0EE
:100B4000000F17BF90F0004F084691F0000F91F092
:100B5000004F14D092EA0C0F01D142020FD193EA58
:100B60000C0F03D14B0218BF084608D180EA0100E0
:100B700000F0004040F0FE4040F40000704740F0BC
:100B8000FE4040F4400070474FF0FF0C1CEAD0528A
:100B90001EBF1CEAD15392EA0C0F93EA0C0F69D0E6
:100BA000A2EB030280EA010C49024FEA402037D051
:100BB0004FF0805343EA111143EA10130CF0004048
:100BC0008B4238BF5B0042F17D024FF4000C8B4238
:100BD00024BF5B1A40EA0C00B3EB510F24BFA3EB18
:100BE000510340EA5C00B3EB910F24BFA3EB9103E8
:100BF00040EA9C00B3EBD10F24BFA3EBD10340EA42
:100C0000DC001B0118BF5FEA1C1CE0D1FD2A3FF687
:100C100050AF8B4240EBC25008BF20F0010070473C
:100C20000CF0004C4CEA50207F32C2BFD2F1FF03DF
:100C300040EAC250704740F400004FF00003013A10
:100C400037E792F0000F00F0004C02BF400010F4B4
:100C5000000F013AF9D040EA0C0093F0000F01F0C8
:100C6000004C02BF490011F4000F013BF9D041EAEA
:100C70000C0195E70CEAD15392EA0C0F08D142021D
:100C80007FF47DAF93EA0C0F7FF470AF084676E7F0
:100C900093EA0C0F04D14B023FF44CAF08466EE7C9
:100CA00030F0004C18BF31F0004CCAD130F0004297
:100CB0007FF45CAF31F000437FF43CAF5FE700BFEF
:100CC00042000ED2B2F1FE4F0BD34FF09E03B3EBB6
:100CD000126209D44FEA002343F0004323FA02F0E2
:100CE00070474FF00000704712F1610F01D14202CE
:100CF00002D14FF0FF3070474FF00000704700BF47
:100D000053B94AB9002908BF00281CBF4FF0FF3172
:100D10004FF0FF3000F074B9ADF1080C6DE904CE6E
:100D200000F006F8DDF804E0DDE9022304B07047C6
:100D30002DE9F047089E0D4604468846002B4DD10C
:100D40008A42944668D9B2FA82F252B101FA02F3A9
:100D5000C2F1200120FA01F10CFA02FC41EA030879
:100D600094404FEA1C45210CB8FBF5FE1FFA8CF7A6
:100D700005FB1E8341EA03430EFB07F199420BD9A1
:100D80001CEB03030EF1FF3080F01E81994240F20C
:100D90001B81AEF1020E63445B1AA4B2B3FBF5F003
:100DA00005FB103344EA034400FB07F7A7420AD9C6
:100DB0001CEB040400F1FF3380F00881A74240F2ED
:100DC000058164440238E41B40EA0E4000211EB154
:100DD000D4400023C6E90043BDE8F0878B4208D920
:100DE000002E00F0EE800021C6E900050846BDE8AF
:100DF000F087B3FA83F100294AD1AB4202D3824291
:100E000000F2F980841A65EB030301209846002E56
:100E1000E2D0C6E90048DFE702B9FFDEB2FA82F2AB
:100E2000002A40F09180A1EB0C054FEA1C471FFA05
:100E30008CFE0121B5FBF7F307FB1350250C45EAA7
:100E400000450EFB03F0A84208D91CEB050503F191
:100E5000FF3802D2A84200F2CB8043462D1AA4B23A
:100E6000B5FBF7F007FB105544EA05440EFB00FE06
:100E7000A64508D91CEB040400F1FF3502D2A645B3
:100E800000F2BB802846A4EB0E0440EA03409EE734
:100E9000C1F120078B4022FA07FC4CEA030C20FA30
:100EA00007F405FA01F31C43FD404FEA1C4900FA20
:100EB00001F3B5FBF9F8200C1FFA8CFE09FB18555D
:100EC00040EA054508FB0EF0A84202FA01F20BD9F0
:100ED0001CEB050508F1FF3A80F08880A84240F23B
:100EE0008580A8F1020865442D1AA4B2B5FBF9F07B
:100EF00009FB105544EA054500FB0EFEAE4508D936
:100F00001CEB050500F1FF346CD2AE456AD90238FE
:100F1000654440EA0840A0FB0294A5EB0E05A542FB
:100F2000C846A64656D353D05EB1B3EB080265EB74
:100F30000E0505FA07F722FA01F3CD401F43C6E973
:100F400000750021BDE8F087C2F1200320FA03F10B
:100F50000CFA02FC25FA03F395400D434FEA1C47B7
:100F60001FFA8CFEB3FBF7F107FB11302B0C43EAA1
:100F7000004301FB0EF0984204FA02F408D91CEB7E
:100F8000030301F1FF382FD298422DD9023963446F
:100F90001B1AADB2B3FBF7F007FB103345EA03456C
:100FA00000FB0EF3AB4208D91CEB050500F1FF383E
:100FB00016D2AB4214D902386544ED1A40EA014119
:100FC00038E73146304607E78646E5E61846FAE652
:100FD0004B45A9D2B9EB020864EB0C0E0138A3E72C
:100FE0004046EAE7204694E74146D1E7D0467BE712
:100FF000023B654432E7084609E76444023842E7A9
:10100000704700BF844641EA000313F003036DD12B
:10101000403A41D351F8043B40F8043B51F8043BBB
:1010200040F8043B51F8043B40F8043B51F8043BC2
:1010300040F8043B51F8043B40F8043B51F8043BB2
:1010400040F8043B51F8043B40F8043B51F8043BA2
:1010500040F8043B51F8043B40F8043B51F8043B92
:1010600040F8043B51F8043B40F8043B51F8043B82
:1010700040F8043B51F8043B40F8043B51F8043B72
:1010800040F8043B51F8043B40F8043B51F8043B62
:1010900040F8043B403ABDD2303211D351F8043B02
:1010A00040F8043B51F8043B40F8043B51F8043B42
:1010B00040F8043B51F8043B40F8043B103AEDD2B1
:1010C0000C3205D351F8043B40F8043B043AF9D202
:1010D000043208D0D2071CBF11F8013B00F8013BD5
:1010E00001D30B8803806046704700BF082A13D3E2
:1010F0008B078DD010F003038AD0C3F10403D21AFA
:10110000DB071CBF11F8013B00F8013B80D331F82D
:10111000023B20F8023B7BE7043AD9D3013A11F8AD
:10112000013B00F8013BF9D20B7803704B78437018
:101130008B7883706046704700000000000000005C
:10114000A2EB0300704700BF02780B78012A28BF8A
:101150009A42F5D16DE9044540EA0104CDE9026700
:101160006FF0000C4FEA447212B380EA010414F0ED
:10117000070F6AD100F0070420F0070004F0030510
:1011800021F007014FEAC505F0E8042314F0040F2D
:10119000F1E804670CFA05F462EA040266EA040660
:1011A0000AD063EA0403624667EA0407664603E07E
:1011B000F0E80423F1E8046782FA4CF582EA0604B9
:1011C000A4FA8CF46CBB83FA4CF583EA0705A5FA04
:1011D0008CF595B950E9022351E9026782FA4CF582
:1011E00082EA0604A4FA8CF483FA4CF583EA070534
:1011F000A5FA8CF52543DBD09CB92DBAB5FA85F458
:1012000024F0070427FA04F1DDE9026723FA04F366
:1012100003F0FF0001F0FF01FDE80445A0EB010031
:10122000704724BAB4FA84F424F0070426FA04F1CF
:10123000DDE9026722FA04F202F0FF0001F0FF018B
:10124000FDE80445A0EB0100704714F0030F3CD10A
:1012500010F0030428D150F8082B51F8083B82FA0B
:101260004CF582EA0305A5FA8CF55DB950F8042C1B
:1012700051F8043C82FA4CF582EA0305A5FA8CF594
:10128000002DE8D02DBAB5FA85F424F0070423FA2E
:1012900004F122FA04F202F0FF0001F0FF01FDE880
:1012A0000445A0EB010070474FEAC40420F003009E
:1012B00050F8082B21F0030151F8083B0CFA04F414
:1012C00062EA040263EA0403C9E710F003041AD0D7
:1012D000A1EB040120F00300E40750F8042B06D032
:1012E0000FD28B785FFAA2F4E41A06D12BB1CB7837
:1012F0005FFAB2F4E41A00D11BB920465DF8104B36
:10130000704701F1040150F8042BCC0721F00301D0
:1013100051F8043B48D824D222F07F4482FA4CF59D
:1013200094EA1325A5FA8CF50AD165B951F8043B66
:1013300084EA0204B4EB036F0ED150F8042BEBE700
:101340004FEA132355E035F07F454DD10878FDE88D
:101350000445C0F1000070474FEA126203F0FF033A
:1013600047E002EA1C4482FA4CF594EA1345A5FAD8
:101370008CF50AD165B951F8043B84EA0204B4EB58
:10138000034F0CD150F8042BEBE74FEA134330E046
:1013900015EA1C4528D10B884FEA124229E04FEA92
:1013A000124203EA1C4324E002F0FF0482FA4CF5E7
:1013B00094EA1365A5FA8CF50AD165B951F8043B96
:1013C00084EA0204B4EB032F09D150F8042BEBE7B5
:1013D0004FEA13630DE015F0FF0F05D10B684FEADC
:1013E000122223F07F4304E04FF00000FDE80445A3
:1013F000704712BA1BBA82FA4CF482EA0304A4FAC8
:101400008CF5B5FA85F402FA04F203FA04F34FEA14
:101410001260FDE80445A0EB136070470000000077
:1014200000000000000000000000000000000000BC
:1014300000000000000000000000000000000000AC
:1014400090F800F06DE9024520F007016FF0000C04
:1014500010F0070491F820F040F049804FF00004AC
:101460006FF00700D1E9002391F840F000F1080087
:1014700082FA4CF2A4FA8CF283FA4CF3A2FA8CF3BF
:101480004BBBD1E9022382FA4CF200F10800A4FA26
:101490008CF283FA4CF3A2FA8CF3E3B9D1E904237A
:1014A00082FA4CF200F10800A4FA8CF283FA4CF3B1
:1014B000A2FA8CF37BB9D1E9062301F1200182FA6B
:1014C0004CF200F10800A4FA8CF283FA4CF3A2FA71
:1014D0008CF3002BC6D0002A04BF04301A4612BA7F
:1014E000B2FA82F2FDE8024500EBD2007047D1E982
:1014F000002304F00305C4F100004FEAC50514F011
:10150000040F91F840F00CFA05F562EA05021CBFE1
:1015100063EA050362464FF00004A9E700000000FB
:1015200001F0FF01102A2BDB10F0070F08D010F894
:10153000013B013A8B422DD010F0070F42B3F6D198
:10154000F0B441EA012141EA014122F007047FF0B1
:1015500000070023F0E80256083C85EA010586EA08
:10156000010685FA47F5A3FA87F586FA47F6A5FA44
:1015700087F68EB9EED1F0BC01F0FF0102F0070250
:1015800032B110F8013B013A83EA010313B1F8D1FB
:101590000020704701387047002D06BF35460338DC
:1015A000073815F0010F07D1013015F4807F02BF15
:1015B000013015F4C03F0130F0BC0138704700BF66
:1015C00070B54FF0FF0C4CF4E06C1CEA11541DBFD9
:1015D0001CEA135594EA0C0F95EA0C0F00F0DEF8A4
:1015E0002C4481EA030621EA4C5123EA4C5350EA89
:1015F000013518BF52EA033541F4801143F48013DA
:1016000038D0A0FB02CE4FF00005E1FB02E506F06A
:101610000042E0FB03E54FF00006E1FB03569CF0BF
:10162000000F18BF4EF0010EA4F1FF04B6F5007FC5
:1016300064F5407404D25FEA4E0E6D4146EB060637
:1016400042EAC62141EA55514FEAC52040EA5E50C0
:101650004FEACE2EB4F1FD0C88BFBCF5E06F1ED86A
:10166000BEF1004F08BF5FEA500E50F1000041EBA1
:10167000045170BD06F0004646EA010140EA02004E
:1016800081EA0301B4EB5C04C2BFD4EB0C0541EA70
:10169000045170BD41F480114FF0000E013C00F385
:1016A000AB8014F1360FDEBF002001F0004170BDA9
:1016B000C4F10004203C35DA0C341BDC04F11404C2
:1016C000C4F1200500FA05F320FA04F001FA05F24E
:1016D00040EA020001F0004221F0004110EBD3701B
:1016E00021FA04F642EB06015EEA430E08BF20EA47
:1016F000D37070BDC4F10C04C4F1200500FA04F3EA
:1017000020FA05F001FA04F240EA020001F000417B
:1017100010EBD37041F100015EEA430E08BF20EAEE
:10172000D37070BDC4F1200500FA05F24EEA020E36
:1017300020FA04F301FA05F243EA020321FA04F065
:1017400001F0004121FA04F220EA020000EBD3701C
:101750005EEA430E08BF20EAD37070BD94F0000F1C
:101760000FD101F00046400041EB010111F4801F50
:1017700008BF013CF7D041EA060195F0000F18BF01
:10178000704703F00046520043EB030313F4801F3D
:1017900008BF013DF7D043EA0603704794EA0C0FF7
:1017A0000CEA135518BF95EA0C0F0CD050EA41060D
:1017B00018BF52EA4306D1D181EA030101F000418A
:1017C0004FF0000070BD50EA410606BF10461946B2
:1017D00052EA430619D094EA0C0F02D150EA0136BE
:1017E00013D195EA0C0F05D152EA03361CBF1046FF
:1017F00019460AD181EA030101F0004141F0FE419E
:1018000041F470014FF0000070BD41F0FE4141F421
:10181000780170BD70B54FF0FF0C4CF4E06C1CEA21
:1018200011541DBF1CEA135594EA0C0F95EA0C0FD6
:1018300000F0A7F8A4EB050481EA030E52EA033591
:101840004FEA013100F088804FEA03334FF08055B2
:1018500045EA131343EA12634FEA022245EA1115DF
:1018600045EA10654FEA00260EF000419D4208BF90
:10187000964244F1FD0404F5407402D25B084FEA3D
:101880003202B61A65EB03055B084FEA32024FF4E9
:1018900080104FF4002CB6EB020E75EB030E22BF46
:1018A000B61A754640EA0C005B084FEA3202B6EB06
:1018B000020E75EB030E22BFB61A754640EA5C00B5
:1018C0005B084FEA3202B6EB020E75EB030E22BF45
:1018D000B61A754640EA9C005B084FEA3202B6EB46
:1018E000020E75EB030E22BFB61A754640EADC0005
:1018F00055EA060E18D04FEA051545EA16754FEA67
:1019000006164FEAC30343EA52734FEAC2025FEA84
:101910001C1CC0D111F4801F0BD141EA00014FF013
:1019200000004FF0004CB6E711F4801F04BF0143E4
:101930000020B4F1FD0C88BFBCF5E06F3FF6AFAE00
:10194000B5EB030C04BFB6EB020C5FEA500C50F190
:10195000000041EB045170BD0EF0004E4EEA113113
:1019600014EB5C04C2BFD4EB0C0541EA045170BD1A
:1019700041F480114FF0000E013C90E645EA060E5E
:101980008DE60CEA135594EA0C0F08BF95EA0C0F8C
:101990003FF43BAF94EA0C0F0AD150EA01347FF4D4
:1019A00034AF95EA0C0F7FF425AF104619462CE7AB
:1019B00095EA0C0F06D152EA03353FF4FDAE10460E
:1019C000194622E750EA410618BF52EA43067FF45F
:1019D000C5AE50EA41047FF40DAF52EA43057FF4EF
:1019E000EBAE12E74A0011D212F5001211D20DD55A
:1019F0006FF47873B3EB62520ED44FEAC12343F015
:101A0000004343EA505323FA02F070474FF00000BE
:101A1000704750EA013002D14FF0FF3070474FF06D
:101A20000000704738B505460C462846214600227E
:101A30000023FEF781FE28B928462146BDE838403C
:101A400000F00AB8284604F1004100F005F84042D1
:101A500061EB410138BD00BFD0B50C4B00220646FA
:101A60000F46FFF7ADFDFFF7BDFF0446FEF78AFD09
:101A7000074B0022FFF7A4FD02460B4630463946CD
:101A8000FEF742FCFFF7AEFF2146D0BD0000F03D5F
:101A90000000F04108B50146014805F01DFC08BDF5
:101AA00038E900084FF07E507047000038B50B4B06
:101AB0001A88B3F90030002B00DB38BDD2B2084CD5
:101AC0000025A554204600F031FD044B1D80C8229E
:101AD0002946204605F0A2FBEFE700BF100B0024CB
:101AE000480A002408B5044B044A07CA83E80700E3
:101AF000184605F053FC08BD000A002444E900081C
:101B000010B5054C054A234607CA03C31A70204680
:101B100005F044FC10BD00BF0C0A002450E9000889
:101B200010B5054C054A234607CA03C31A70204660
:101B300005F034FC10BD00BFF40900245CE9000886
:101B400008B5054B054A92E803001860197118465C
:101B500005F024FC08BD00BFEC09002468E900087A
:101B600008B50348034B036005F018FC08BD00BF2F
:101B7000E809002435313200002918BF002826D09A
:101B800000B586468C4688420BD100201DE002F14C
:101B900020010FE0814217D1DAB10EF1010E0CF1F4
:101BA000010C9EF800200C4BD35C03F00303012BC7
:101BB000EDD011469CF80000074BC35C03F0030313
:101BC000012BE7D12030E5E7081A5DF804FB01207E
:101BD00070470020F9E700BFF9EA00082E2070479F
:101BE0008446002318460AE0A1F14102D2B2052A38
:101BF00011D808443738022B00D800010133032BD9
:101C000011D81CF80310A1F13002D2B2092AEBD886
:101C100008443038EFE7A1F16102D2B2052A03D8B7
:101C200008445738E7E7704700207047F8B50B1AAB
:101C3000052B60DD06460F4615460230FFF7D0FF44
:101C40000446A0F55C43B3F5806F56D3A0F5584326
:101C5000B3F5806F1CD2B11D7F1A052F4FDDB3790C
:101C60005C2B4ED1F379752B4DD106F10800FFF7AF
:101C7000B7FFA0F55C43B3F5806F46D2254B03EA6E
:101C80008424C0F30900204300F580340C2000E0D8
:101C900006207F2C0BD9B4F5006F0DD3B4F5803F2F
:101CA0000DD3B4F5881F32D2F027042601E00027B7
:101CB0000126731EDBB20EE0C0270226F9E7E027FB
:101CC0000326F6E704F03F012A6841F08001D15471
:101CD000A409013BDBB2002BF4D1012E06D92B68FD
:101CE0003C431C702B6833442B6005E02B6804F0E8
:101CF0007F041C70F6E70020F8BD0020FCE7002000
:101D0000FAE70020F8E70020F6E70020F4E70020DB
:101D1000F2E700BF00FC0F002DE9F04182B00E4653
:101D20000F688B685D1C3D440022019207EB030C99
:101D3000FB5C222B40F0858080462C46104600E05C
:101D40000134E11B726891420AD22378222B07D01A
:101D50005C2BF5D10134E31B934272D20130EFE7E3
:101D600091426ED22378222B6BD1A4EB0C0CACEBFE
:101D70000000336901309847074600285DD0019084
:101D80002BE0631B002B58DD6B78752B55D85C2B33
:101D900011D35C3B192B50D8DFE803F0114F4F4FA4
:101DA0004F4F184F4F4F2B4F4F4F4F4F4F4F324FBB
:101DB0004F4F394F4047222B01D02F2B3DD1019B54
:101DC0005A1C01926A781A70022305E0019B5A1C82
:101DD000019208221A7002231D44A54239D22B78A1
:101DE0005C2BCED0019B5A1C019215F8012B1A7066
:101DF000F3E7019B5A1C01920C221A700223EBE7B5
:101E0000019B5A1C01920A221A700223E4E7019BEB
:101E10005A1C01920D221A700223DDE7019B5A1C05
:101E2000019209221A700223D6E701AA2146284608
:101E3000FFF7FCFE03460028CED117B17369384680
:101E40009847ADB13368ED1AB560002002B0BDE827
:101E5000F081019B00221A701023C8F80C30C8F8DA
:101E600010703368E41AB4600134B4600120EDE707
:101E70000020EBE70246D0B110B40468ACB183682F
:101E80004068834202D30AE001339360936898422A
:101E900002D9E15C2029F7D99368984202D0104614
:101EA00010BC7047013B9360F9E72246F7E77047A3
:101EB00010B5036828209847044618B1282200214D
:101EC00005F0ACF9204610BD38B5044678B100687D
:101ED00078B1A5687DB92B1D6268934207D20322B1
:101EE0000649284405F08AFD08B90335A560204657
:101EF00038BD0446FBE70024F9E700BF70E900089D
:101F00002DE9F04393B005460C4600231193FFF7EB
:101F100065FE002C00F099802368002B00F097806C
:101F2000002331E0652A29D048336B44002203F8AE
:101F3000442C0DF1040911A9484606F039FD064666
:101F40000F46DDF84480C84500F08380C5E9066788
:101F500041A3D3E90023FEF703FC002864D06FF00F
:101F600000436B610823EB6001ABA8EB0308A36897
:101F70004344A360012013B0BDE8F08303F148019E
:101F8000694401F8442C01333E2BCDD8A2681A4491
:101F900061688A42C8D221688A5C452AC2D82B2A45
:101FA000C2D3A2F12B011A29BED801A656F821F0FE
:101FB0007D1F0008291F00087D1F00081D20000844
:101FC000291F00087D1F00087D1F00087D1F0008D5
:101FD0007D1F00087D1F00087D1F00087D1F000871
:101FE0007D1F00087D1F00087D1F0008291F0008B5
:101FF000291F0008291F0008291F0008291F0008A1
:10200000291F0008291F0008291F0008291F000890
:10201000291F0008291F00087D1F000803F148023E
:102020006A4402F8440CAEE700220D4B30463946B4
:10203000FEF78CFB18B14FF000436B6192E730461E
:102040003946FEF7B7FB68618CE7002093E7002074
:1020500091E700208FE700BF0000C0FFFFFFDF41D6
:102060000000E0C138B5002918BF00281AD00D467D
:1020700084680AB90AE024687CB1216A69B12846FB
:10208000FFF762F80028F6D107E024682CB1216A36
:102090002846FFF771FD0028F7D12CB1236A2BB138
:1020A000204638BD0024FBE70024F9E70024F7E7C9
:1020B00038B5044616E0E36813F4807F04D1206944
:1020C00010B10F4B5B689847E36813F4007F04D1AD
:1020D000206A10B10A4B5B689847094B5B68204641
:1020E00098472C4654B12568E36813F4807FE2D109
:1020F000A0680028DFD0FFF7DBFFDCE738BD00BFBA
:1021000000000024CB68B3F57A7F80F08B802DE946
:10211000F04106460C460133CB60002900F0848074
:102120008B684A68934280F081800A68D25C7B2A7F
:1021300002D00020BDE8F08101338B600846FFF734
:1021400099FEA3686268934203D22268D35C7D2B18
:1021500059D0A3686268934204D2013BA360002572
:102160002F4634E0013BA3600020E3E70746A36865
:102170000133A3602046FFF77DFE21462846FFF786
:10218000CBFD002839D02046FFF774FE2B692B6267
:1021900000232B61A368626893422ED22268D25C2E
:1021A0003A2A2AD10133A3602046FFF763FE214675
:1021B000284600F03FF800B32046FFF75BFEA36817
:1021C0006268934211D22268D35C2C2B0DD1A846B1
:1021D00004F11000FFF76CFE054670B1002FC5D06A
:1021E000C8F80000C0F80480C1E7A36862689342A1
:1021F00003D22268D35C7D2B07D0CFB13846FFF7DE
:1022000057FF002096E700252F46E368013BE36077
:1022100007B17D604023F360B760A3680133A3601A
:10222000012087E700207047002083E7002081E736
:1022300000207FE7002975D070B506460C460D6872
:10224000002D71D08868021D4B689A4206D804227E
:102250003749284405F0D2FB00283AD0A068421D37
:1022600063689A4206D805223249284405F0C6FB25
:10227000002835D0A068021D63689A4206D804225F
:102280002D49284405F0BAFB00282FD0A3686268C6
:10229000934202D2EB5C222B30D0A3686268934257
:1022A00007D2EA5CA2F13003DBB22D2A18BF092B5A
:1022B00029D9A3686268934202D2EB5C5B2B27D0DA
:1022C000A3686268934231D2EB5C7B2B25D000205F
:1022D0002DE00423F360A3680433A360012026E00B
:1022E0000120F060A2680532A26020E00223F360C2
:1022F00001207061A2680432A26018E021463046D5
:10230000FFF70AFD13E021463046FFF7F9FD0EE026
:102310002146304600F012F809E021463046FFF72A
:10232000F1FE04E000207047002000E0002070BDB6
:1023300074E9000894E900089CE90008CB68B3F54B
:102340007A7F6DD22DE9F04106460C460133CB6011
:102350000A688B68D25C5B2A02D00020BDE8F0815D
:1023600001338B600846FFF785FD3CB1A3686268C6
:10237000934203D22268D35C5D2B48D044B1A3685A
:102380006268934204D2013BA36000252F461EE001
:10239000A368013BA3600020E0E7C8F80000C0F894
:1023A0000480A3680133A3602046FFF763FD214644
:1023B0002846FFF73FFF68B32046FFF75BFDA368A1
:1023C000626893420ED22268D35C2C2B0AD1A846B5
:1023D00004F11000FFF76CFD0546D8B1002FDCD1E9
:1023E0000746DEE7A3686268934213D22268D35C93
:1023F0005D2B0FD1E368013BE36007B17D602023D3
:10240000F360B760A3680133A3600120A6E700254D
:102410002F46EFE737B13846FFF74AFE00209DE729
:1024200000207047002099E7F0B58BB015461E4696
:102430000024039404940594069407940894099442
:102440002B4B1C605C600446002918BF002817D184
:10245000002C4AD0019400230293059A049B9A42CF
:102460003ED2029215B1029B23442B60204B01AA5D
:1024700092E8030083E80300002738460BB0F0BD64
:10248000039004911B4B93E807000AAF07E907008C
:102490001846FFF70DFD0746E0B103A8FFF714FD4E
:1024A000FFF7E8FC01463846FFF7C4FE90B136B9A5
:1024B000002DE2D0039B059A13442B60DDE703A8AF
:1024C000FFF7D8FC059B049A934203D2039AD35C8E
:1024D000002BEDD0002FBBD03846FFF7E9FDB7E762
:1024E000002BBFD0013B0293BCE72746C5E700BFE6
:1024F000180A00240000002470B5044648B10D46B7
:102500001646FEF79DFF33462A46411C2046FFF73C
:102510008BFF70BD08B500221146FFF7EDFF08BD27
:1025200008B50022FFF79EFD08BD00002DE9F84F19
:10253000044601463E4804F0CFFE2046FFF7EAFF7E
:10254000002871D004463B49FFF7EAFF05463A49A7
:102550002046FFF7E5FF064638492046FFF7E0FF33
:10256000804637492046FFF7DBFF074635492046BE
:10257000FFF7D6FF824634492046FFF7D1FF814658
:1025800032492046FFF7CCFF8346002D18BF002EAE
:1025900045D03B1E18BF0123B8F1000F3FD0002BE0
:1025A0003DD0B9F1000318BF0123BAF1000F36D0B6
:1025B000002B34D0002832D06969254804F08CFE05
:1025C0007169244804F088FED8F81410224804F0F9
:1025D00083FE7969214804F07FFEDAF81410204860
:1025E00004F07AFED9F814101E4804F075FEDBF8EA
:1025F00014101D4804F070FED8F814201B4B9A608C
:1026000072695A606A691A607A69DA60DAF81420C5
:102610001A61D9F814205A61DBF814201A76204682
:10262000FFF746FDBDE8F88F114804F0B7FEF9E763
:10263000A4E90008B8E90008C4E90008C8E90008EE
:10264000CCE90008DCE90008ECE9000800EA000831
:1026500018EA00082CEA000834EA00083CEA0008FE
:1026600050EA000864EA00087CEA0008200A002416
:1026700098EA000800487047200A002430B589B065
:102680000024039404940594069407941B4BD3F8F8
:10269000E02042F08002C3F8E020D3F8E02002F00E
:1026A00080020092009AD3F8E02042F00102C3F8C1
:1026B000E020D3F8E02002F001020192019AD3F861
:1026C000E02042F00202C3F8E020D3F8E03003F04B
:1026D00002030293029B0A4D22460221284601F082
:1026E0009BF802230393012204920594069303A905
:1026F000284600F07DFF09B030BD00BF00440258FD
:102700000000025872B6FEE700B59FB04C220021CF
:102710000BA804F083FD2022002103A804F07EFD15
:10272000022001F07FF800230093384BDA6A22F090
:102730000102DA62DB6A03F001030093344B9A6909
:1027400042F440429A619B6903F440430093009B2A
:102750002F4B9B6913F4005FFAD02E4BD3F8F42073
:1027600042F00202C3F8F420D3F8F43003F002037D
:102770000193019B00230293254B9A6942F4404246
:102780009A619B6903F440430293204BDA6A42F05A
:102790000102DA62DB6A03F001030293029B1C4B25
:1027A0009B6913F4005FFAD001230B934FF480333D
:1027B0000C930223149315931693F02217921893F7
:1027C00019931A9308231B9300231C931D930BA8A2
:1027D00001F052F8B0B93F2303930323049300237D
:1027E0000593082306934023079308934FF48062D0
:1027F00009920A93042103A801F0A4FC20B91FB098
:102800005DF804FBFFF77EFFFFF77CFF0004005834
:10281000004802580044025810B5444B5B6913F459
:10282000003F13D1BFF34F8FBFF36F8F3F4B002299
:10283000C3F85022BFF34F8FBFF36F8F5A6942F432
:1028400000325A61BFF34F8FBFF36F8F374B5B6915
:1028500013F4803F27D1354B0022C3F88420BFF307
:102860004F8FD3F88040C4F34E3000E01846C4F3D5
:10287000C90243F6E07303EA401343EA82732B492B
:10288000C1F860321346013A002BF2D1431E0028F2
:10289000ECD1BFF34F8F4B6943F480334B61BFF3EF
:1028A0004F8FBFF36F8F00F01BFBFFF72DFFFFF77C
:1028B000E5FE00F071F900F0ABF91D4800F03CF8BE
:1028C000FFF7F4F8FFF7D6FE04464368012B14D057
:1028D000A368012B14D0E368012B14D02369012BCA
:1028E00014D06369012B14D02368012B14D0207EEF
:1028F0000028E5D0FFF7CEF8E2E7FFF7F3F8E7E7C7
:10290000FFF7FEF8E7E7FFF70BF9E7E7FFF718F93E
:10291000E7E7FFF725F9E7E7FFF7C4F8FDF754FE0F
:1029200002460B46034804F0D7FCE0E700ED00E068
:10293000A80B0024ACEA000808B5054B1860054B4D
:102940001868002302221946806804F039FF08BD88
:102950003C0A00241C000024022801D801207047F2
:1029600008B504F071F909230360002008BD0000D8
:1029700010B5013801280AD814464FF0FF3392B23F
:102980000748006803F07EFE40B9204610BD04F001
:102990005BF9092303604FF0FF30F7E70520F5E707
:1029A0003C0A0024022801D80020704708B504F032
:1029B0004BF9092303604FF0FF3008BD08B504F060
:1029C00043F9092303604FF0FF3008BD08B548B94B
:1029D0004FF0FF3301220848006803F0BBFE40B906
:1029E000012008BD04F030F9092303604FF0FF30E7
:1029F000F7E70520F5E700BF3C0A002408B50228E8
:102A000004D84FF400534B60002008BD04F01CF9BB
:102A100009230360F8E7000082B0074BD3F8F420E5
:102A200042F00202C3F8F420D3F8F43003F00203BA
:102A30000193019B02B0704700440258FEE7FEE795
:102A4000FEE7FEE7FEE770477047704708B500F005
:102A500075FA08BD08B5024802F0E8FD08BD00BFE0
:102A6000140B002408B5024802F0E0FD08BD00BFC9
:102A7000A80B00240120704708B504F0E5F81623E0
:102A800003604FF0FF3008BD08B54FF0FF31FFF78E
:102A9000F3FFFEE710B503460C4A0D490D480068E8
:102AA00040B10C4800680344521A934206D8094AC0
:102AB000136010BD0748084C0460F2E704F0C4F846
:102AC0000C2303604FF0FF30F3E700BF0000082441
:102AD00000040000400A0024880C0024244B1B68DA
:102AE00003F00F03062B06D8214A136823F00F03C7
:102AF00043F0070313601F4B1A6842F001021A608B
:102B000000221A6119681C4A0A401A60184B1B6897
:102B100013F0080F06D0164A136823F00F0343F092
:102B200007031360134B00229A61DA611A6213499A
:102B300099621349D962134919635A639963DA6335
:102B400019645A64196821F4802119601A660E4BC1
:102B50001A680E4B1340B3F1005F03D20C4B0122F5
:102B6000C3F808210B4B43F2D2021A60704700BF32
:102B700000200052004402587FEDF6EA00020202F3
:102B80000000FF01800201010010005C0000FFFF57
:102B9000008000510040005208B51A481A4B0360EB
:102BA0004FF4E133436000238360C36003610C2270
:102BB00042618361C36103624362836203F0BAFED0
:102BC00098B900210F4803F0F5FF88B900210D489E
:102BD00004F015F878B90B4803F0CDFF70B9012265
:102BE0000A49084803F078FF08BDFFF78BFDE8E7C6
:102BF000FFF788FDEAE7FFF785FDECE7FFF782FDC9
:102C0000EDE700BF140B002400100140440A00242B
:102C100008B51A481A4B03604FF4E13343600023B0
:102C20008360C36003610C2242618361C3610362FC
:102C30004362836203F07EFE98B900210F4803F0DF
:102C4000B9FF88B900210D4803F0D9FF78B90B48C6
:102C500003F091FF70B901220A49084803F03CFFD4
:102C600008BDFFF74FFDE8E7FFF74CFDEAE7FFF788
:102C700049FDECE7FFF746FDEDE700BFA80B002498
:102C800000480040440A002410B5BAB004460021B0
:102C900035913691379138913991C02204A804F0CA
:102CA000BDFA23683E4A934204D03E4A93423CD048
:102CB0003AB010BD01220023CDE9042304A801F09D
:102CC000DDFC78BB384BD3F8F02042F01002C3F89B
:102CD000F020D3F8F02002F010020092009AD3F80E
:102CE000E02042F00102C3F8E020D3F8E03003F026
:102CF00001030193019B4FF4C06335930223369384
:102D00000024379438940723399335A9274800F0D5
:102D10006FFC22462146252000F03AF9252000F0DC
:102D20006DF9C5E7FFF7EEFCCCE702220023CDE901
:102D3000042304A801F0A2FC78BB1B4BD3F8E820C5
:102D400042F48022C3F8E820D3F8E82002F480227D
:102D50000292029AD3F8E02042F00202C3F8E02087
:102D6000D3F8E03003F002030393039B4FF4406376
:102D700035930223369300243794389407233993EC
:102D800035A90B4800F034FC22462146272000F0EC
:102D9000FFF8272000F032F98AE7FFF7B3FCCCE711
:102DA0000010014000480040004402580000025852
:102DB0000004025808B502681A4B9A4200D008BDB8
:102DC000194A1388B2F90020002A09DB13F4804F56
:102DD00011D0164A12780A2A08D0134B00221A8002
:102DE00001221249124803F077FEE8E7114A1A431C
:102DF0000D4B1A80F4E70D4A12780D2A0DD0C3F35B
:102E00000D010D48425401339BB2074A1380C72B72
:102E1000E6D9134600221A80E2E743F48043024ACF
:102E20001380DDE700480040100B0024440A002412
:102E3000A80B00240080FFFF480A0024DFF834D0EC
:102E4000FFF74CFE0C480D490D4A002302E0D45810
:102E5000C4500433C4188C42F9D30A4A0A4C0023E4
:102E600001E013600432A242FBD303F0F3FEFFF74C
:102E7000D3FC70470000082400000024CC09002483
:102E800000F10008CC090024880C0024FEE70000B3
:102E9000104B1B780BB90120704710B504464FF456
:102EA0007A70B0FBF3F30C4A1068B0FBF3F000F05B
:102EB000B3F868B90F2C01D901200AE0002221469D
:102EC0004FF0FF3000F064F8044B1C60002000E07D
:102ED000012010BD140000240C0000241800002460
:102EE00010B5032000F042F801F020F80F498B697B
:102EF000C3F303230E4AD35C03F01F03D8408B694E
:102F000003F00F03D35C03F01F0320FA03F3094A15
:102F10001360094B18600F20FFF7BAFF10B10124AE
:102F2000204610BD0446FFF777FDF9E7004402583C
:102F3000C0EA0008100000240C000024034B1B789A
:102F4000034A11680B441360704700BF140000244B
:102F50003C0C0024014B1868704700BF3C0C002457
:102F6000014B1868000C70470010005C0649CB68E4
:102F700023F4E0631B041B0C000200F4E060034335
:102F8000024A1A43CA60704700ED00E00000FA05EB
:102F900000B5174BDB68C3F30223C3F1070CBCF188
:102FA000040F28BF4FF0040C03F1040EBEF1060F0E
:102FB00014D9033B4FF0FF3E0EFA0CFC21EA0C0142
:102FC00099400EFA03F322EA03031943002807DBB2
:102FD0000901C9B2074B19545DF804FB0023E9E766
:102FE00000F00F000901C9B2034B1954F4E700BF08
:102FF00000ED00E000E400E014ED00E0002807DB55
:1030000000F01F02400901239340024A42F8203099
:10301000704700BF00E100E00138B0F1807F0BD2C3
:103020004FF0E0235861054AF02182F82310002078
:10303000986107221A6170470120704700ED00E097
:1030400070B50446FFF786FF002C00F0918105461D
:1030500094F83530DBB2022B06D080236365002361
:1030600084F83430012070BD23688C498C4A934227
:1030700018BF8B4230D0183293422DD01832934271
:103080002AD01832934227D01832934224D01832D3
:10309000934221D0183293421ED002F556729342C9
:1030A0001AD01832934217D01832934214D01832E3
:1030B000934211D0183293420ED0183293420BD063
:1030C0001832934208D01832934205D01A6822F081
:1030D0000E021A60266809E01A6822F01E021A60C1
:1030E0002268536923F080035361266823686B4983
:1030F0006B4A934218BF8B4242D0183293423FD062
:10310000183293423CD01832934239D0183293424D
:1031100036D01832934233D01832934230D002F571
:10312000567293422CD01832934229D018329342CF
:1031300026D01832934223D01832934220D018322E
:1031400093421DD0183293421AD01832934217D0AE
:10315000544A934214D01432934211D01432934201
:103160000ED0143293420BD01432934208D0143252
:10317000934205D01432934202D01432934204D1C8
:10318000226E136823F48073136023684349444A12
:10319000934218BF8B422FD0183293422CD0183252
:1031A000934229D01832934226D01832934223D02A
:1031B0001832934220D0183293421DD002F5567235
:1031C000934219D01832934216D01832934213D03A
:1031D0001832934210D0183293420DD018329342D5
:1031E0000AD01832934207D01832934204D01A689A
:1031F00022F001021A6003E01A6822F001021A604C
:10320000336813F0010F0ED0FFF7A4FE431B052B0C
:10321000F6D920236365032384F83530002384F82E
:10322000343001201FE723681C491D4A934218BF10
:103230008B4239D01832934236D01832934233D071
:103240001832934230D0183293422DD01832934224
:103250002AD01832934227D002F55672934223D0D7
:103260001832934220D0183293421DD01832934224
:103270001AD01832934217D01832934214D0183211
:10328000934211D0183293420ED0A16DE36D03F03A
:103290001F02012393404B600DE000BF100002406D
:1032A0002800024008540258A16DE36D03F01F028C
:1032B0003F2393408B6023682E492F4A934218BFC7
:1032C0008B4242D0183293423FD0183293423CD0C6
:1032D0001832934239D01832934236D01832934282
:1032E00033D01832934230D002F5567293422CD02C
:1032F0001832934229D01832934226D01832934282
:1033000023D01832934220D0183293421DD0183265
:1033100093421AD01832934217D0184A934214D0CD
:103320001432934211D0143293420ED0143293428D
:103330000BD01432934208D01432934205D0143289
:10334000934202D0143293420BD1636EA26E5A6044
:10335000E36E33B11A6822F480721A60236F626FD1
:103360005A60012384F83530002084F834007AE66E
:10337000012078E61000024028000240085402585C
:10338000002800F0298108B5024690F83530DBB2FC
:10339000022B03D080234365012008BD03689048B9
:1033A00090498B4218BF83420CBF0121002166D097
:1033B0003030834263D01830834260D0183083426B
:1033C0005DD0183083425AD01830834257D018301D
:1033D000834254D000F55670834250D01830834257
:1033E0004DD0183083424AD01830834247D018302D
:1033F000834244D01830834241D0183083423ED0BB
:10340000183083423BD0196821F00E01196013680F
:10341000A0F5956073498B4218BF83426AD0724908
:103420008B4267D018318B4264D018318B4261D007
:1034300018318B425ED018318B425BD018318B42F1
:1034400058D001F556718B4254D018318B4251D06F
:1034500018318B424ED018318B424BD018318B42F1
:1034600048D018318B4245D018318B4242D01831A8
:103470008B423FD0196821F0010119603EE0042021
:1034800082F8350081BB584A93422DD018329342BE
:103490002AD01832934227D01832934224D01832BF
:1034A000934221D0183293421ED002F556729342B5
:1034B0001AD01832934217D01832934214D01832CF
:1034C000934211D0183293420ED0183293420BD04F
:1034D0001832934208D01832934205D01A6822F06D
:1034E00001021A60002058E71A6822F001021A60EF
:1034F000002052E7196821F001011960136838486B
:1035000038498B4218BF834242D018318B423FD09A
:1035100018318B423CD018318B4239D018318B4254
:1035200036D018318B4233D018318B4230D001F570
:1035300056718B422CD018318B4229D018318B42D6
:1035400026D018318B4223D018318B4220D018312D
:103550008B421DD018318B421AD018318B4217D0B4
:1035600022498B4214D014318B4211D014318B423A
:103570000ED014318B420BD014318B4208D0143151
:103580008B4205D014318B4202D014318B4217D1BB
:10359000116E0B6823F480730B60906DD36D03F094
:1035A0001F0101238B404360536E916E5960D36EAF
:1035B00033B1196821F480711960136F516F59602C
:1035C000012382F83530002382F83430136D2BB19B
:1035D000104698470020E0E6012070470020DCE616
:1035E00010000240280002404000024008540258E7
:1035F00070B582B000236EE085685E000324B4409D
:1036000025EA0405CC68B4402C438460446824EA6D
:103610000C0C4C68C4F300149C4044EA0C04446055
:103620006CE0DD08083550F8256003F007044FEA28
:10363000840C0F2404FA0CF426EA040E0C6904FA34
:103640000CF444EA0E0440F825406FE0092400E041
:10365000002404FA0EF42C430CF1020C6B4D45F8D7
:103660002C404FF0B0442568D44325EA0206D1F837
:1036700004C01CF4801F01D042EA05064FF0B0459B
:103680002E606D6804EA0506D1F804C01CF4001F22
:1036900001D042EA05064FF0B0456E60D5F884507F
:1036A00004EA0506D1F804C01CF4003F01D042EA48
:1036B00005064FF0B045C5F88460D5F880502C4021
:1036C0004E6816F4803F01D042EA05044FF0B04244
:1036D000C2F8804001330A6832FA03F400F09380A4
:1036E0004FF0010C0CFA03FC1CEA0202F2D04C6809
:1036F00004F00304013C012C7FF67EAF4C6804F01B
:103700000304032C0CD0C4685D004FF0030C0CFACA
:1037100005FC24EA0C0C8C68AC4044EA0C04C46040
:103720004C6804F00304022C3FF47BAF04684FEABA
:10373000430E4FF0030C0CFA0EFC24EA0C0C4C6800
:1037400004F0030404FA0EF444EA0C0404604C6828
:1037500014F4403FBED02E4CD4F8F45045F002058E
:10376000C4F8F450D4F8F44004F002040194019C2D
:103770004FEA930C0CF10205244C54F8255003F049
:1037800003044FEA840E0F2404FA0EF425EA04051C
:10379000204CA0423FF45CAF04F58064A04222D0EC
:1037A00004F58064A04220D004F58064A0421ED0BD
:1037B00004F58064A0421CD004F58064A0421AD0B5
:1037C00004F58064A04218D004F58064A04216D0AD
:1037D00004F58064A04214D004F58064A0423FF454
:1037E00035AF0A2435E7012433E7022431E7032407
:1037F0002FE704242DE705242BE7062429E70724D7
:1038000027E7082425E702B070BD00BF0004005878
:1038100000440258000002580AB18161704709044F
:1038200081617047134BDB6813F0040F07D1114B14
:10383000DB6803F0070383421AD00120704710B5FC
:103840000C4AD36823F007031843D060FFF782FBCC
:103850000446084B5B6813F4005F07D1FFF77AFB5F
:10386000001BB0F57A7FF4D9012000E0002010BDE4
:103870000020704700480258002800F0398338B50E
:103880000446036813F0010F25D0944A136903F02E
:103890003803926A102B15D0182B0FD06368B3F53C
:1038A000803F3FD0002B53D18C4B1A6822F48032DA
:1038B0001A601A6822F480221A6038E002F00302CB
:1038C000022AEBD1854B1B6813F4003F03D06368D9
:1038D000002B00F00F83236813F0020F00F0A1808B
:1038E0007E4A1369926A13F038035AD0182B55D0C8
:1038F000E368002B00F0DE8078490A6822F01902A4
:1039000013430B60FFF726FB0546744B1B6813F04F
:10391000040F40F0AD80FFF71DFB401B0228F4D9D7
:103920000320EEE26D4A136843F48033136063684A
:103930002BB3FFF70FFB0546684B1B6813F4003FE2
:10394000C9D1FFF707FB401B6428F5D90320D8E253
:10395000B3F5A02F09D0614B1A6822F480321A60A7
:103960001A6822F480221A60E1E75C4B1A6842F47C
:1039700080221A601A6842F480321A60D7E7FFF793
:10398000E9FA0546554B1B6813F4003FA3D0FFF737
:10399000E1FA401B6428F5D90320B2E212F0030FCC
:1039A000A6D14E4B1B6813F0040F03D0E368002B25
:1039B00000F0A282494A136823F01903E1680B431F
:1039C0001360FFF7C7FA0546444B1B6813F0040F5A
:1039D00006D1FFF7BFFA401B0228F5D9032090E279
:1039E000FFF7BEFA41F20303984212D82269402A37
:1039F00007D03A494B6823F47C3343EA02334B60E7
:103A00000FE0364A536823F47C3343F400335360A9
:103A100007E0324A536823F0FE43216943EA016319
:103A20005360236813F0100F00F088802B4A13694D
:103A300003F03803926A082B56D0182B50D0E36954
:103A4000002B00F0B880254A136843F08003136010
:103A5000FFF780FA0546214B1B6813F4807F40F086
:103A60008880FFF777FA401B0228F4D9032048E248
:103A7000FFF776FA41F20303984212D82269402AEE
:103A800007D016494B6823F47C3343EA02334B607A
:103A9000C7E7124A536823F47C3343F4003353607E
:103AA000BFE70E4A536823F0FE43216943EA0163EE
:103AB0005360B6E7094A136823F001031360FFF768
:103AC00049FA0546054B1B6813F0040FA9D0FFF710
:103AD00041FA401B0228F5D9032012E200440258A3
:103AE00002F00302012AAAD1A14B1B6813F4807FC4
:103AF00003D0E369802B40F00182FFF731FA41F2F5
:103B00000303984212D8226A202A07D098494B68AA
:103B100023F0F84343EA82634B600FE0944A536812
:103B200023F0F84343F08043536007E0904AD368A2
:103B300023F07C53216A43EA0163D360236813F0C6
:103B4000080F60D06369002B49D0894A536F43F056
:103B500001035367FFF7FEF90546854B5B6F13F0D2
:103B6000020F50D1FFF7F6F9401B0228F5D90320C8
:103B7000C7E1FFF7F5F941F20303984212D8226A30
:103B8000202A07D07A494B6823F0F84343EA82633E
:103B90004B60D3E7764A536823F0F84343F0804301
:103BA0005360CBE7724AD36823F07C53216A43EA1F
:103BB0000163D360C2E76E4A136823F08003136089
:103BC000FFF7C8F905466A4B1B6813F4807FB5D030
:103BD000FFF7C0F9401B0228F5D9032091E1644AA0
:103BE000536F23F001035367FFF7B4F90546604BA9
:103BF0005B6F13F0020F06D0FFF7ACF9401B0228F1
:103C0000F5D903207DE1236813F0200F29D0A369A3
:103C10009BB1574A136843F480531360FFF79AF936
:103C20000546534B1B6813F4005F1AD1FFF792F956
:103C3000401B0228F5D9032063E14D4A136823F4A1
:103C400080531360FFF786F90546494B1B6813F450
:103C5000005F06D0FFF77EF9401B0228F5D903204C
:103C60004FE1236813F0040F21D1636A002B00F0A9
:103C700047813F4A126902F03802182A00F0EE80AC
:103C8000022B79D03A4A136823F080731360FFF750
:103C900061F90446364B1B6813F0007F00F0DC80AE
:103CA000FFF758F9001B0228F4D9032029E1314A13
:103CB000136843F480731360FFF74CF905462D4BEE
:103CC0001B6813F4807F06D1FFF744F9401B64287A
:103CD000F5D9032015E1A368012B0AD00BBB244BB7
:103CE0001A6F22F001021A671A6F22F004021A6793
:103CF00004E01F4A136F43F001031367A36833B353
:103D0000FFF728F905461A4B1B6F13F0020FACD1D1
:103D1000FFF720F9401B41F288339842F3D9032082
:103D2000EFE0052B09D0124B1A6F22F001021A673F
:103D30001A6F22F004021A67E0E70D4B1A6F42F087
:103D400004021A671A6F42F001021A67D6E7FFF7FA
:103D500001F90546064B1B6F13F0020F85D0FFF7E4
:103D6000F9F8401B41F288339842F3D90320C8E0A8
:103D70000044025800480258694A136823F08073CF
:103D80001360FFF7E7F80546654B1B6813F0007FEB
:103D900006D0FFF7DFF8401B0228F5D90320B0E07A
:103DA0005F4B996A5F4A0A40A16AE06A41EA0011E2
:103DB0000A439A62226B013AC2F30802616B01392D
:103DC000490289B20A43A16B0139090401F4FE01D9
:103DD0000A43E16B0139090601F0FE410A431A6307
:103DE000DA6A22F00102DA62596B4F4A0A40A16C8A
:103DF00042EAC1025A63DA6A22F00C02216C0A43D9
:103E0000DA62DA6A22F00202616C0A43DA62DA6A82
:103E100042F48032DA62DA6A42F40032DA62DA6A52
:103E200042F48022DA62DA6A42F00102DA621A6847
:103E300042F080721A60FFF78DF80446384B1B6819
:103E400013F0007F06D1FFF785F8001B0228F5D993
:103E5000032056E0002054E0002052E0304A916AEE
:103E6000106B012B4ED001F00303A26A93424BD199
:103E7000C1F30511E36A994248D1C0F30802236BEC
:103E8000013B9A4244D1C0F34622636B013B9A4204
:103E900040D1C0F30642A36B013B9A423CD1C0F330
:103EA0000660E36B013B984238D11D4B5B6BC3F35B
:103EB000CC03A26C9A4201D1002022E0184AD36AB6
:103EC00023F00103D362FFF745F80546FFF742F8F8
:103ED000A842FBD0124A516B134B0B40A16C43EA32
:103EE000C1035363D36A43F00103D362002008E0A7
:103EF00001207047012004E0012002E0012000E0E1
:103F0000002038BD0120FCE70120FAE70120F8E796
:103F10000120F6E70120F4E70120F2E70120F0E7B5
:103F2000004402580CFCFFFF0700FFFFF8B57E4B72
:103F30001B6903F03803102B00F0F280182B10D00F
:103F400013B17A4C2046F8BD774B1B6813F0200F55
:103F500000F0E880744B1868C0F3C100744CC44092
:103F6000F0E7714B9D6A05F003059C6AC4F30514E4
:103F7000D86A00F001005B6BC3F3CC0303FB00F0D5
:103F8000FCF7F6FC0646002CDCD0012D76D0022D85
:103F900000F0A4800DB32046FCF7EAFC014665481A
:103FA000FCF7F2FD0446604B186BC0F30800FCF709
:103FB000DFFC05464FF064513046FCF731FD014609
:103FC0002846FCF725FC4FF07E51FCF721FC01460A
:103FD0002046FCF725FD044671E0534B1B6813F0A7
:103FE000200F29D0504F3B68C3F3C1035048D8403D
:103FF000FCF7BEFC05462046FCF7BAFC0146284605
:10400000FCF7C2FD0446386BC0F30800FCF7B0FCB7
:1040100005464FF064513046FCF702FD0146284644
:10402000FCF7F6FB4FF07E51FCF7F2FB0146204611
:10403000FCF7F6FC044642E02046FCF799FC0146FA
:104040003D48FCF7A1FD0446374B186BC0F3080050
:10405000FCF78EFC05464FF064513046FCF7E0FC5F
:1040600001462846FCF7D4FB4FF07E51FCF7D0FB0D
:1040700001462046FCF7D4FC044620E02046FCF72D
:1040800077FC01462B48FCF77FFD0446264B186B56
:10409000C0F30800FCF76CFC05464FF06451304655
:1040A000FCF7BEFC01462846FCF7B2FB4FF07E5100
:1040B000FCF7AEFB01462046FCF7B2FC04461A4B67
:1040C0001B6BC3F34623581CFCF752FC01462046E9
:1040D000FCF75AFDFCF7F4FD044633E72046FCF7F5
:1040E00047FC01461548FCF74FFD04460E4B186B84
:1040F000C0F30800FCF73CFC05464FF06451304625
:10410000FCF78EFC01462846FCF782FB4FF07E51FF
:10411000FCF77EFB01462046FCF782FC0446CEE716
:10412000074C0FE7024C0DE70044025800093D0020
:104130000090D0030024744A0024744C0024F44AF4
:1041400000127A00002800F0328170B50D46044656
:104150009B4B1B6803F00F038B420BD2984A1368EA
:1041600023F00F030B431360136803F00F038B421C
:1041700040F01F81236813F0040F0CD02269914B8B
:104180009B6903F070039A4205D98E498B6923F02D
:1041900070031A438A61236813F0080F0CD0626918
:1041A000884BDB6903F070039A4205D98549CB69D6
:1041B00023F070031A43CA61236813F0100F0CD068
:1041C000A269804BDB6903F4E0639A4205D97D491B
:1041D000CB6923F4E0631A43CA61236813F0200F0C
:1041E0000CD0E269774B1B6A03F070039A4205D941
:1041F00074490B6A23F070031A430A62236813F0B0
:10420000020F0CD0E2686F4B9B6903F00F039A42D8
:1042100005D96C498B6923F00F031A438A6123681F
:1042200013F0010F41D0674A936923F47063A168CA
:104230000B4393616368022B0AD0032B27D0012B19
:104240002CD0604A126812F0040F06D10120ADE0B4
:10425000126812F4003F00F0AE805A490A6922F059
:10426000070213430B61FEF775FE0646554B1B69AB
:1042700003F038036268B3EBC20F16D0FEF76AFE94
:10428000801B41F288339842F0D903208EE04D4ADA
:10429000126812F0007FE0D1012087E0494A1268DD
:1042A00012F4807FD9D1012080E0236813F0020F3F
:1042B0000CD0E268434B9B6903F00F039A4205D28E
:1042C00040498B6923F00F031A438A613C4B1B68FA
:1042D00003F00F03AB420AD9394A136823F00F03E6
:1042E0002B431360136803F00F03AB4265D12368BF
:1042F00013F0040F0CD02269324B9B6903F070035A
:104300009A4205D22F498B6923F070031A438A61C0
:10431000236813F0080F0CD062692A4BDB6903F0A5
:1043200070039A4205D22749CB6923F070031A43E0
:10433000CA61236813F0100F0CD0A269214BDB690E
:1043400003F4E0639A4205D21E49CB6923F4E0638B
:104350001A43CA61236813F0200F0CD0E269194B8D
:104360001B6A03F070039A4205D216490B6A23F0C8
:1043700070031A430A62FFF7D9FD12498B69C3F330
:104380000323114AD35C03F01F03D8408B6903F069
:104390000F03D35C03F01F0320FA03F30B4A1360EF
:1043A0000B4B18600B4B1868FEF772FD70BD0120B7
:1043B00070470120FAE70120F8E70120F6E700BF87
:1043C0000020005200440258C0EA000810000024F7
:1043D0000C0000241800002408B5FFF7A7FD0B4AC5
:1043E0009369C3F303230A49CB5C03F01F0320FA4C
:1043F00003F3926902F00F02885C00F01F0023FAB9
:1044000000F0044A1060044A136008BD00440258DA
:10441000C0EA0008100000240C00002408B5FFF7D3
:10442000DBFF054BDB69C3F30213044AD35C03F0E3
:104430001F03D84008BD00BF00440258C0EA00086E
:1044400008B5FFF7C9FF054BDB69C3F30223044A34
:10445000D35C03F01F03D84008BD00BF00440258DE
:10446000C0EA0008404B9B6A03F00303032B79D09A
:1044700070B505460E463C4A136823F0806313600E
:10448000FEF768FD0446384B1B6813F0006F06D03A
:10449000FEF760FD031B022BF5D9032070BD324BE4
:1044A0009A6A22F47C32296842EA01329A626A6886
:1044B000013AC2F30802A9680139490289B20A43E4
:1044C000E9680139090401F4FE010A432969013947
:1044D000090601F0FE410A439A63DA6A22F0C0023B
:1044E00069690A43DA62DA6A22F02002A9690A439A
:1044F000DA62DA6A22F01002DA62D96B1B4A0A40E9
:10450000E96942EAC102DA63DA6A42F01002DA6269
:10451000C6B91A46DB6A43F40023D362124A136811
:1045200043F080631360FEF715FD04460E4B1B68D5
:1045300013F0006F14D1FEF70DFD001B0228F5D912
:104540000320ABE7012E05D0074AD36A43F40013DA
:10455000D362E3E7044AD36A43F48013D362DDE70E
:1045600000209BE701207047004402580700FFFF2E
:10457000404B9B6A03F00303032B79D070B50546CB
:104580000E463C4A136823F080531360FEF7E2FCAA
:104590000446384B1B6813F0005F06D0FEF7DAFCC8
:1045A000031B022BF5D9032070BD324B9A6A22F00F
:1045B0007C72296842EA01529A626A68013AC2F33F
:1045C0000802A9680139490289B20A43E968013938
:1045D000090401F4FE010A4329690139090601F0C1
:1045E000FE410A431A64DA6A22F4406269690A43A6
:1045F000DA62DA6A22F40072A9690A43DA62DA6AD4
:1046000022F48072DA62596C1B4A0A40E96942EA74
:10461000C1025A64DA6A42F48072DA62C6B91A4692
:10462000DB6A43F48003D362124A136843F0805379
:104630001360FEF78FFC04460E4B1B6813F0005FFF
:1046400014D1FEF787FC001B0228F5D90320ABE745
:10465000012E05D0074AD36A43F08073D362E3E7A3
:10466000044AD36A43F40003D362DDE700209BE7EA
:1046700001207047004402580700FFFFF8B50446C8
:10468000036813F0006F30D0836EB3F5001F26D09F
:104690000ED8EBB1B3F5801F07D102210830FFF728
:1046A000E1FE054645B12E4621E0012635461EE0D5
:1046B000B3F5401F09D10025984A136D23F4401328
:1046C000A16E0B431365002611E0012635460EE06E
:1046D000924AD36A43F40033D3620025ECE7022107
:1046E0002830FFF745FF0546DCE7002635462368FE
:1046F00013F4807F14D0A36D042B32D8DFE803F0CD
:1047000003232A080800854AD36A43F40033D3629E
:1047100055BB824A136D23F00703A16D0B4313654C
:10472000236813F4007F31D0E36D802B4CD020D868
:10473000002B43D0402B19D1002104F10800FFF7D2
:1047400091FE05461AE0002104F10800FFF78AFEF9
:104750000546DDE7002104F12800FFF709FF0546C3
:10476000D6E701263546DBE72E46D9E70126354652
:104770000CE0C02B02D0B3F5807F1CD15DBB674A33
:10478000136D23F4E073E16D0B431365236813F499
:10479000806F46D0D4F8A830B3F5800F39D01FD839
:1047A0008BB3B3F5001F18D1002104F10800FFF707
:1047B00059FE05461AE001263546E7E7574AD36A0F
:1047C00043F40033D362D9E7002104F12800FFF756
:1047D000CFFE0546D2E72E46D8E70126354620E033
:1047E000B3F5C00F02D0B3F5000F09D1C5B94B4ADC
:1047F000936D23F46003D4F8A8100B43936510E085
:10480000012635460DE0454AD36A43F40033D362AE
:10481000ECE7002104F12800FFF7AAFE0546E5E7D2
:104820002E46236813F4006F24D0D4F8AC30B3F1D3
:10483000007F42D00ED8002B39D0B3F1807F06D153
:10484000002104F10800FFF70DFE054608E00126EF
:1048500035460FE0B3F1407F02D0B3F1806F23D132
:10486000002D31D12D4A936D23F0E063D4F8AC10C4
:104870000B439365236813F0007F2ED0E36C202B4D
:1048800040D026D833B1102B20D1244AD36A43F428
:104890000033D362002D3CD1204AD36C23F0300387
:1048A000E16C0B43D36418E001263546E2E71B4A6E
:1048B000D36A43F40033D362D2E7002104F1280025
:1048C000FFF756FE0546CBE72E46D3E701263546D1
:1048D00003E0302BDED001263546236813F4805FD9
:1048E0002DD0236EB3F5005F4FD019D8002B46D0E2
:1048F000B3F5805F0FD1002104F10800FFF7B2FD8E
:10490000054613E0022104F10800FFF7ABFD054660
:10491000C0E72E46E1E70126354610E00044025884
:10492000B3F5405F02D0B3F5804F25D1002D33D1D0
:10493000774A136D23F4E043216E0B43136523681C
:1049400013F4005F38D0636EB3F5003F53D028D81E
:1049500043B1B3F5803F21D1012104F10800FFF7F5
:1049600081FD0546002D4DD1694A136D23F4E023E6
:10497000616E0B4313651FE001263546DFE7644A8D
:10498000D36A43F40033D362D0E7002104F1280056
:10499000FFF7EEFD0546C9E72E46D0E7012635466E
:1049A0000AE0B3F5802FDDD0B3F5A02FDAD0B3F550
:1049B000403FD7D001263546236813F4804F31D0CD
:1049C000D4F8B030B3F1005F45D020D843B1B3F193
:1049D000805F19D1012104F10800FFF743FD05466E
:1049E000002D3FD14A4A936D23F0E043D4F8B01034
:1049F0000B43936516E0012104F12800FFF7B8FD91
:104A00000546AFE72E46D7E7012635460AE0B3F163
:104A1000804FE5D0B3F1A04FE2D0B3F1405FDFD0DB
:104A200001263546236813F4004F09D0236FB3F1F4
:104A3000805F19D0B3F1005F24D0D3B10126354691
:104A4000236813F0807F33D0A36C032B5BD8DFE89F
:104A500003F027225327012104F12800FFF788FDE6
:104A60000546BDE72E46DDE7294AD36A43F4003305
:104A7000D36275B9264A136D23F04053216F0B435F
:104A80001365DDE7012104F10800FFF7EBFC0546A3
:104A9000EFE72E46D4E71E4AD36A43F40033D362CD
:104AA000A5BB1B4AD36C23F00303A16C0B43D36457
:104AB000236813F4800F2DD1236813F0010F00F049
:104AC000A580E36F282B00F29F80DFE803F08D9D27
:104AD0009D9D9D9D9D9D879D9D9D9D9D9D9D969D23
:104AE0009D9D9D9D9D9D8D9D9D9D9D9D9D9D8D9D16
:104AF0009D9D9D9D9D9D8D00022104F10800FFF765
:104B0000B1FC0546CCE701263546D1E72E46CFE776
:104B100000440258914A136843F480731360FEF70F
:104B200019FA07468D4B1B6813F4807F05D1FEF7F9
:104B300011FAC01B6428F5D90325002D4AD1884BF2
:104B40001B6FD4F8B420534013F4407F0CD0844B37
:104B50001A6F22F44072196F41F480311967196F8E
:104B600021F4803119671A67D4F8B430B3F5807F27
:104B700015D08DBBD4F8B43003F44072B2F5407F49
:104B80001ED0774A136923F47C53136174490B6F69
:104B9000D4F8B420C2F30B0213430B678CE7FEF783
:104BA000D9F907466E4B1B6F13F0020FE1D1FEF7E8
:104BB000D1F9C01B41F288339842F3D90325D8E7D5
:104BC0006748026922F47C52664901EA13131343D1
:104BD0000361DBE72E466FE72E466DE7012104F106
:104BE0000800FFF73FFC0546E5B95D4A536D23F029
:104BF0003803E16F0B43536508E0012104F12800FD
:104C0000FFF7B6FC0546EFE701263546236813F0AB
:104C1000020F17D0A36F052B28D8DFE803F00B0590
:104C2000200B0B0B2E46F1E7012104F10800FFF7E2
:104C300019FC0546EDB94A4A536D23F00703A16FED
:104C40000B435365236813F0040F23D0D4F894303A
:104C5000052B45D8DFE803F0150F3D15151501218B
:104C600004F12800FFF784FC0546E3E701263546FA
:104C7000E8E72E46E6E7012104F10800FFF7F2FB22
:104C8000054685BB364A936D23F00703D4F894108C
:104C90000B439365236813F0200F34D0D4F8903081
:104CA000B3F1005F4ED023D843B1B3F1805F1CD184
:104CB000002104F10800FFF7D5FB0546002D48D17F
:104CC000274A536D23F0E043D4F890100B4353650B
:104CD00019E0012104F12800FFF74AFC0546D0E75E
:104CE00001263546D6E72E46D4E7012635460AE0AA
:104CF000B3F1804FE2D0B3F1A04FDFD0B3F1405F0A
:104D0000DCD001263546236813F0400F37D0D4F8A5
:104D10009C30B3F5006F53D026D843B1B3F5806F04
:104D200019D1002104F10800FFF79CFB0546002D76
:104D30004DD10B4A936D23F4E053D4F89C100B43F0
:104D400093651CE0022104F12800FFF711FC0546E1
:104D5000B4E72E46D7E70126354610E00048025852
:104D600000440258CFFFFF00B3F5805FDFD0B3F5FA
:104D7000A05FDCD0B3F5406FD9D00126354623685B
:104D800013F0800F33D0D4F8A030B3F5804F00F08B
:104D9000A38021D843B1B3F5005F1AD1002104F1FB
:104DA0000800FFF75FFB0546002D40F09C80814A1C
:104DB000936D23F46043D4F8A0100B43936516E081
:104DC000022104F12800FFF7D3FB0546AFE72E468A
:104DD000D5E7012635460AE0B3F5004FE4D0B3F538
:104DE000204FE1D0B3F5C04FDED001263546236811
:104DF00013F0080F0CD0D4F88430B3F5805F74D072
:104E00006C4A536D23F44053D4F884100B4353651C
:104E1000236813F0100F0CD0D4F89830B3F5807FCE
:104E20006CD0644A936D23F44073D4F898100B430C
:104E30009365236813F4002F0BD0D4F8A430B3F596
:104E4000803F74D0B3F5003F67D0002B5FD00126C0
:104E50003546236813F4802F0CD0D4F88830B3F58E
:104E6000001F7CD0B3F5401F6FD0B3F5801F67D013
:104E700001263546236813F4803F08D0236D002BAC
:104E800076D0B3F5803F00F0818001263546236857
:104E900013F0005F40F08380236813F4003F00F0BC
:104EA0008E80D4F88030B3F5807F00F0EC8040F243
:104EB0008380B3F5007F03D0B3F5407F40F0E180FD
:104EC000002D40F0E6803B4A536D23F44073D4F844
:104ED00080100B43536572E0022104F12800FFF7B4
:104EE00047FB054660E72E4681E7022104F12800D2
:104EF000FFF73EFB002883D0012681E7022104F161
:104F00002800FFF735FB00288BD0012689E7002118
:104F100004F10800FFF7A6FA05467DB9254A936D0E
:104F200023F44033D4F8A4100B43936591E7022196
:104F300004F12800FFF71CFB0546EEE72E4688E744
:104F40001C4AD36A43F40033D3627DB9194A536DC6
:104F500023F44013D4F888100B4353658AE70121EA
:104F600004F12800FFF704FB0546EEE72E4681E733
:104F7000104AD36A43F40033D36275B90D4AD36C37
:104F800023F48033216D0B43D36480E7022104F1C5
:104F90000800FFF767FA0546EFE72E4677E702219C
:104FA00004F12800FFF7E4FA00283FF475AF01266A
:104FB00072E700BF00440258002B81D0012623680D
:104FC00013F4801F06D04F4A136D23F00043616F26
:104FD0000B431365236813F0805F07D0494A1369B8
:104FE00023F48043D4F8B8100B431361236813F4FF
:104FF000001F06D0434A136D23F08073E16E0B430C
:105000001365236813F0804F09D03E4B1A6922F4D0
:1050100000421A611A69D4F8BC100A431A61236865
:10502000002B06DA374AD36C23F04053616D0B43F3
:10503000D364236813F4000F07D0324A536D23F46E
:105040004003D4F88C100B435365636813F0010FD1
:1050500021D1636813F0020F26D1636813F0040FA7
:105060002BD1636813F0080F30D1636813F0100F71
:1050700035D1636813F0200F3AD106B101263046CE
:10508000F8BD01269BE71F4AD36A43F40033D3627D
:1050900016E72E4693E7002104F10800FFF7E2F936
:1050A0000028D6D00646D4E7012104F10800FFF716
:1050B000D9F90028D1D00646CFE7022104F1080033
:1050C000FFF7D0F90028CCD00646CAE7002104F14A
:1050D0002800FFF74DFA0028C7D00646C5E7012192
:1050E00004F12800FFF744FA0028C2D00646C0E7C2
:1050F000022104F12800FFF73BFA0028BDD0064644
:10510000BBE700BF0044025808B5FFF765F9054B3F
:105110001B6AC3F30213044AD35C03F01F03D84095
:1051200008BD00BF00440258C0EA00082DE9F04164
:105130000446864B9D6A9E6AC6F30536D86AC0F35C
:105140000010DB6BC3F3CC0303FB00F0FBF710FC98
:10515000002E00F0F58005F003050746012D79D0FB
:10516000022D00F0CB800DB33046FBF701FC014669
:105170007748FBF709FD0546744B986BC0F30800B0
:10518000FBF7F6FB06464FF064513846FBF748FC48
:1051900001463046FBF73CFB4FF07E51FBF738FBF6
:1051A00001462846FBF73CFC054674E0674B1B684C
:1051B00013F0200F2CD0DFF89481D8F80030C3F31F
:1051C000C1036448D840FBF7D3FB05463046FBF7E4
:1051D000CFFB01462846FBF7D7FC0546D8F8380038
:1051E000C0F30800FBF7C4FB06464FF06451384695
:1051F000FBF716FC01463046FBF70AFB4FF07E51E9
:10520000FBF706FB01462846FBF70AFC054642E091
:105210003046FBF7ADFB01464F48FBF7B5FC0546B2
:105220004A4B986BC0F30800FBF7A2FB06464FF011
:1052300064513846FBF7F4FB01463046FBF7E8FAC9
:105240004FF07E51FBF7E4FA01462846FBF7E8FBF6
:10525000054620E03046FBF78BFB01463C48FBF758
:1052600093FC0546394B986BC0F30800FBF780FBB5
:1052700006464FF064513846FBF7D2FB01463046F4
:10528000FBF7C6FA4FF07E51FBF7C2FA01462846FB
:10529000FBF7C6FB05462D4EB06BC0F34620FBF76F
:1052A00067FB4FF07E51FBF7B3FA01462846FBF748
:1052B0006BFCFBF705FD2060B06BC0F30640FBF70D
:1052C00057FB4FF07E51FBF7A3FA01462846FBF748
:1052D0005BFCFBF7F5FC6060B06BC0F30660FBF7AE
:1052E00047FB4FF07E51FBF793FA01462846FBF748
:1052F0004BFCFBF7E5FCA060BDE8F0813046FBF716
:1053000037FB01461548FBF73FFC05460F4B986BF2
:10531000C0F30800FBF72CFB06464FF064513846FB
:10532000FBF77EFB01463046FBF772FA4FF07E51E9
:10533000FBF76EFA01462846FBF772FB0546AAE723
:10534000002323606360A360D6E700BF00440258D7
:105350000024744A0090D0030024744C0024F44AC2
:105360002DE9F0410446864B9D6A9E6AC6F30556B8
:10537000D86AC0F300205B6CC3F3CC0303FB00F0DE
:10538000FBF7F6FA002E00F0F58005F0030507465E
:10539000012D79D0022D00F0CB800DB33046FBF704
:1053A000E7FA01467748FBF7EFFB0546744B186CAC
:1053B000C0F30800FBF7DCFA06464FF064513846AC
:1053C000FBF72EFB01463046FBF722FA4FF07E51E9
:1053D000FBF71EFA01462846FBF722FB054674E060
:1053E000674B1B6813F0200F2CD0DFF89481D8F89E
:1053F0000030C3F3C1036448D840FBF7B9FA05464F
:105400003046FBF7B5FA01462846FBF7BDFB0546DB
:10541000D8F84000C0F30800FBF7AAFA06464FF0A0
:1054200064513846FBF7FCFA01463046FBF7F0F9C9
:105430004FF07E51FBF7ECF901462846FBF7F0FAF6
:10544000054642E03046FBF793FA01464F48FBF72A
:105450009BFB05464A4B186CC0F30800FBF788FA23
:1054600006464FF064513846FBF7DAFA01463046FB
:10547000FBF7CEF94FF07E51FBF7CAF901462846FB
:10548000FBF7CEFA054620E03046FBF771FA0146FD
:105490003C48FBF779FB0546394B186CC0F3080014
:1054A000FBF766FA06464FF064513846FBF7B8FA48
:1054B00001463046FBF7ACF94FF07E51FBF7A8F9F7
:1054C00001462846FBF7ACFA05462D4E306CC0F37A
:1054D0004620FBF74DFA4FF07E51FBF799F9014654
:1054E0002846FBF751FBFBF7EBFB2060306CC0F369
:1054F0000640FBF73DFA4FF07E51FBF789F9014674
:105500002846FBF741FBFBF7DBFB6060306CC0F328
:105510000660FBF72DFA4FF07E51FBF779F9014653
:105520002846FBF731FBFBF7CBFBA060BDE8F08121
:105530003046FBF71DFA01461548FBF725FB0546EB
:105540000F4B186CC0F30800FBF712FA06464FF039
:1055500064513846FBF764FA01463046FBF758F9C8
:105560004FF07E51FBF754F901462846FBF758FAF5
:105570000546AAE7002323606360A360D6E700BF67
:10558000004402580024744A0090D0030024744C54
:105590000024F44A026852E8003F23F4907342E882
:1055A00000310029F6D1026802F1080353E8001F18
:1055B0000D4B0B40083242E800310029F3D1C36E95
:1055C000012B06D02023C0F88C300023C36643672C
:1055D0007047026852E8003F23F0100342E80031B0
:1055E0000029F6D1EEE700BFFEFFFFEF704708B5D8
:1055F000026852E8003F23F0400342E800310029EE
:10560000F6D12023C0F8883000238367FFF7EEFF30
:1056100008BD704708B5806B0023A0F85E30A0F885
:105620005630FFF7F6FF08BD7047000070B504461E
:105630000168CB6908688D6840F60F021A4008D1EE
:1056400013F0200F05D010F0200F34D115F0805F3B
:1056500031D12AB18B4A2A4033D18B4E304230D1DE
:10566000E26E012A00F0C68013F4801F03D015F407
:10567000800F40F09B8113F0800F07D010F0800F57
:1056800040F09B8115F4000F40F0978113F0400F1C
:1056900003D010F0400F40F0978113F4000F03D0B7
:1056A00010F0804F40F0948113F0807F02D00028EA
:1056B000C0F2928170BD636F002BFBD020469847EB
:1056C000F8E713F0010F09D010F4807F06D001260F
:1056D0000E62D4F890103143C4F8901013F0020F0A
:1056E0000BD015F0010F08D0216802260E62D4F805
:1056F000901041F00401C4F8901013F0040F0BD087
:1057000015F0010F08D0216804260E62D4F890101D
:1057100041F00201C4F8901013F0080F0BD010F004
:10572000200F00D13AB1226808211162D4F89020EC
:105730000A43C4F8902013F4006F0CD010F0806F6F
:1057400009D022684FF400611162D4F8902042F031
:105750002002C4F89020D4F89020002AAAD013F098
:10576000200F09D010F0200F02D115F0805F03D078
:10577000636F0BB120469847D4F8902023689B684C
:1057800013F0400F02D112F0280F2CD02046FFF763
:1057900001FF23689B6813F0400F20D0226802F1BC
:1057A000080353E8003F23F04003083242E8003189
:1057B0000029F3D1D4F880306BB1344A1A65D4F89B
:1057C0008000FDF7DDFD00283FF474AFD4F88000C1
:1057D000036D98476EE72046FFF71BFF6AE72046F8
:1057E000FFF717FF66E72046FFF713FF0023C4F813
:1057F00090305FE713F0100F3FF436AF10F0100F4A
:105800003FF432AF10230B6223689B6813F0400F04
:1058100000F09280D4F8802013681D481D498B4207
:1058200018BF834238D018318B4235D018318B42A3
:1058300032D018318B422FD018318B422CD01831F6
:105840008B4229D018318B4226D001F556718B42FC
:1058500022D018318B421FD018318B421CD0183106
:105860008B4219D018318B4216D018318B4213D08D
:1058700018318B4210D018318B420DD05B689BB22F
:105880000CE000BF010000102001000415560008C4
:1058900010000240280002405B689BB2002B3FF4DE
:1058A00009AFB4F85C1099427FF604AFA4F85E30FB
:1058B000D369B3F5807F32D0226852E8003F23F4E9
:1058C000807342E800310029F6D1226802F1080312
:1058D00053E8003F23F00103083242E80031002979
:1058E000F3D1226802F1080353E8003F23F040039C
:1058F000083242E800310029F3D12023C4F88C306B
:105900000023E366226852E8003F23F0100342E8D8
:1059100000310029F6D1D4F88000FDF791FB022375
:105920002367B4F85C10B4F85E309BB2C91A89B230
:105930002046FFF779FEBDE6B4F85C10B4F85E309F
:105940009BB2C91A89B2B4F85E309BB2002B3FF407
:10595000B1AE00293FF4AEAE226852E8003F23F416
:10596000907342E800300028F6D1226802F1080363
:1059700053E8000F1A4B0340083242E80030002879
:10598000F3D12023C4F88C300023E36663672268D8
:1059900052E8003F23F0100342E800300028F6D11F
:1059A000022323672046FFF73FFE83E64FF4801370
:1059B0000B62204601F0DCF87CE6A36F002B3FF47D
:1059C00079AE2046984775E62046FFF710FE71E64F
:1059D000204601F0CFF86DE6204601F0CAF869E6EE
:1059E000FEFFFFEF08B5B0F86030D0F88C20222A17
:1059F00005D00268936943F00803936108BD02680B
:105A0000516ADBB2826D0B401370836D0133836585
:105A1000B0F85E309BB2013B9BB2A0F85E30B0F8AC
:105A20005E309BB2002BE9D1026852E8003F23F4BC
:105A3000907342E800310029F6D1026802F10803B0
:105A400053E8003F23F00103083242E80031002907
:105A5000F3D12023C0F88C30002343670367036829
:105A6000164A93420CD05B6813F4000F08D002680A
:105A700052E8003F23F0806342E800310029F6D16C
:105A8000C36E012B16D10023C366026852E8003FA3
:105A900023F0100342E800310029F6D10368DA69E7
:105AA00012F0100F01D010221A62B0F85C10FFF74C
:105AB000BBFDA3E7FDF77EF9A0E700BF000C00588F
:105AC00008B5B0F86020D0F88C30222B05D00268E1
:105AD000936943F00803936108BD03685B6A816DB5
:105AE00013400B80836D02338365B0F85E309BB248
:105AF000013B9BB2A0F85E30B0F85E309BB2002B49
:105B0000EAD1026852E8003F23F4907342E8003182
:105B10000029F6D1026802F1080353E8003F23F0A0
:105B20000103083242E800310029F3D12023C0F8F4
:105B30008C300023436703670368164A93420CD0F6
:105B40005B6813F4000F08D0026852E8003F23F0AE
:105B5000806342E800310029F6D1C36E012B16D1D3
:105B60000023C366026852E8003F23F0100342E8B6
:105B700000310029F6D10368DA6912F0100F01D064
:105B800010221A62B0F85C10FFF74EFDA4E7FDF793
:105B900011F9A1E7000C00582DE9F843B0F8606056
:105BA0000368DD69D3F80090D3F80880D0F88C2022
:105BB000222A05D09A6942F008029A61BDE8F8836A
:105BC0000446B0F8687008E0D4F89030002B4CD14F
:105BD000B4F85E309BB2002B4ED0002F00F09880BE
:105BE00015F0200F00F094802368596AF3B2A26D7B
:105BF0000B401370A36D0133A365B4F85E309BB204
:105C0000013B9BB2A4F85E302368DD6915F0070FF5
:105C1000DED015F0010F09D019F4807F06D00122E3
:105C20001A62D4F890301343C4F8903015F0020F84
:105C30000BD018F0010F08D0236802221A62D4F8A2
:105C4000903043F00403C4F8903015F0040FBBD03B
:105C500018F0010FB8D0236804221A62D4F89030EB
:105C600043F00203C4F89030AEE72046FFF7D1FCC2
:105C70000023C4F89030ABE7226852E8003F23F4D9
:105C8000807342E800310029F6D1226802F108034E
:105C900053E8001F304B0B40083242E80031002926
:105CA000F3D12023C4F88C30002363672367236873
:105CB0002A4A934203D05B6813F4000F06D1E36EC7
:105CC000012B0DD02046FDF775F886E7226852E8D3
:105CD000003F23F0806342E800310029F6D1EEE76F
:105CE0000023E366226852E8003F23F0100342E8F5
:105CF00000310029F6D12368DA6912F0100F01D0C3
:105D000010221A62B4F85C102046FFF78DFC64E79D
:105D1000B4F85E309BB2002B3FF450AFB4F868206B
:105D20009A427FF64BAF226802F1080353E8003F26
:105D300023F08053083242E800310029F3D1084BA8
:105D40006367226852E8003F43F0200342E80031D5
:105D50000029F6D132E700BFFEFFFFEF000C00582C
:105D6000E55900082DE9F843B0F860600368DD6983
:105D7000D3F80090D3F80880D0F88C20222A05D0E0
:105D80009A6942F008029A61BDE8F8830446B0F8C7
:105D9000687008E0D4F89030002B4BD1B4F85E3036
:105DA0009BB2002B4DD0002F00F0978015F0200FF4
:105DB00000F0938023685B6AA26D33401380A36D6B
:105DC0000233A365B4F85E309BB2013B9BB2A4F8EA
:105DD0005E302368DD6915F0070FDFD015F0010F85
:105DE00009D019F4807F06D001221A62D4F89030CD
:105DF0001343C4F8903015F0020F0BD018F0010FC8
:105E000008D0236802221A62D4F8903043F00403C9
:105E1000C4F8903015F0040FBCD018F0010FB9D0C1
:105E2000236804221A62D4F8903043F00203C4F8C5
:105E30009030AFE72046FFF7ECFB0023C4F890302A
:105E4000ACE7226852E8003F23F4807342E8003157
:105E50000029F6D1226802F1080353E8001F304BF5
:105E60000B40083242E800310029F3D12023C4F866
:105E70008C3000236367236723682A4A934203D048
:105E80005B6813F4000F06D1E36E012B0DD02046A2
:105E9000FCF790FF87E7226852E8003F23F0806319
:105EA00042E800310029F6D1EEE70023E3662268DC
:105EB00052E8003F23F0100342E800310029F6D1F8
:105EC0002368DA6912F0100F01D010221A62B4F8B8
:105ED0005C102046FFF7A8FB65E7B4F85E309BB284
:105EE000002B3FF451AFB4F868209A427FF64CAFD4
:105EF000226802F1080353E8003F23F08053083280
:105F000042E800310029F3D1074B6367226852E869
:105F1000003F43F0200342E800310029F6D133E787
:105F2000FEFFFFEF000C0058C15A000870B586B0A4
:105F30000446016883680269134342691343C269D6
:105F400013430868884A024013430B602268536871
:105F500023F44053E1680B435360A1692268834BEB
:105F60009A4201D0236A19439068814B03400B4346
:105F700093602268D36A23F00F03616A0B43D362F4
:105F800022687C4B9A4221D07B4B9A4200F08C8055
:105F90007A4B9A4200F0A280794B9A4200F0B58089
:105FA000784B9A4200F0C880774B9A4200F0F48018
:105FB000764B9A4200F01981754B9A4200F02C8181
:105FC0006A4B9A4200F03F81802333E0714B5B6D56
:105FD00003F03803282B65D8DFE813F029006400AC
:105FE0006400640064006400640064004D016400A7
:105FF0006400640064006400640064002B006400BA
:106000006400640064006400640064005E00640076
:106010006400640064006400640064006000640064
:106020006400640064006400640064006200012392
:1060300000E008234D498A4200F02F81E069B0F565
:10604000004F00F0AF81202B00F20782202B00F2DE
:106050005182DFE813F01E0224024F024F02270292
:106060004F024F024F022C024F024F024F024F02CB
:106070004F024F024F0231024F024F024F024F02B6
:106080004F024F024F024F024F024F024F024F0288
:106090004F024F024F023D021023CBE72023C9E7F6
:1060A0004023C7E78023C5E73A4B5B6D03F0070346
:1060B000052B11D8DFE813F00600E10008000A0004
:1060C0000C000E000023B5E70823B3E71023B1E767
:1060D0002023AFE74023ADE78023ABE72D4B5B6D7B
:1060E00003F00703052B0ED8DFE803F003C905070B
:1060F000090B00239EE708239CE710239AE720233F
:1061000098E7402396E7802394E7224B5B6D03F0EA
:106110000703052B0ED8DFE803F003B40507090BCE
:10612000002387E7082385E7102383E7202381E7FF
:1061300040237FE780237DE7164B5B6D03F0070369
:10614000052B0ED8DFE803F0039F0507090B00239A
:1061500070E708236EE710236CE720236AE74023EB
:1061600068E7802366E700BFF369FFCF000C0058A3
:10617000FFF4FF11001001400044004000480040BF
:10618000004C0040005000400014014000780040E6
:10619000007C0040004402587D4B5B6D03F03803E7
:1061A000282B20D8DFE803F0151F1F1F1F1F1F1FFC
:1061B000711F1F1F1F1F1F1F171F1F1F1F1F1F1FA5
:1061C000191F1F1F1F1F1F1F1B1F1F1F1F1F1F1FE9
:1061D0001D0001232EE708232CE710232AE72023A4
:1061E00028E7402326E7802324E7694B5B6D03F013
:1061F0000703052B0ED8DFE803F0034A0507090B58
:10620000002317E7082315E7102313E7202311E7DE
:1062100040230FE780230DE75D4B5B6D03F0070321
:10622000052B0ED8DFE803F003350507090B002323
:1062300000E70823FEE61023FCE62023FAE64023CD
:10624000F8E68023F6E603F50E339B6D03F00703B3
:10625000052B0ED8DFE803F0031F0507090B022307
:10626000E8E60823E6E61023E4E62023E2E64023FE
:10627000E0E68023DEE60423DCE60423DAE60423FA
:10628000D8E60423D6E60423D4E60423D2E6042386
:10629000D0E60423CEE60423CCE6202B27D8022B1D
:1062A000C0F01A81023B1E2B00F21881DFE813F0C8
:1062B0005000160156001601160116015B0016016A
:1062C00016011601160116011601160160001601CD
:1062D0001601160116011601160116011601160106
:1062E0001601160116011601160116016C00402B4D
:1062F0002CD14FF40040626A264B33F81220B0FBD9
:10630000F2F3656805EB4501994200F2E980B3EBD1
:10631000053F00F2E780002633463146FAF7F0FCED
:10632000090241EA106100026B08C0182A46334690
:1063300041F10001FAF7E4FCA0F54072164B9A42D5
:1063400000F2D2802368D8603046D4E00120D2E049
:10635000FEF7DAFE0028CED10020CCE003A8FEF73D
:10636000E5FE0498F6E76846FEF7FAFF0198F1E7C4
:10637000074B1B6813F0200F08D0054B1B68C3F3B5
:10638000C1030648D840E5E70548B4E70348B2E74B
:1063900000440258D0EA0008FFFC0F000090D00330
:1063A00000093D00202B15D8202B00F29F80DFE84C
:1063B00003F031379D9D3A9D9D9D3F9D9D9D9D9DE7
:1063C0009D9D449D9D9D9D9D9D9D9D9D9D9D9D9D56
:1063D0009D9D5000402B1BD1626A4D4B33F812300B
:1063E000B0FBF3F06268530803EB4000B0FBF2F03F
:1063F000A0F110024FF6EF739A4279D883B223F0DE
:106400000F03C0F3420018432368D860002072E0F5
:10641000012070E0FEF702F80028DDD100206AE0DC
:10642000FEF70EF8F8E703A8FEF780FE0498F3E7FE
:106430006846FEF795FF0198EEE7364B1B6813F0B0
:10644000200F08D0334B1B68C3F3C1033248D84038
:10645000E2E73248C0E73048BEE7402B17D14FF49F
:106460000040626A2A4B33F81230B0FBF3F06368E5
:1064700000EB5300B0FBF3F0A0F110024FF6EF7306
:106480009A4242D8236880B2D860002033E00120CD
:1064900031E0FDF7C3FF0028E3D100202BE0FDF73A
:1064A000CFFFF8E703A8FEF741FE0498F3E768463C
:1064B000FEF756FF0198EEE7164B1B6813F0200F0E
:1064C00008D0144B1B68C3F3C1031348D840E2E75C
:1064D0001248C6E71048C4E701200CE001200AE09A
:1064E000012008E0012006E0012004E0012002E094
:1064F000012000E001200123A4F86A30A4F86830EC
:1065000000236367A36706B070BD0120F3E700BFF7
:10651000D0EA0008004402580090D00300093D0072
:10652000836A13F0010F06D00268536823F4003326
:10653000C16A0B435360836A13F0020F06D00268EE
:10654000536823F48033016B0B435360836A13F069
:10655000040F06D00268536823F48023416B0B4379
:106560005360836A13F0080F06D00268536823F45F
:106570000043816B0B435360836A13F0100F06D006
:106580000268936823F48053C16B0B439360836A62
:1065900013F0200F06D00268936823F40053016CB7
:1065A0000B439360836A13F0400F0AD0026853686C
:1065B00023F48013416C0B435360436CB3F5801F8D
:1065C0000BD0836A13F0800F06D00268536823F45F
:1065D0000023C16C0B43536070470268536823F477
:1065E000C003816C0B435360EBE72DE9F84305468C
:1065F0000F4616469946DDF820802C68E46937EA94
:1066000004030CBF4FF0010C4FF0000CB44532D125
:10661000B8F1FF3FF1D0FCF79DFCA0EB090040452D
:106620002CD8B8F1000F2BD02B681A6812F0040F89
:10663000E3D0DA6912F0080F11D1DA6912F4006FB1
:10664000DBD04FF400621A622846FEF7A3FF202336
:10665000C5F89030002385F8843003200CE008242E
:106660001C622846FEF796FFC5F89040002385F887
:106670008430012000E00020BDE8F8830320FBE720
:106680000320F9E72DE9F04182B01E46D0F88830AA
:10669000202B5BD104460D469046002A18BF0029E6
:1066A00001D1012053E00023C0F890302123C0F82D
:1066B0008830FCF74FFC0746A4F85480A4F85680B5
:1066C000A368B3F5805F02D04FF0000816E023699D
:1066D00043B34FF0000811E02023C4F888300320B2
:1066E00035E038F8023B2268C3F308039362B4F83C
:1066F000562092B2013A92B2A4F85620B4F856301D
:106700009BB293B100963B46002280212046FFF7C2
:106710006CFF0028E0D1002DE3D015F8012B236891
:106720009A62E4E7A8460025E8E700963B46002287
:1067300040212046FFF759FF18B92023C4F88830BC
:1067400005E02023C4F88830032000E0022002B0D6
:10675000BDE8F0812DE9F04383B01E46D0F88C30BF
:10676000202B7ED104460D469046002A18BF0029F2
:1067700001D1012076E00023C0F890302222C0F839
:106780008C20C366FCF7E6FB0746A4F85C80A4F8FF
:106790005E80A368B3F5805F06D0A3B9226972B9A1
:1067A000FF22A4F8602014E0226922B940F2FF120F
:1067B000A4F860200DE0FF22A4F8602009E07F2209
:1067C000A4F8602005E0B3F1805F0AD00022A4F8AD
:1067D0006020B4F86080B3F5805F0CD04FF0000902
:1067E00024E022691AB97F22A4F86020F1E73F2251
:1067F000A4F86020EDE7236913B14FF0000915E01C
:10680000A946002512E02023C4F88C30032029E09B
:1068100023685A6A5FFA88F3134005F8013BB4F81D
:106820005E2092B2013A92B2A4F85E20B4F85E30D3
:106830009BB28BB100963B46002220212046FFF7F9
:10684000D4FE0028DFD1002DE2D123685B6A08EA7C
:10685000030329F8023BE2E72023C4F88C30002030
:1068600000E0022003B0BDE8F08330B583B00446F9
:106870000023C0F89030FCF76DFB054622681268D3
:1068800012F0080F10D123681B6813F0040F28D1F1
:106890002023C4F88830C4F88C300020E0662067DC
:1068A00084F8840003B030BD6FF07E43009303464C
:1068B00000224FF400112046FFF797FE0028E2D097
:1068C000226852E8003F23F0800342E800310029AB
:1068D000F6D12023C4F88830002384F884300320C4
:1068E000E0E76FF07E4300932B4600224FF48001D7
:1068F0002046FFF77AFE0028CAD0226852E8003FFF
:1069000023F4907342E800310029F6D1226802F1A5
:10691000080353E8003F23F00103083242E8003146
:106920000029F3D12023C4F88C30002384F884306C
:106930000320B7E778B310B50446D0F888300BB31E
:106940002423C4F888302268136823F001031360FD
:106950002046FFF7EBFA012813D0A36ABBB92268DF
:10696000536823F4904353602268936823F02A030A
:1069700093602268136843F0010313602046FFF719
:1069800074FF10BD80F88430FCF77EF9D8E720460C
:10699000FFF7C6FDE3E701207047000010B48165F2
:1069A000A0F85C20A0F85E20002343678368B3F55D
:1069B000805F06D0A3B9036973B9FF23A0F86030E4
:1069C00014E0036923B940F2FF13A0F860300DE032
:1069D000FF23A0F8603009E07F23A0F8603005E0D5
:1069E000B3F1805F2DD00023A0F860300023C0F801
:1069F00090302223C0F88C30016801F1080353E87D
:106A0000003F43F00103083141E80034002CF3D18A
:106A1000436EB3F1005F1ED08368B3F5805F42D050
:106A2000294B43670369002B43D0026852E8003FBB
:106A300043F4907342E800310029F6D1002010BCE5
:106A4000704703691BB97F23A0F86030CEE73F236E
:106A5000A0F86030CAE7B0F868309342DCD88368A9
:106A6000B3F5805F19D0194B4367036943B10268DE
:106A700052E8003F43F4807342E800310029F6D128
:106A8000026802F1080353E8003F43F080530832E4
:106A900042E800310029F3D1D0E70369002BE2D1AD
:106AA0000B4B4367E1E70369002BB9D1094B4367FF
:106AB000B8E7026852E8003F43F0200342E80031A3
:106AC0000029F6D1BAE700BFE5590008995B000834
:106AD000655D0008C15A000838B5D0F88C30202B0D
:106AE00019D1002A18BF002917D00023C3660368F4
:106AF0000B4CA3420CD05B6813F4000F08D0046861
:106B000054E8003F43F0806344E80035002DF6D19F
:106B1000FFF744FF00E0022038BD0120FCE700BF82
:106B2000000C0058436E2BB90123A0F86A30A0F87E
:106B30006830704730B403689A68C2F3426299685B
:106B4000490F094D6B5C1B01084C615C93FBF1F331
:106B5000A0F86A30AB5C1B01A25C93FBF2F3A0F8D7
:106B6000683030BC704700BFF0EA0008E8EA00086F
:106B700070477047704790F88430012B18D001237C
:106B800080F884302423C0F8883003681A681968B4
:106B900021F00101196022F00052002343660168D0
:106BA0000A602022C0F8882080F884301846704798
:106BB0000220704738B590F88430012B1DD0044670
:106BC000012380F884302423C0F8883003681D68CE
:106BD0001A6822F001021A600268936823F0604389
:106BE00019439160FFF79EFF23681D602023C4F8BE
:106BF0008830002084F8840038BD0220FCE738B5D6
:106C000090F88430012B1DD00446012380F8843095
:106C10002423C0F8883003681D681A6822F0010236
:106C20001A600268936823F0606319439160FFF76C
:106C300079FF23681D602023C4F88830002084F881
:106C4000840038BD0220FCE7014B1868704700BF84
:106C50001C00002470B50D4E0D4D761BB61006D0ED
:106C6000002455F8043B01349847A642F9D1094E57
:106C7000094D761B07F052FEB61006D0002455F8D9
:106C8000043B01349847A642F9D170BDF4F00008E6
:106C9000F4F00008FCF00008F4F00008024B014694
:106CA000186800F00BB800BF1C000024024B01461E
:106CB000186804F087BE00BF1C0000242DE9F04FC7
:106CC00001F10B06162E83B0044624D8102900F2D9
:106CD000BA8000F0F5FA102618220220B54F3A4487
:106CE000A2F1080153688B4200F0BA805A68D96853
:106CF00022F003021A449D68E9608D60516841F0FA
:106D000001012046516003F1080500F0DFFA284632
:106D100003B0BDE8F08F36F0070600F19480B14271
:106D200000F2918000F0CCFAB6F5FC7FC0F09A81B9
:106D3000730A00F08F80042B00F26F81B30903F116
:106D4000390003F1380CC3009A4F3B44A3F1080506
:106D50005B689D4206D10CE0002980F22781DB6848
:106D60009D4206D05A6822F00302911B0F29F3DDE1
:106D700060463D69DFF840C265457CD06A6822F014
:106D80000302931B0F2B00F37B81002BC7E904CC7C
:106D900080F26C81B2F5007F80F01A81D3087968A7
:106DA00001334FEA521E012202FA0EF20A4357F84B
:106DB00033E0C5F808E007EBC3010839E9607A6001
:106DC00047F83350CEF80C5083100121994091427E
:106DD00057D8114206D120F003004900114200F1BA
:106DE0000400FAD007EBC0094D468646D5F80C8062
:106DF000454508D11DE1002B80F22481D8F80C8094
:106E0000454500F01681D8F8042022F00302931BB8
:106E10000F2BF0DD2046D8E9025408EB060146F0BE
:106E20000106C8F80460EC60A56043F00104C7E9FE
:106E30000411C1E902CC4C6048F8023000F046FA77
:106E400008F1080502E00C2323600025284603B062
:106E5000BDE8F08F4FF4007340204FF03F0C73E714
:106E6000D3689A4208BF02307FF440AF3D69DFF833
:106E700048C1654582D17A688310012199409142C9
:106E8000A7D9BD686B6823F003094E4503D8A9EB69
:106E900006030F2B7ADCDFF824B1494BDBF8002026
:106EA0001B680132334405EB090A00F0338103F516
:106EB00080530F3323F47F6828F00F0841462046A3
:106EC00000F06CFC411C024600F0F380824500F2A9
:106ED000EE803C4B196841441960084600F04E8131
:106EE000DBF80010019301311BBFA2EB0A0A5044EA
:106EF000CBF80020186012F0070B00F01781CBF1DF
:106F000008010A44CBF5805190440831A1EB0801F7
:106F1000C1F30B0A51462046009200F03FFC421C90
:106F2000DDE9002300F04F81801A00EB0A081968A0
:106F3000BA6048F001005144BD425060196000F051
:106F40002981B9F10F0F40F227816868A9F10C0C73
:106F50002CF0070C00F0010040EA0C0068604FF0D4
:106F6000050E05EB0C00BCF10F0FC0E901EE00F2BD
:106F7000328150681546144B1A688A4238BF19602E
:106F8000124B1A688A4238BF196094E0AA1943F07C
:106F9000010346F001066E602046BA60536000F0BF
:106FA00095F90835284603B0BDE8F08FD9681A4432
:106FB000A1E600BF48040024500400245008002427
:106FC000700C0024400C0024680C00246C0C00247D
:106FD000B2F5206F4FEA522363D3142B00F2B7802F
:106FE00003F15C01C9005B3307EB010E7958AEF188
:106FF000080E8E4500F091804B6823F00303934206
:1070000002D989688E45F7D1D1F80CE07A68C5E9D4
:10701000021ECEF80850CD60D6E6142B59D9542B59
:1070200000F29D80330B03F16F0003F16E0CC3007F
:107030008AE60EF1010E1EF0030F05F108057FF43C
:10704000D5AE51E0424445465368D8F80C1043F0A1
:107050000103536055F8083F2046D9608B6000F06B
:1070600035F9F3E6F00806F1080237E62A4420462F
:10707000536843F001035360083500F027F9E5E653
:10708000A919204646F0010643F001046E60C7E9E5
:107090000411C1E902CC4C60AB5000F017F908357F
:1070A000D4E6930903F13901C90038339CE7BD42A6
:1070B0005FD0BD68686820F003084645A8EB06036A
:1070C00002D80F2B3FF762AF204600F0FFF80025F3
:1070D000BCE603F15C0003F15B0CC30034E659F835
:1070E00008394B4540F0968010F0030F00F1FF3057
:1070F000F5D17B6823EA01037B60490099423FF6A2
:10710000C0AE19B9BDE649000EF1040E1942FAD01D
:10711000704667E603F11008D0E69A104FF00108B8
:107120007B6808FA02F21A437A6070E702EB080102
:107130004942C1F30B0A51462046009200F02EFB53
:10714000431CDDE900237FF4EFAEDA46EFE6542B73
:1071500025D8130B03F16F01C9006E3344E7B3F573
:10716000AA7F25D8F30B03F1780003F1770CC30055
:10717000EAE5294B186840441860B1E6CAF30B0CE5
:10718000BCF1000F7FF4ACAEBD68C84448F001000C
:107190006860F0E61546EEE60123536094E7B3F528
:1071A000AA7F23D8D30B03F17801C90077331BE7FB
:1071B00040F25452934223D8B30C03F17D0003F103
:1071C0007C0CC300C0E5ABF1080BD844A8EB020867
:1071D0004FF0000AABE605F108012046009304F0E9
:1071E000F1FBBD68009B68681968C4E640F2545121
:1071F0008B420BD8930C03F17D01C9007C33F3E67D
:107200004FF47E737F204FF07E0C9DE54FF47E712E
:107210007E23E9E67B6870E7400C0024830730B5E5
:1072200048D0541E002A3FD0CAB2034601E0013CB8
:107230003AD303F8012B9D07F9D1032C2DD9CDB2F8
:1072400045EA05250F2C45EA054536D9A4F110027B
:1072500022F00F0C03F1200EE6444FEA121C03F15A
:10726000100242E9045542E9025510327245F8D144
:107270000CF1010214F00C0F03EB021204F00F0CDE
:1072800013D0ACF1040323F003030433134442F896
:10729000045B9342FBD10CF003042CB1CAB21C4432
:1072A00003F8012B9C42FBD130BD64461346002CF1
:1072B000F4D1F9E703461446BFE71A46A446E0E7CF
:1072C000014805F04BBA00BF780C0024014805F0D6
:1072D00047BA00BF780C00240FB400B5074983B04B
:1072E00004AB086853F8042B8168019301F06EFB2E
:1072F00003B05DF804EB04B0704700BF1C0000242D
:1073000070B5054688B008460C46FAF799F8224E43
:10731000AA6B059001214318CDE9066104A802215A
:1073200004940393AC680190029122B3636E13F04E
:10733000010FB4F90C309AB201D1980525D591040A
:1073400006D4626E43F4005322F40052A3816266B5
:10735000284601AA214604F03BFC636E002814BFB6
:107360004FF0FF350A25DA0702D4A3899B0506D51D
:10737000284608B070BD284604F02CFAD6E7A06D68
:1073800005F0EEF9284608B070BDA06D05F0E6F9ED
:10739000B4F90C309AB2D2E7B4E90008024B0146C6
:1073A0001868FFF7ADBF00BF1C00002410B4044CE8
:1073B00003460A46206810BC194600F003B800BF17
:1073C0001C0000242DE9F84F1746002900F0988092
:1073D00007F10B0580460C46FFF772FF162D5DD8AE
:1073E00010252A46AF425ED854F8041C21F003064B
:1073F0009642A4F1080962DABC4BD3F808C009EB45
:107400000600844500F09780D0F804C02CF00103FA
:1074100003445B68DB0768D42CF0030C06EB0C0319
:10742000934247DACB0710D454F8083CA9EB030A7F
:10743000DAF8043023F003018C44B444944580F21C
:1074400011817318934280F2E88039464046FFF775
:1074500035FC0746E0B154F8043C23F001034B44EB
:10746000A0F10802934200F0D280321F242A00F2D9
:10747000F580132A00F2AC80034622461168196099
:107480005168596092689A602146404604F09AFA21
:107490004046FFF71BFF3846BDE8F88F25F007058B
:1074A000002D2A469EDA0C23C8F800300027384603
:1074B000BDE8F88F1E46D0E90223D3609A60731BA3
:1074C0000F2B22D8D9F8043003F0010333434E4484
:1074D000C9F80430736843F00103736040462746DF
:1074E000FFF7F4FE3846BDE8F88FC907ADD454F86D
:1074F000083CA9EB030ADAF8041021F00301A0E725
:10750000BDE8F84F1146FFF7D9BBD9F8041001F0D8
:1075100001012943C9F8041009EB05014E4443F069
:1075200001034B60736843F0010308317360404608
:1075300004F048FAD2E7DCF8040020F0030B06EB75
:107540000B0C05F1100084454DDAC9073FF57DAFFE
:1075500054F8081CA9EB010ADAF8041021F0030121
:107560008B44B34458453FF76CAF5746DAF80C10DC
:1075700057F8080F321F242AC160886000F2DB80B0
:10758000132A40F2D6802168CAF808106168CAF848
:107590000C101B2A00F2DF8008340AF11002216867
:1075A000116061685160A16891600AEB0501ABEB65
:1075B000050242F0010299604A60DAF8043003F0F3
:1075C00001031D434046CAF80450FFF77FFE6EE7F3
:1075D00023680360636843601B2A68D804F10802CB
:1075E00000F108034AE709EB05029A60ACEB0503DA
:1075F00043F00103536054F8043C03F001031D43BE
:10760000404644F8045CFFF761FE27464FE750F818
:10761000043C23F003031E4451E75746DAF80C10EC
:1076200057F8080F321F242AC16088604CD8132AEB
:1076300048D92168CAF808106168CAF80C101B2ADA
:1076400056D808340AF110021E4623681360636896
:107650005360A3689360D1463C4630E7214605F06D
:107660004DF911E7D0E902135746CB60996057F8FE
:10767000081FDAF80C30CB60321F242A99602DD80D
:10768000132A29D92368CAF808306368CAF80C306D
:107690001B2A42D808340AF1100322681A60626873
:1076A0005A60A2689A606646D1463C4607E7A368DE
:1076B0008360E368C360242A26D004F1100200F13D
:1076C0001003DBE63A46BFE7214638461E46D14660
:1076D00005F014F93C46F2E63B46DEE72146384623
:1076E0006646D14605F00AF93C46E8E6480400241F
:1076F000A168CAF81010E168CAF81410242A20D032
:1077000010340AF118029FE723690361616941613E
:1077100004F1180200F11803B0E6A368CAF81030AB
:10772000E368CAF81430242A21D010340AF118036F
:10773000B3E73A4633E72146384605F0DFF8164B03
:1077400033E72269CAF818206269CAF81C20183485
:107750000AF1200278E7A168CAF81010E168CAF8B7
:107760001410242A0DD010340AF1180217E72369E7
:10777000CAF818306369CAF81C3018340AF12003BB
:107780008BE72269CAF818206269CAF81C201834ED
:107790000AF1200203E700BF4804002438B5074D72
:1077A0000022044608462A60FBF774F9431C00D007
:1077B00038BD2B68002BFBD0236038BD840C00241F
:1077C0002DE9F043694CD4F8008083B004460E469E
:1077D00017461D46B8F1000F03D0D8F83830002BFB
:1077E00077D0022F05D0012F00F2AC80002DC0F21F
:1077F000A980636EDA0752D52146404603F0B6FFF2
:10780000216B41B104F14003994202D0404604F09B
:10781000D9F800232363B4F90CC000231CF0800FB7
:10782000A361636064D12CF44A6C2CF0030C022F2A
:10783000A4F80CC06AD001AB6A462146404605F068
:1078400017F8A3891843A081002D2FD0002E2ED029
:10785000D8F83830002B38D0009B2660AB42B4F902
:107860000C301CBF43F40063A381012F04BF43F01D
:107870000103A3819AB213F00803C4E904652CD074
:10788000D1075DD56D42A561656E002315F0010538
:10789000A36027D00025284603B0BDE8F083A38964
:1078A0009B05A9D4A06D04F059FFA5E7009D2846CB
:1078B000FFF7F4F90646002847D0A38943F0800378
:1078C000A381D8F83830002BC6D1404603F082FFA0
:1078D000C2E7404603F07EFF83E7A360656E15F0C4
:1078E0000105D7D1930524D5284603B0BDE8F08320
:1078F0002169404604F066F8B4F90CC02CF44A6CD7
:107900002CF0030C022FA4F80CC094D10025002207
:1079100004F14303A2600122C4E904322360636ED0
:107920004CF0020CD807A4F80CC0DDD41CF4007F86
:10793000DAD1A06D04F014FF284603B0BDE8F0834F
:10794000A560CBE74FF0FF35CEE7DDF80090A94505
:1079500004D04846FFF7A2F9064620B9B4F90CC096
:107960004FF0FF35D3E74D46A7E700BF1C000024CA
:1079700010B50C46B1F90E1005F056FD002803DBDA
:10798000236D0344236510BDA38923F48053A38191
:1079900010BD00BF2DE9F0410C46B1F90C101F4697
:1079A000CB05054616460BD421F48051A1813B46F8
:1079B000B4F90E1032462846BDE8F04102F0B0BDE1
:1079C000B4F90E100223002204F0CCFEB4F90C101E
:1079D000EAE700BF10B50C46B1F90E1004F0C2FE84
:1079E000A389421C0EBF23F4805343F480532065C7
:1079F000A38110BDB1F90E1002F022BEA2B330B5C2
:107A000040EA0104A40784460B462AD09CF80000F3
:107A10000C7884422FD1012A0DD0E64660B11EF8C1
:107A2000010F11F8014F6FEA0E03A042134422D157
:107A30001CEB0303F2D1002030BD0468194653F853
:107A4000045BA4F1013EAC4284462EEA040E00F130
:107A500004000BD1043A84461946ECD01EF0803F56
:107A6000E9D1032AE9D8D1E7104670479CF8000015
:107A70000C78A042D1D0001B30BD00BF0000000038
:107A80002DE9F04F1C46984B1B68A1B0002581469C
:107A90001846884608921C950493F9F7D1FC0021FA
:107AA00083460020CDE90601CDF86C80424617469A
:107AB00012F8013B2D2B2FD8DFE813F0A1002E0088
:107AC0002E002E002E002E002E002E002E00AF00C5
:107AD000AF00AF00AF00AF002E002E002E002E0032
:107AE0002E002E002E002E002E002E002E002E0026
:107AF0002E002E002E002E002E002E00AF002E0095
:107B00002E002E002E002E002E002E002E002E0005
:107B10002E0006042E00FC0300220A92302B7ED099
:107B2000002209922F2B1C4640F233854FF0000AA9
:107B300038465646554612E00130082D1B90C8BF06
:107B40000AEB8A0A0478C6BF03EB4A03A3F1300AA2
:107B5000A2F130062F2C05F10105234670DD06EB5E
:107B60008602392C03EB4202E6DD04995A46FFF700
:107B700045FF0346002835D11B9A11465A441B92F3
:107B800011F80B40002D40F0AC85302C40F064859E
:107B9000C2F10101531801321B921478302CF9D034
:107BA000A4F13102082A00F23883A4F1300E1B9CA4
:107BB00003F1010B002301252746049306EB8606FB
:107BC0000EEB46060023621C1B926478A4F1300180
:107BD000092900F2ED8201338E46002940F0B88475
:107BE0001B9CF0E70023652C04959B469E4601D024
:107BF000452C32D1002D7CD1099A1A4378D1089BAB
:107C000013B1089BC3F800804FF0000BCDF810B003
:107C10000499584621B0BDE8F08F1B9247E77B7866
:107C200003F0DF03582B00F0748401371B973B7877
:107C3000302BFAD0002B00F0CC800122099271E7A2
:107C400004995A46FFF7DAFE0346002800F0D68072
:107C500004954FF0000B5B46DE4600220B92002D90
:107C600000F09380049A1346002A08BF2B46304642
:107C70000493F8F787FC0B460246CDE906230B9BDD
:107C8000102DA3EB0B032C46A8BF1024092D0E9337
:107C900013DD164B03EBC40353E91223F9F790FCF1
:107CA000CDE906015046F8F76DFC02460B46DDE9CA
:107CB0000601F8F72BFBCDE906010F2D00F3A78095
:107CC0000E9B002B00F018840E9B40F39283162B22
:107CD00040F3F9840E9AC5F12503934280F20C8596
:107CE0000E9B2C1B1C4498E0F4EE0008B8EF000833
:107CF0000025DDF86C8008F101021B9298F8014024
:107D00002B2C00F087822D2C00F0218200220E9275
:107D1000A4F13002092A00F21582302C05D11B9AF9
:107D200001321B921478302CFAD0A4F13102082AC7
:107D300093D81B990B914A1C1B92A4F130004C78EC
:107D40002F2C09DC00F034BC01321B929CF801405E
:107D50002F2CA1F1300006DD00EB8001392C944678
:107D600004EB4101F0DD0B99521A082A40F32084FC
:107D700044F61F620B920E9A002A3FF470AF0B9AE2
:107D800052420B92002D7FF46DAF099A134320D11C
:107D9000BEF1000F7FF433AF692C00F03B8400F399
:107DA0004183492C00F036844E2C7FF428AFAC4937
:107DB0001BA804F0D5FB00283FF421AF1B9B1B78C8
:107DC000282B00F06D85A74805F07CFB83460491C5
:107DD00003E04FF0000BCDF810B0089A0AB11B9BDE
:107DE00013600A9B002B3FF413AF049901F1004389
:107DF00004930499584621B0BDE8F08F1B9A04956E
:107E000002EB0B011B9112F80B409B46DEE60E9B2A
:107E10002C1B1C44002C40F30A8314F00F000AD0E2
:107E2000914901EBC001DDE90623D1E90001F9F731
:107E3000C7FBCDE9060134F00F0340F08B8200232D
:107E40000993049A00962B463946484604F052FEA0
:107E50001390002800F055830B9BABEB03000E9BA7
:107E6000002BB4BF024600220F9223EAE3730022E4
:107E7000934612939046139C4846616804F0BAFDFD
:107E80000746002800F0418122690232920004F185
:107E90000C010C30F9F7B6F8DDE9060104910B4648
:107EA0001EA901911DA90B9002460091484605F0BC
:107EB000CDF91C90002800F018810121484604F0FB
:107EC000C1FE8046002800F020811D9B002BC0F2DF
:107ED0000F810F9A129D9E18099A1E9C9B1A23448B
:107EE000624A013B9342C4F1360480F2AE80D21A5A
:107EF0001F2AA4EB020400F31D814FF0010A0023A6
:107F00000AFA02FA0C93099B25443444A6421D4404
:107F10003346A8BF2346AB42A8BF2B46002B02DD49
:107F2000E41AED1AF61A0F9B002B00F3BE80002C0A
:107F300000F3D2800E9B002B00F3DE80002D00F3B7
:107F4000EF80002E08DD41463246484604F0B6FF79
:107F50008046002800F0D9801C993A46484605F032
:107F600045F88346002800F0D0800026C368C6602C
:107F70004146109305F01AF8B042C0F2638400F055
:107F8000D2834146584605F0C3F900224FF08043A2
:107F900004460D46F8F7DAFB00286FD0109B002B43
:107FA00000F0E180079B1193314B314C0022CDE969
:107FB0000C2335462F4E119A2F4B02EA060A9A459A
:107FC00000F0FC80099B93B1BAF1D46F0FD822A3C3
:107FD000D3E9002328462146F8F7B8FB002840F0F3
:107FE00087810D9B03F1D663A3EB0A030D93049ED7
:107FF0000B98DDE90C233146CDE9042305F09CF80C
:1080000002460B46DDE90401F9F7DAFA33460B9A2A
:10801000F8F77CF9CDE906010E46099B23B9154B0B
:1080200033409A4500F002811C99484604F008FD4F
:108030003946484604F004FD4146484604F000FD38
:108040005946484604F0FCFC15E700230C934FF01A
:10805000010A58E7AFF300800000C0FFFFFFDF41D7
:108060000CEC000828EA0008B8EF000802FCFFFF4B
:108070000000F03F0000F07F0000E07FAE4B2046A4
:1080800029460022F9F79CFA109B024605460C4649
:10809000002B64D101F1004314901593079B1193B9
:1080A000DDE91423CDE90C2384E741461A4648460E
:1080B00004F0A4FE804640B301461C9A484604F0F2
:1080C000EFFD10B310901C99484604F0B9FC109BCA
:1080D0001C93002C7FF72EAF1C992246484604F0D3
:1080E000EDFE1C9000287FF425AFBA465E460FE0F7
:1080F000129A0F9ED51AEFE63946129A484604F0B6
:108100007DFE074600287FF419AFBA465E461C98EC
:108110002223C9F80030894B04934FF0000BB4E0E0
:1081200039462A46484604F0C9FE074600287FF42F
:1081300008AFEAE7824A4FF0010AD31A0AFA03F3BA
:108140000C93E0E60022CDF86C800B9287E50122CB
:108150000E9208F102021B9298F80240D8E50B46F5
:10816000CDE914239AE7DDE90612002940F0AF803B
:10817000C2F313031192002B40F0AF80714B002229
:1081800020462946F8F7D8FA002840F0AE826A4B1C
:10819000204629460022F9F713FA01F1004305466B
:1081A0000C4618901993DDE91823CDE90C2301E75B
:1081B000652C4FF0010E3FF49CAD19E5A2F154730C
:1081C0000793DDE90623DDE90C01CDE90601104640
:1081D0001946CDE90C2304F0AFFF02460B46DDE95A
:1081E0000601F9F7EDF9DDE90C23F8F78FF8564AA7
:1081F0000E409642CDE9060176D9049A534B9A4235
:1082000002D10B9B013380D0504A4FF0FF33CDE9B0
:10821000063209E700220E929BE7652C00F0FB80F6
:10822000452C00F0F8804FF0010EAEE528462146BF
:10823000F9F7F8FBF8F7F2F90B4602462146284613
:10824000F8F762F8109C069DC6F3130644EA050C85
:108250005CEA060304460D4600F0C28032A3D3E96F
:108260000023F8F769FA48B931A3D3E9002320467F
:108270002946F8F77FFA00283FF4D6AEDDE9063448
:108280001C9804945E46BA469B460146484604F054
:10829000D7FB5146484604F0D3FB4146484604F01C
:1082A000CFFB1399484604F0CBFB3146484604F017
:1082B000C7FB92E501230A937A1C1B927B78002B63
:1082C0003FF49DAC174629E400230A93F4E7DDE967
:1082D0000612012900F0748111921D4B194C0022E5
:1082E000CDE90C23002565E601F15476079694E666
:1082F00021462846F9F776FB012838BF0120F8F718
:1083000041F9109B024605460C46002B40F069815E
:1083100001F1004316901793DDE91623CDE90C23F4
:108320005FE600BFAFF300809535A094FFFFDF3F0D
:1083300035E5AF350000E03F0000E03F0000F07F92
:10834000E2FBFFFF0000F03FFFFF9F7CFFFFEF7F9E
:108350000000F0BFB3F59A7F00F3D380102B4FEAF3
:108360002314A54B40F3C682DDE906019846099324
:1083700000239A4614F0010F0AF1010A4FEA64043F
:1083800004D0D8E90023F9F71BF90123012C08F1E7
:108390000808EFD10BB1CDE90601099B03EBCA0137
:1083A000079BA3F154730793DDE90623D1E900018C
:1083B000F9F706F9914BCDE906010B400A469049C1
:1083C0008B4200F29E80A1F580118B4240F21C820C
:1083D0008C494FF0FF33CDE906310023099330E596
:1083E00083A3D3E90023F8F7A7F900283FF41CAED4
:1083F00044E71633FFF60BAD0B9BABEB0302824B4E
:1084000003EBC203DDE90601D3E90023F9F702FA21
:1084100083460491E1E40022049293464FF0010E5A
:10842000FFF7EABB6E2C3FF4C2ACFFF7E8BB3FF4AA
:1084300006AD644214F00F020AD0734B03EBC20383
:10844000DDE90601D3E90023F9F7E4F9CDE90601F6
:1084500024113FF4F4AC1F2C35DC14F01003DDE9DB
:10846000060118BF6A23DFF8A48109930023E207FD
:1084700004D5D8E90023F9F7A3F80123641008F123
:108480000808F4D10BB1CDE90601099B93B1DDE9F0
:108490000601C1F30A52C2F16B03002B0ADD1F2B48
:1084A00040F350820020342B069040F356824FF068
:1084B0005C730793DDE9060100220023F8F732F927
:1084C00000283FF4BEAC22234FF0000BC9F8003067
:1084D000CDF810B081E41E9B06931D9B03F233423E
:1084E0001F9B23F4801343EA02530793200742BFE4
:1084F000079B43F000430793DDE906349B46049451
:108500006BE43E4A04922223C9F800304FF0000B7E
:1085100063E40A9B01931CAB029400933C4A1DAB9D
:108520001BA9484603F03EFD10F0070504463FF442
:1085300050AC062D40F09380089B0137002B3FF490
:1085400063AB4FF0000B1F60CDF810B0FFF760BBBE
:108550006A1C012B1B9C9B44104615D02B4403F135
:10856000FF3C03E0460094450DD001322B46082B1A
:10857000154606EB8600F5D9102ADCBF0AEB8A0AFD
:108580004FEA4A0AEFE7981C082D5BDC0546FFF727
:1085900015BB04995A463846FFF730FA002800F018
:1085A000888000231D4604939A461E46FFF751BB60
:1085B00044F61F629042A8BF10460B90FFF7DBBB4A
:1085C000DDE906341194002C7FF487AEBA465E468E
:1085D00022234FF0000B1C98C9F80030CDF810B0E2
:1085E00053E60B46CDE9162396E600BFAFF30080B5
:1085F0009535A094FFFFCF3F90EF00080000F07F7B
:108600000000A07CFFFFEF7FB8EF000838EC000807
:1086100010EC0008AD491BA803F0A2FF00283FF4AE
:10862000EEAA1B9BAA49013B1BA81B9303F098FFD2
:1086300010B91B9B01331B93A64B04934FF0000B07
:10864000FFF7CBBB1028DCBF0AEB8A0A01EB4A0A12
:1086500005460023FFF7B7BA0023FFF7A1BA1C9A1B
:108660003AB135211EA804F081FE1C99484604F059
:10867000E7F9013D042D3FF639AF01A353F825F08A
:10868000D7840008A9860008A386000895860008FC
:10869000D78400084FF0FF336FF00045CDE9063571
:1086A00024E78C4B079321E71E9B06931F9B0793A0
:1086B0001CE71B9A13465A441B9213F80B400646BC
:1086C0008246FFF762BA0E98834901EBC001DDE9EB
:1086D0000623D1E90001F8F773FF83460491FFF701
:1086E0007CBB04958346FFF771BA7C4B7C4C109D94
:1086F0000022CDE9182356E5774CC5F10F0504EBB0
:10870000C501DDE90623D1E90001F8F759FF0E9B09
:108710005D1B04EBC504D4E90023F8F751FF834641
:108720000491FFF75ABB109B5E46D446BA46DDE97A
:108730000BB7002B6FD0DDE906456A4BC5F313017B
:1087400099422A463CD0002F00F0A380DDE90623A1
:108750001F421C4621D0109B04995846002B00F064
:10876000CD8004F0E9FC099D02460B467DB1C4F3BF
:108770000A54C4F16B04002C09DD240504F17F5375
:10878000002203F54013F8F71BFF02460B4604993D
:108790005846F7F7BBFD83460491099B73B10499D2
:1087A000514B58460022F8F70BFF03460B4308BF16
:1087B00022238346049108BFC9F800301C9864E561
:1087C000099B0699002B00F0C580424B2B40B3F16A
:1087D000D46F00F2BF801B0DC3F16B034FF0FF306D
:1087E00000FA03F39942AED1404B9A4200F0D88090
:1087F000384B134003F58013079300230693DDE9FC
:1088000006349B460494C8E702F15473079300238F
:108810000993FFF716BBDDE90612C2F313030B43FE
:10882000144690D1099B002B40F0AF80294B234088
:10883000A3F580136FEA13536FEA035307934FF0C6
:10884000FF33DBE7DDE90612109B0B4358465E461B
:10885000BA46DDF82CB0A0D1C2F313031446002BA6
:108860009BD122F000431B0D1B05B3F1D66F94D9A9
:10887000436913B90369012B8FDD31460122484654
:1088800004F01CFB4146064604F090FB002884DD02
:10889000C8E7DDE906341CEA030F3FF47EAF5AE770
:1088A00013491BA81EAA03F075FE05287FF48BAAA6
:1088B0001F9B43F0FF4343F4E00307931E9B069383
:1088C000DDE906349B460494FFF787BA00EC000804
:1088D00004EC00080000F07FB8EF00080000E0BFE3
:1088E0000000E03FFFFF0F0000005039FFFFEF7F67
:1088F00024EC000809934FF0000A4EE504F01CFC3C
:10890000099D02460B4695B3C4F30A54C4F16B04A7
:10891000002C09DD240504F17F53109A03F5401360
:10892000F8F74EFE02460B4604995846F7F7ECFC62
:108930000022002383460491F7F7F4FE00283FF459
:108940002EAF45E64FF0FF3202FA03F3069A1A40C3
:108950000692AFE54FF0FF3344E74FF0FF33C2F12B
:108960004B0203FA02F202EA01030793A2E504991B
:108970005846F7F7C9FC0022002383460491F7F715
:10898000D1FE00283FF41AAF22E6084B2340B3F192
:10899000D66F3FF74DAFB3F15C7F3FF700AF17E6FF
:1089A00001317FF425AFFFF7B2BB00BF0000F07FBD
:1089B00010B4044C044B84460A46206810BC61463F
:1089C000FFF75EB81C000024600800242DE9F04F7A
:1089D000D5B01C46079191460546099003F0B6FEB6
:1089E0000268179210460E94F8F72AFD16901DB1F2
:1089F000AB6B002B00F02A82079A536EDD0740F123
:108A00003881B2F90C2091B28F0409D4079B42F44B
:108A100000529A8191B21A465B6E23F4005353665A
:108A20000E0740F1CB80079B1B69002B00F0C6802E
:108A300001F01A030A2B00F0CF8000242BAB4D4627
:108A4000CDE92944CDE91944CDE91B44129428937A
:108A50009846189400230B940024CDE914342B7805
:108A6000002B00F09D81AA4604E01AF8013F002B7C
:108A700000F0C780252BF8D1BAEB050640F0C58081
:108A80009AF80030002B00F08B8100234FF0FF326A
:108A90009AF801608DF883300A930AF1010A08926E
:108AA0001F462B244FF020090AF1010AA6F12003EA
:108AB0005A2B00F2ED80DFE813F0EB02EB00EB0045
:108AC000E602EB00EB00EB006A00EB00EB005C025F
:108AD0008002EB0067028A02EB0085025B005B000C
:108AE0005B005B005B005B005B005B005B00EB001E
:108AF000EB00EB00EB00EB00EB00EB007A01EB008E
:108B0000F801D2017A017A017A01EB00EB00EB0067
:108B1000EB00E102EB00EB002D02EB00EB00EB00C1
:108B20000202EB00A402EB00EB008307EB00EB007A
:108B3000EB00EB00EB00EB00EB00EB007A01EB004D
:108B4000F801D4017A017A017A01C702D401CD017A
:108B5000EB00D402EB006C022F02B502CD01EB005A
:108B600002027E008007EB00EB006107EB007E0055
:108B7000A6F1300300221AF8016B02EB820203EB2C
:108B80004202A6F13003092BF5D90A928EE7DDF8EF
:108B900024B0584603F0DAFD43681B931846F8F7F3
:108BA0004FFC1C900646584603F0D0FD836819938D
:108BB000002E40F0CD869AF8006075E7079D099871
:108BC000294601F0C3FC002841F01C83A98901F06B
:108BD0001A030A2B7FF431AF079AB2F90E30002B3B
:108BE000FFF62BAF536ED80702D4890541F13B81C4
:108BF0000799099823464A4655B0BDE8F04F01F061
:108C00004FBCBAEB050600F0CB802A9B33442A9375
:108C1000299B0133072BC8E90056299305DC08F18D
:108C200008080B9B33440B932AE70799099828AA55
:108C300004F0BCFC80B90DF1AC08F2E70799099883
:108C400028AA04F0B3FC002800F09B800D9B1BB108
:108C50000998194602F0B6FE079A536ED90740F1FB
:108C6000EA8093895B0601F1D9820B9855B0BDE883
:108C7000F08F079BB3F90C20900591B23FF5C4AE7D
:108C80001D46986D03F06AFDB5F90C2091B2BBE664
:108C9000002E00F0858000228DF8EC608DF8832096
:108CA0000123CDE90C32069308920F921392109291
:108CB0003BAD17F0020302D006990231069117F07E
:108CC000840B07D10A990698A1EB0009B9F1000FAE
:108CD00000F370832A9C8AB1299A0DF18301013235
:108CE0000134C8F80010072A4FF001012A94299294
:108CF000C8F8041000F3B68308F1080883B1299B73
:108D000021AA01330234C8F80020072B4FF00202D9
:108D10002A942993C8F8042000F3B28308F10808C4
:108D2000BBF1800F00F06982089B0C9AA3EB020B49
:108D3000BBF1000F00F3AA82FB0500F100820C9B3F
:108D4000C8F804301C44299BC8F800500133072B95
:108D50002A94299300F3228308F10808780705D59F
:108D60000A9B069A9D1A002D00F39683DDE90A23DB
:108D700006998A42ACBF9B185B180B93002C7FF4BA
:108D80005DAF002329930D9B1BB10D99099802F04B
:108D900019FE0DF1AC0855462B78002B7FF463AE1D
:108DA0002A9B002B41F0D3810023299354E70E9B8B
:108DB000073323F00702F2E80234CDE91434DDE989
:108DC000143424F000440E92994618462146B54BBF
:108DD0004FF0FF32F7F7D8FC002840F0EF84B14B9A
:108DE000484621464FF0FF32F7F7B0FC002840F02C
:108DF000E584DDE9140100220023F7F79DFC00283B
:108E000040F067879DF88320A74DA84B27F0800787
:108E10000321472EC8BF1D4600230D9306910C91D8
:108E200008930F9313931093002A3FF442AF069BCD
:108E3000013306933DE7079B9B899A053FF512AFE7
:108E4000079CA06D03F08CFCA3890BE7099802F046
:108E5000C1FCD1E59AF8006047F0200724E647F00E
:108E60001007BA060E9B40F13B84073323F007033B
:108E70001A465B6852F8084B0E929946002BC0F2D6
:108E80004C84089B013300F0D88254EA090327F090
:108E9000800B40F0D382089B002B40F0D4825F46C9
:108EA000002308930C9354AD1DE10E9B002253F850
:108EB000041B8DF883208DF8EC100E93F0E60E9CC9
:108EC000089B54F8045B4FF000098DF88390002D47
:108ED00000F093855A1C00F051861A4649462846F0
:108EE000F8F71EFB0D90002801F00E810D9BCDF8C8
:108EF00020905B1B0C930E9423EAE3739DF8832070
:108F00000693CDF83490CDF83C90CDF84C90CDF848
:108F1000409089E747F0100717F0200900F0D2834E
:108F20000E9B073323F00703D3F8049053F8084B44
:108F30000E9327F4806B002300228DF88320089A7B
:108F4000511C00F0B88054EA09012BF0800740F072
:108F5000B180002A40F0F685002BA1D11BF001035F
:108F60000C9300F0148430238DF84F310DF24F151F
:108F7000B9E00E9B53F8042B0A92002A80F2DA83A0
:108F80000A9A0E9352420A929AF8006047F0040738
:108F90008AE5BD0600F1D184FC0600F1D88578068B
:108FA00000F1A586B90540F1D2850E9B0B9953F8C7
:108FB000042B0E9311705546EEE69AF800608DF87A
:108FC000834071E59AF8006047F080076CE55246EF
:108FD00012F8016B2A2E01F03F82A6F13003092B13
:108FE000924698BF002201F2BC801AF8016B02EB96
:108FF000820203EB4202A6F13003092BF5D9089255
:1090000054E547F0100B1BF0200900F076830E9B0F
:10901000073323F00703D3F8049053F8084B0E935B
:10902000012389E70E9B53F8044B0E9330237826D7
:109030008DF884301E4B189347F0020B8DF8856035
:109040004FF00009022377E79AF80060682E03BF0B
:109050009AF8016047F400770AF1010A47F04007E7
:1090600022E59AF800606C2E03BF9AF8016047F081
:1090700020070AF1010A47F0100715E59AF8006089
:1090800047F0080710E59AF8006047F001070BE584
:109090009DF88330002B7FF48EAD9AF800608DF838
:1090A000839001E5FFFFEF7F60EC000864EC0008AF
:1090B00070EC0008BB46012B00F0C081022B54ADC0
:1090C00020D1189A04F00F032409D35C05F8013D60
:1090D00044EA09744FEA191954EA0903F2D154AB6E
:1090E0005B1B5F460C9308990C989DF88320814286
:1090F0004FF00003B8BF01460D9306910F931393F1
:10910000109391E604F00703E40844EA49744FEA37
:10911000D909303354EA09012A4605F8013DF1D155
:109120001BF0010FDBD0302BD9D03023023A05F8E9
:10913000013C54AB9B1A5F460C931546D3E7652E52
:1091400040F3E680DDE9140100220023F7F7EAFA94
:10915000002800F0DC81299BBF4AC8F800200133B9
:1091600001340122072B2A942993C8F8042000F324
:10917000CC8408F10808229B129A934280F2D6828E
:10918000169B179A1C44C8E90023299B2A94013393
:10919000072B299300F3248408F10808129B5D1E15
:1091A000002D7FF7DBAD102D299BDFF8B09240F347
:1091B000BD8449462246B946DDF824B0079C1026F6
:1091C0000F4605E008F10808103D102D40F3AA8471
:1091D00001331032072BC8E90076CDE92932F1DDE1
:1091E00028AA2146584604F0E1F900287FF42EAD64
:1091F000DDE929320DF1AC08E6E70A9B069AA3EBFC
:10920000020BBBF1000F7FF78FADBBF1100F299A56
:10921000DFF848922CDD1D9621464E46079CDDF86E
:109220002490102306E0ABF1100BBBF1100F08F1F6
:1092300008081ADD01321031072AC8E90063CDE9B8
:109240002921F0DD28AA214648460DF1AC0804F09A
:10925000ADF900287FF4FAACABF1100BBBF1100FA5
:10926000DDE929214FF01003E4DCB1461D9E0C46D8
:1092700001325C44072ACDE92924C8F80090C8F8D7
:1092800004B000F3A08308F108084DE5BBF1100F0E
:10929000299ADFF8C8912DDD41462046A8464C4664
:1092A000079DDDF82490102306E0ABF1100BBBF115
:1092B000100F01F1080119DD01321030072AC1E950
:1092C0000043CDE92920F0DD28AA2946484604F0CC
:1092D0006DF900287FF4BAACABF1100BBBF1100FA5
:1092E000DDE929202BA94FF01003E5DC4546A14616
:1092F0008846044601325C44072ACDE92924C8F88F
:109300000090C8F804B000F3D08108F1080813E514
:10931000129B012B40F38081299EC8F80050013632
:1093200001340123072E2A942996C8F8043000F34B
:109330007C8308F10808169B179A01361C44072EF7
:10934000C8E90023CDE9296400F37C8308F108080B
:10935000DDE9140100220023F7F7E4F9002840F0CA
:109360007881129B0136013B01351C44072EC8F859
:1093700000502996C8F804302A9400F35D8108F162
:1093800008081A9BC8F8043001361C44072E24AB89
:10939000CDE92964C8F800307FF7DEAC0799099859
:1093A00028AA04F003F900287FF450AC2A9C0DF1A0
:1093B000AC08D3E4B9F1100FDDE929212BDDCDE9AB
:1093C0001D3B1F96DDF824B04E461024A946079D8C
:1093D00004E0103E102E08F1080817DD0132204B82
:1093E0001031072AC8E90034CDE92921F1DD28AA86
:1093F000294658460DF1AC0804F0D8F800287FF44F
:1094000025AC103E102EDDE92921E7DCDDE91D3B0E
:109410004D46B1461F9EC8F80490013209EB010485
:10942000072A0F49C8F80010CDE9292400F3518319
:109430009DF8832008F108084DE4BB460A2C79F119
:10944000000380F00C83303401238DF84F415F46D8
:109450000C930DF24F1546E6A0EC0008B4EC0008A2
:10946000A4EC0008079909981D9328AA04F09EF817
:1094700000287FF4EBAB2A9C1D9B0DF1AC083DE46A
:109480000799099828AA04F091F800287FF4DEAB28
:109490002A9C0DF1AC0843E4102D299B21DD099F86
:1094A000DDF81C90102604E0103D102D08F108088E
:1094B00017DD0133BB4A1034072BC8E90026CDE97C
:1094C0002934F1DD28AA494638460DF1AC0804F0EC
:1094D0006DF800287FF4BAAB103D102DDDE929347A
:1094E000E7DC0133AF4AC8F804502C44072BCDE920
:1094F0002934C8F800207FF739AC0799099828AAC1
:1095000004F054F800287FF4A1AB2A9C2EE42299A1
:10951000002940F31481DDF84090129B9945A8BFC3
:109520009946B9F1000F0BDD299B01334C44072B01
:10953000C8E900592A94299300F39A8508F108088C
:10954000109EB9F1000FA8BFA6EB0906002E00F38C
:109550004683DDF840B07905AB4400F1CE84229B10
:10956000129A934202DBFA0740F1B883169A1799D0
:109570001444C8E90012299A2A940132072A299230
:1095800000F3838508F10808129AAE18A6EB0B06C3
:10959000D51AAE42A8BF2E46002E0DDD299BC8F875
:1095A00000B001333444072BC8F804602A9429938F
:1095B00000F3F18508F10808002EA8BFAD1B002DAF
:1095C0007FF7CCAB102D299BDFF8DC9140F3AE8206
:1095D00049462246B946DDF824B0079C10260F46BE
:1095E00005E008F10808103D102D40F39B8201337F
:1095F0001032072BC8E90076CDE92932F1DD28AA1F
:109600002146584603F0D2FF00287FF41FABDDE966
:1096100029320DF1AC08E6E7FE073FF57DAE299E45
:10962000C8F80050013601340123072E2A942996E8
:10963000C8F804307FF7A3AE0799099828AA03F069
:10964000B5FF00287FF402ABDDE929640DF1AC0819
:1096500097E6129B5D1E002D7FF793AE102DDFF86D
:10966000489140F37F8222460897099C079F4FF05C
:10967000100B05E008F10808103D102D40F3708232
:1096800001361032072EC8E9009BCDE92962F1DDD1
:1096900028AA3946204603F089FF00287FF4D6AA7D
:1096A000DDE929620DF1AC08E6E70799099828AAD7
:1096B00003F07CFF00287FF4C9AA2A9C0DF1AC08B6
:1096C000FFF73ABB17F0100372D117F0400200F019
:1096D000BD820E9A52F8044B0E929946A4B228E429
:1096E00053F8044B0E93FB0656D47D0651D544F334
:1096F000C0394B4624B2FFF7C1BB1BF0100340F04A
:1097000036811BF0400200F092820E9A52F8044B10
:109710000E929946A4B201230EE42D2364428DF8E3
:10972000833069EB4909BB46012308E4F8077FF55C
:1097300015AB25E59AF800600E93FFF7B5B9299BA4
:109740001A4AC8F80020013301340122072B2A9459
:109750002993C8F8042000F3708408F10808002950
:1097600040F01E82129A07F0010313433FF4F6AA59
:10977000169B1799E218C8E90013299B2A92013316
:10978000072B299300F3618308F1080819E254AD0F
:10979000A9E4B80500F1B4824FEAE4794B46FFF73B
:1097A0006DBB00BFA4EC0008B4EC0008A0EC0008FE
:1097B0000E9B53F8044B0E93FFF7BBBBDDE914017E
:1097C00002460B46F6F7E0FF002840F0A085612E28
:1097D00000F05085412E00F09982089B013326F05D
:1097E0002003069300F08F85472B00F07985DDE993
:1097F000141247F480730F931346002BC0F2ED85CB
:109800000C9300231D938B460D93069B462B00F073
:109810004A84452B00F04F850899019126A90491AF
:1098200023A9039122A9029102210C9B099800917E
:109830005A4600F0A9FF069B472B054640F01C86C0
:1098400017F0010FB9460F9F40F0D984269B5B1B90
:109850001293069B472B00F01883069B462B00F0C3
:109860005F84229B1093109B069A013B412A22930E
:1098700000F0AA85F2B20021002BB8BF109B8DF832
:109880009020BABFC3F101032D222B22092B8DF8A2
:10989000912040F363850DF19F04BD4F2246104691
:1098A00087FB0321DA17C2EBA10202EB8201A3EBD3
:1098B0004101303100F8011C19466329134600F1BB
:1098C000FF32ECDC3033D9B2831E9C4202F8011C1B
:1098D00040F2CE8513460DF1920201E013F8011B10
:1098E00002F8011B9C42F9D10DF1A1030DF1920286
:1098F0001B1A134424AA9B1A1A93129B1A9A012B1F
:109900001A440C9240F372850C9B169A13440C93E4
:109910000C9A002329F4806722EAE27247F48077E8
:109920000F930692139310931D9B002B40F0DE8241
:109930009DF883200893FFF777BA0E9B0B9853F896
:10994000041B0E93C217C1E900025546FFF724BA63
:10995000199B002B3FF42FA9199B1B78002B3FF478
:109960002AA99AF8006047F48067FFF79DB80E9B1C
:1099700053F8044B0E930123FFF7DEBA854B18937F
:1099800017F0200949D00E9B073323F00703D3F8C3
:10999000049053F8084B0E93F80709D554EA0903CD
:1099A00006D030238DF8856047F002078DF88430AB
:1099B00027F4806B0223FFF7BFBABB46FFF723BB38
:1099C000754B1893DCE70799099828AA03F0EEFD78
:1099D00000287FF43BA92A9C0DF1AC08FFF7A4B93D
:1099E0000799099828AA03F0E1FD00287FF42EA921
:1099F0002A9C0DF1AC08FFF7D1BB062B294628BFE6
:109A0000062308950D952A460693644D0E940C93F3
:109A10000F9113911091FFF707BA17F0100369D057
:109A20000E9B53F8044B0E93B6E70799099828AAA2
:109A300003F0BCFD00287FF409A9DDE929640DF1DC
:109A4000AC0878E40799099828AA03F0AFFD00282C
:109A50007FF4FCA8DDE929640DF1AC0878E40BF48F
:109A600080630022CDE90CA80696DDF8648054AF2F
:109A700016469A460CE00023204649460A22F7F78C
:109A80003FF90A2C79F100031BD3044689462F467F
:109A900020460A2200234946F7F732F930327D1E6C
:109AA000013607F8012CBAF1000FE4D098F8003025
:109AB0009E42E0D1FF2EDED00A2C79F1000380F027
:109AC000F480CDF864801296DDE90CA8069EFFF7BD
:109AD00006BB079909981D9328AA03F067FD002883
:109AE0007FF4B4A89DF883202A9C1D9B0DF1AC083F
:109AF000FFF7F1B817F0400200F0B6800E9A52F866
:109B0000044B0E929946A4B246E70799099828AAF1
:109B100003F04CFD00287FF499A82A9C0DF1AC08B5
:109B2000FFF729BB14463A464F46914601332C4471
:109B3000072BC8F80090C8F80450CDE929347FF706
:109B40000BA92BE4012BBB467FF4B8AA7BE40E9B48
:109B50000B9953F8042B554611600E93FFF71CB96F
:109B6000089F144601362C44072ECDE92964C8F815
:109B70000090C8F804507FF702AC5DE52846CDF8A8
:109B800020900E94F7F75CFC03460C90FFF7B4B9F5
:109B90006766666670EC000884EC000898EC0008C4
:109BA000169B1798E218C8E90003299B2A920133F3
:109BB000072B299300F3498108F108080029C0F216
:109BC000FA821299C8F8005001338C18072BCDE99E
:109BD0002934C8F804107FF7BFA8FFF7DFBB102EA9
:109BE000299BDFF8C09252DD484642462146A846EE
:109BF000B946099C079D4FF0100B074603E0083259
:109C0000103E102E3DDD01331031072BC2E9007BE1
:109C1000CDE92931F3DD28AA2946204603F0C6FC08
:109C200000287FF413A8DDE929312BAAE8E70E9B71
:109C30001BF4007914BF53F8044B53F8044B0E93F4
:109C40001CBF9146E4B20123FFF776B90E9B17F4CF
:109C5000007914BF53F8044B53F8044B0E931CBF08
:109C60009146E4B2FFF765B90E9B17F4007914BF73
:109C700053F8044B53F8044B0E931CBF9146E4B2C7
:109C80008AE6454690463A460C464F469146013391
:109C90003444072BCDE92934C8F80090C8F8046093
:109CA00000F3E68008F1080853E41C9B1B99ED1AA9
:109CB0001A46284603F00CFC98F801300BB108F165
:109CC0000108204649460A2200230026F7F718F823
:109CD000DBE62D228DF88320FFF796B8129AAE1896
:109CE000A6EB0B06D51AAE42A8BF2E4664E40E9B27
:109CF0000B9953F8042B0E9311805546FFF74CB87F
:109D000044F3C0194B4664B2FFF7B8B830238DF85E
:109D1000843058238DF88530089B632B47F002046C
:109D200000F39B8200230D933BADDDE9141247F451
:109D300081730F931346002B2746C0F220820C93A9
:109D400026F02003069300238B461D93612E00F01E
:109D5000ED82412E7FF459AD22AA0C99584603F0AA
:109D600079FB00224FF07F53F7F72AFC02460B469F
:109D7000CDE9102300220023F6F7D4FC08B101231B
:109D80002293494B0C93089BCDE912A6CDE91E788E
:109D9000DDF830A0DDE9106703F1FF39AB4610951F
:109DA00006E00022002309F1FF39F6F7BBFCE8B911
:109DB0003E4B002230463946F7F702FC0F46064676
:109DC000F6F7F8FC0446F6F7EDFB0B46024639467B
:109DD0003046F6F799FA1AF80430B9F1FF3FD84641
:109DE0004D460BF8013B06460F46DAD13046394660
:109DF0002F4BDDF848A0139ECDF848800022A946DD
:109E0000DDF87C80109D1E9FCDE91001F6F7B2FCB5
:109E1000002840F03482DDE91001254B0022F6F7DE
:109E200081FC10B1E10700F12A824B46002B06DBD2
:109E300001335B4430220BF8012B5B45FBD1ABEBCC
:109E40000503B94612930F9F03E50799099828AABD
:109E500003F0ACFB00287EF4F9AEDDE9293222994B
:109E60000DF1AC08AAE6906D02F07AFCFEF7C0BED8
:109E70000799099828AA03F099FB00287EF4E6AE1A
:109E80002A9C0DF1AC08FFF764BB229B1093DA1CEF
:109E900002DB089A93420DDD023E26F02003069372
:109EA000E1E400BFB4EC000884EC0008000030409E
:109EB0000000E03F109B129A9342C0F2568119F0C5
:109EC000010F00F08782169A13440C9319F4806FE7
:109ED00003D0109B002B00F350820C9B23EAE3730A
:109EE0000693672600230F9313931DE52D2200236D
:109EF0008DF883200893FEF79ABF129BCDF830A00F
:109F00004246DDF84C801097EB1808935E46199F87
:109F1000DDF87090DDF824A0DDF81CB00F9B1395E0
:109F20002146B8F1000F2ED0002B6BD1013F08F174
:109F3000FF381B9BC2E90039299B01334944072B99
:109F40002A91299362DC0832089B38789B1B834254
:109F5000A8BF0346002B1C460ADD2998013019448E
:109F60000728C2E900632A9129905ADC3878083220
:109F7000002CACBF051B0546002D15DC06440F9BCD
:109F8000B8F1000FD0D1002B3CD1DDE91235EB1830
:109F90009E421997B346DDF830A0109F90460C46BC
:109FA00028BF9B46FFF7DBBA102D29981DDD102432
:109FB00004E0103D102D02F1080216DD0130AC4B1B
:109FC00010310728C2E90034CDE92901F1DD28AAC2
:109FD0005946504603F0EAFA00287EF437AE103DA9
:109FE000102DDDE929012BAAE8DC0130A04B5560DA
:109FF00029440728CDE9290113602CDC3878083280
:10A000000644BCE70F9B013B0F9392E728AA5946F1
:10A01000504603F0CBFA00287EF418AE2A992BAAFA
:10A0200092E728AA5946504603F0C0FA00287EF469
:10A030000DAE38782A992BAA9AE70799099828AA89
:10A0400003F0B4FA00287EF401AE22992A9C0DF1A7
:10A05000AC08FFF784BB28AA5946504603F0A6FA7D
:10A0600000287EF4F3AD38782A992BAA064486E7B7
:10A070000799099828AA03F099FA00287EF4E6AD1A
:10A080002A9C0DF1AC08FFF75BBA0799099828AA3A
:10A0900003F08CFA00287EF4D9AD229B2A9C0DF1A6
:10A0A000AC08FFF771BA0899019126A9049123A978
:10A0B000039122A9029103210C9B099800915A4611
:10A0C00000F062FB0378302B054600F09581229B5F
:10A0D000089AB94613440F9FEC180C995846002271
:10A0E0000023F6F71FFB10B12346FFF7B0BB269BFA
:10A0F000A342BFF4ACAB30215A1C26921970269BA8
:10A100009C42F9D8FFF7A3BB089B9DF883200E94CF
:10A1100006930C9308900F9013901090FEF784BE56
:10A12000229A1092002A40F38181089909F00103D4
:10A130000B4340F05581109B0C93662619F4806FF9
:10A1400040F01C810C9B23EAE3730693CAE607994F
:10A15000099828AA03F02AFA00283EF425AEFEF753
:10A160007BBD00230893FEF7A1BC129B169A9A1898
:10A17000109B0C92002B40F34D816726DEE726F002
:10A1800020030693DDE914349B4604F100430C934D
:10A190002D231D93DAE50799099828AA03F006FAFA
:10A1A00000287EF453AD229D129B2A9C5D1B0DF16D
:10A1B000AC08FFF701BA4E421031DFF8B49034DA40
:10A1C0004146DDF824B0A8461024079D03E008317D
:10A1D000103E102E27DD01331032072BC1E9009409
:10A1E000CDE92932F3DD28AA2946584603F0DEF9E5
:10A1F00000287EF42BADDDE929322BA9E8E7089B86
:10A20000EC186AE7079B5B6EDD0707D4079B9B8909
:10A210009C0503D4079B986D02F0A2FA4FF0FF3320
:10A220000B93FEF722BD4546884601333244072B87
:10A23000CDE92932C8F80090C8F804607FF7A4AAD5
:10A240000799099828AA03F0B1F900287EF4FEAC1A
:10A25000DDE929320DF1AC08B3E40998591CFCF78B
:10A260002DFD0546002800F00D810D905DE500BF35
:10A27000B4EC000830238DF8843078234AE5129B33
:10A2800026930C9B1BF8012CD97B8A425B4609D193
:10A29000302003F8010C269B5A1E269213F8012C3D
:10A2A0009142F6D0392A0BBF0C9A0132927AD2B27F
:10A2B00003F8012CC3E508990C9B09984C1C26A9AE
:10A2C000049123A9039122A9029102215A460194E3
:10A2D000009100F059FA0546B9462C440F9FFCE660
:10A2E000089B002B08BF0123089347F480730F934A
:10A2F000159B002BC0F2AE80DDF850B01D900C9382
:10A300000D90FFF789BA06230893FFF770BA159BE3
:10A31000604D002BB4BF2D229DF883205E4BB8BF4B
:10A320008DF8832027F08007FEF772BD22AA0C99D2
:10A33000584603F08FF800224FF07F53F7F740F9AB
:10A3400002460B46CDE9102300220023F6F7EAF976
:10A3500008B101232293514B0C9314E5002962D1DB
:10A3600030228DF892200DF19302303302F8013B38
:10A3700024ABD31A1A93FFF7C0BA672619990B7842
:10A38000FF2B7BD00024109A204603E001300131DE
:10A39000FF2B08D0934206DAD21A4B78002BF5D166
:10A3A0000B780134F4E71991109213900F940F9ADF
:10A3B000139B1C9913440C9A01FB03230C9323EA6F
:10A3C000E3730693FFF7B0BA06F10F02D2B2012190
:10A3D000FFF752BA109B0C9378E500230D93D1E65A
:10A3E000169BD31819440C916626A7E619F0010FA5
:10A3F0003FF48EAAFFF788BA0C9958460022002332
:10A40000F6F790F900287FF462AE089BC3F10103D0
:10A4100022935DE6C3F101031A4422EAE2730C922F
:10A42000069367265EE50DF192029EE7089A09F011
:10A43000010959EA020304D10123069366260C930D
:10A4400050E5169B01331A4422EAE2730C920693FC
:10A45000662647E50D9095E60E9B9AF801609246B8
:10A4600053F8042B0E9342EAE2720892FEF71CBBEB
:10A4700002231A93FFF741BA089C2DE700230F939C
:10A48000139394E7079A938943F040039381FEF76F
:10A49000E3BB00BF68EC00086CEC000870EC00083F
:10A4A000F0B51F468B89ADF26C4D23F00203ADF879
:10A4B0000C304B6E1993CB89ADF80E30CB690793F6
:10A4C0004B6A09931AAB009304934FF480631546CB
:10A4D00006460293059316A800230C46069302F045
:10A4E00039F92A463B4669463046FEF76FFA051EA3
:10A4F00007DB6946304601F039F9002818BF4FF0F4
:10A50000FF35BDF80C305B0603D5A38943F040034B
:10A51000A381169802F020F928460DF26C4DF0BD8B
:10A5200038B50C46084D8446114620461A4600238D
:10A530002B606446F8F71CFA431C00D038BD2B682A
:10A54000002BFBD0236038BD840C002438B5334B7E
:10A550001B6805460C460BB19A6B12B3B4F90C306C
:10A5600018079AB225D5216900292DD012F00100D3
:10A5700007D00020A06060694042A06139B100208E
:10A5800038BD950758BF6069A0600029F7D1120651
:10A5900058BF0846F4D543F04003A3814FF0FF3085
:10A5A00038BD184601F016F9B4F90C3018079AB204
:10A5B000D9D4D1062AD5520714D4216943F008030F
:10A5C000A3819AB20029D1D102F42070B0F5007FA6
:10A5D000CCD02146284602F0DBF8B4F90C302169D2
:10A5E0009AB2C3E7216B51B104F14002914204D009
:10A5F000284601F0E7F9B4F90C3000222263216902
:10A600000022C4E9001223F02403D7E7092243F013
:10A6100040032A604FF0FF30A38138BD1C000024A6
:10A62000024B13B1024800F005B87047000000006B
:10A63000F9B80008002301461A46184603F0DEBEAA
:10A6400038B5074D0022044608462A60F8F7AAF9F3
:10A65000431C00D038BD2B68002BFBD0236038BDD5
:10A66000840C00242DE9F04F03690C69A34283B0E8
:10A67000C0F28680013C01F11405A30000F114082A
:10A68000009355F8243058F8242001338A469A4222
:10A6900008EB8401814605EB84070191B2FBF3F6D8
:10A6A00038D30023AE4640469B465EF8041B026842
:10A6B0001FFA81FC06FB0C33090C4FEA134C06FB16
:10A6C00001CC99B2ABEB01011FFA8CF311FA82F1C4
:10A6D000C3EB124202EB214289B241EA02417745C3
:10A6E00040F8041B4FEA1C434FEA224BDDD2009B8B
:10A6F00058F8033073B9019B043B984504D307E035
:10A70000984504F1FF3403D253F80429002AF7D006
:10A71000C9F810405146484602F048FC00282BDB9F
:10A7200001364046002355F8041BD0F800C08AB219
:10A730009A1A0B0C12FA8CF2C3EB1C4303EB224364
:10A7400092B242EA0342AF4240F8042B4FEA23435D
:10A75000E9D258F8242008EB84036AB9043B9845F1
:10A7600004D307E0984504F1FF3403D253F80429D9
:10A77000002AF7D0C9F81040304603B0BDE8F08F8A
:10A78000002003B0BDE8F08F2DE9F04F016C99B0C7
:10A7900090469946CDE90489259D044641B1426C15
:10A7A0004A60012393408B6002F04AF9002323643E
:10A7B000B9F1000AB4BF012300232B60764BBCBF64
:10A7C0002AF0004ACDF814A033EA0A0300F0AA8068
:10A7D000DDE904231046194600220023CDE90A01D1
:10A7E000F5F7A0FF074670B1249A01231360269B5A
:10A7F000002B00F0E48269481860431E039303981D
:10A8000019B0BDE8F08F16AB019317AB009320464B
:10A81000DDE90A2302F01AFD5FEA1A56054640F008
:10A820009780DDE916763E4406F23240202840F358
:10A83000B583C0F140000AFA00FA06F2124028FA85
:10A8400000F04AEA0000F5F79DFE0123013EA1F168
:10A85000F8710F93524B0022F5F756FD48A3D3E948
:10A860000023F6F7ADFE48A3D3E90023F5F74EFD2C
:10A87000804630468946F5F795FE45A3D3E9002387
:10A88000F6F79EFE02460B4640464946F5F73EFD6A
:10A8900080468946F5F78EFF002283460023404616
:10A8A0004946F5F749FF002840F07C82BBF1160FBE
:10A8B00000F26B823B4B03EBCB03D3E90023DDE9D2
:10A8C0000A01F5F739FF002872D00023BE1B0E9352
:10A8D000731E0BF1FF3B069300F15E820023099388
:10A8E000BBF1000F6BDA099BCDF81CB0A3EB0B0397
:10A8F0000993CBF100030D93229B092B4FF0000B22
:10A9000066D8052B40F34883043B22930026229B04
:10A91000023B032B00F26886DFE813F05C04590465
:10A9200050043304249A42F20F73CAF3130A1360DB
:10A930005AEA08031AD1269B002B00F064861A4BB2
:10A9400003930833269A0398136019B0BDE8F08F7B
:10A95000DDE90A12C2F31303084643F07F510F9753
:10A96000A6F2FF36169F41F4401173E7269B002B99
:10A9700040F0EA830D4B039341E700BFAFF3008043
:10A9800061436F63A787D23FB3C8608B288AC63FF5
:10A99000FB799F501344D33F0000F07FA1EC0008E7
:10A9A0000000F83FB8EF0008C8EC0008C4EC00084D
:10A9B000BE1B731E069300F185840E900990069BC2
:10A9C0005B44CDE9063B00230D93229B092B98D9CC
:10A9D0000023CDE9223301264FF0FF330C96089374
:10A9E000089B129300216164204602F003F8039053
:10A9F000002800F00186039B2364089B0E2B00F2C5
:10AA00001381002E00F010810799002940F35C8427
:10AA1000AE4B01F00F0203EBC2034FEA2118C90548
:10AA2000D3E9006740F11484A94BDDE90A01D3E9B9
:10AA30000823F6F7EFFECDE9100108F00F084FF0FC
:10AA4000030AB8F1000F13D0DFF8849218F0010F59
:10AA500009D030463946D9E90023F6F7B1FD0AF1AD
:10AA6000010A06460F465FEA680809F10809EDD1B8
:10AA7000DDE9100132463B46F6F7CCFE80468946BA
:10AA80000E9B43B1934B002240464946F5F754FED6
:10AA9000002840F030855046F5F784FD42464B468D
:10AAA000F6F78EFD8C4B0022F5F730FCA1F15073C8
:10AAB000CDE910011193089B002B00F09780079BB4
:10AAC0001493089B13930C9B002B00F0A584139AFE
:10AAD0007E4B8249039E03EBC20353E9022300200D
:10AAE000F6F798FEDDE91023F5F70EFCCDE910012D
:10AAF00049464046F5F75EFE0746F5F753FD024628
:10AB00000B4640464946F5F7FFFB3037DDE9102399
:10AB100006F8017B80468946F5F70EFE002840F0D6
:10AB20002985CDF854B00027DDE910AB1095139DB1
:10AB300013942AE00137AF4280F22C85684B5046CF
:10AB400059460022F6F73CFD654B002282468B46B3
:10AB500040464946F6F734FD89468046F5F72AFE19
:10AB60000446F5F71FFD02460B4640464946F5F7F9
:10AB7000CBFB303406F8014B52465B468046894693
:10AB8000F5F7DAFD002840F0F38442464B46514980
:10AB90000020F5F7B9FB52465B46F5F7CDFD0028DE
:10ABA000C8D0DDE91343109D039A079302E0964253
:10ABB00000F0C884B24616F8013D392BF7D00133B6
:10ABC000DBB23370079B01330793C8E15046F5F7BA
:10ABD000E9FC42464B46F6F7F3FC3F4B0022F5F703
:10ABE00095FBA1F15073CDE9100111933D4B404607
:10ABF00049460022F5F788FBDDE910894B464246BD
:10AC000006460F46F5F7B6FD8146002840F0AA84B7
:10AC1000DDE91001024601F1004330463946F5F7FF
:10AC20008BFD002840F04583179B002BC0F28C80E1
:10AC3000079A0E2A00F38880244B03EBC203D3E962
:10AC400000AB239B002B1BDA089B002B18DC40F089
:10AC50002E83244B002250465946F6F7B1FC02469B
:10AC60000B46DDE90A01F5F771FDDDF820904E464F
:10AC7000002800F0C782239BDDF80C80DF43C9E287
:10AC8000DDE90A7852465B4638464146F6F7C2FD92
:10AC9000F5F790FD81460990F5F784FC52465B4636
:10ACA000F6F78EFC039E0B46024641463846F5F702
:10ACB0002BFB09F1300306F8013B089B012B00F048
:10ACC0005C830694012704951C462AE0B8EF00082F
:10ACD00090EF00080000F03F00001C400000E03F43
:10ACE000000024400000144052465B46404649465E
:10ACF000F6F790FDF5F75EFD0546F5F753FC524675
:10AD00005B46F6F75DFC01370B4602464946404676
:10AD1000F5F7FAFA05F13003A74206F8013B00F017
:10AD20002983AC4B0022F6F74BFC0022002380461F
:10AD30008946F5F7F7FC0028D6D0049D069C079BB2
:10AD400001330793B2460AE10C9A002A3DD0229AB9
:10AD5000012A40F39C82089B03F1FF380D9B434579
:10AD6000C0F26D82A3EB0808089B002BC0F23C8365
:10AD7000069A1A440692099A17461A440992012122
:10AD8000204601F05FFF064623E00123BE1B0E9321
:10AD9000731E06937FF5A2ADC6F10103099300234C
:10ADA00006939DE55846F5F7FDFB42464B46F5F701
:10ADB000B9FC00287FF47AAD0BF1FF3B76E5864BBA
:10ADC0000393039819B0BDE8F08FDDF83480099F34
:10ADD0000C9E002F0CDD069900290B4608DD099A10
:10ADE000B942A8BF3B46D21AFF1ACB1A0992069362
:10ADF0000D9BDBB10C9B002B00F05D82B8F1000FC6
:10AE00000FDD31464246204601F0F8FF2A46014652
:10AE10000646204601F044FF29460546204601F03B
:10AE20000FFE0D9BB3EB080240F0D88201212046B3
:10AE300001F008FFBBF1000F814600F3B480229BB4
:10AE4000012B40F386814FF0000A0120BBF1000F77
:10AE500040F0B580069A104410F01F0000F0938077
:10AE6000C0F12003042B40F3D283099BC0F11C00E6
:10AE700003440244099307440692099B002B05DD15
:10AE800029461A46204602F019F80546069B002B73
:10AE900005DD49461A46204602F010F881460E9B11
:10AEA000002B40F03681089B002B40F31D810C9B4A
:10AEB000002B40F0A080079B01330793DDF80C8046
:10AEC000DDF820A0012707E0294600230A222046BA
:10AED00001F0C0FD0137054649462846FFF7C2FB91
:10AEE000574500F1300308F8013BEDDB089A002AD2
:10AEF000C8BF9346039AD8BF4FF0010B9344002775
:10AF0000294601222046049301F0D8FF4946054610
:10AF100002F04CF8002840F3A8811BF8013C039A8A
:10AF20000BF1FF3B04E05A4500F0AA811BF8013DFC
:10AF3000392B0BF1010AF6D001338BF8003049466A
:10AF4000204601F07DFD56B12FB1B74203D03946FE
:10AF5000204601F075FD3146204601F071FD29467D
:10AF6000204601F06DFD00238AF80030249B079AEB
:10AF70001A60269B002B3FF442AC0398C3F800A054
:10AF800019B0BDE8F08F1C20099B03440993069B70
:10AF900003440744069370E70126B8E4C0F120009B
:10AFA00008FA00F04FE401465A46204601F026FF19
:10AFB000229B012B814640F3B3814FF0000AD9F860
:10AFC000103009EB8303186901F0EEFDC0F1200099
:10AFD00040E700BF00002440A0EC000831460023F9
:10AFE0000A22204601F036FD129B002B064640F354
:10AFF000E782CDE90783002F00F31A81BAF1000F31
:10B0000040F0D581B046049B039F089903F00102EC
:10B010007B1E1944229B0C92134309910A934946C3
:10B020002846FFF71FFB31468346284601F0BEFF46
:10B03000424649468246204601F0D8FFC268014692
:10B040000BF13003002A42D106902846089301F004
:10B05000ADFF06990490204601F0F2FC049A089B8B
:10B060001AB90A99002900F09B82BAF1000FC0F2C8
:10B07000638122994AEA010A0C9951EA0A0100F017
:10B080005B81002A00F3B481099A3B7007F1010A41
:10B090009742D34600F0B281294600230A22204677
:10B0A00001F0D8FC4645054631464FF000034FF00D
:10B0B0000A02204612D001F0CDFC4146064600238C
:10B0C0000A22204601F0C6FC57468046A7E72046E4
:10B0D000049301F0B5FC049B0122C6E701F0BAFC21
:10B0E0005746064680469AE7229B022B79DC0C9B4A
:10B0F000002B80D1079B4946013328460793FFF771
:10B10000B1FADDF80CB000F130030BF8013B002779
:10B11000F6E64946284601F049FF0028BFF6C3AECF
:10B12000294600230A22204601F094FC079B03F1E4
:10B13000FF380C9B0546002B7FF450AF129B002B71
:10B1400040F335820893B9E6AF4B03930333FFF71F
:10B15000F9BBDDE9041200297FF475AEC2F31303D5
:10B16000002B7FF470AEA94B1340002B00F0FE8142
:10B17000099B01330993069B013306934FF0010AA3
:10B1800063E601230C93239B079A13441293013324
:10B19000012B1F460893B8BF01270021172F6164B8
:10B1A0007FF722AC012204235B0003F11400B842B4
:10B1B000114602F10102F7D9616415E401230C93F1
:10B1C000239B002B4CDD129308931F46E5E70023D9
:10B1D0000C93D8E700230C93F2E7129BCDF81C8068
:10B1E0000893089B002B7FF446AD49460522204674
:10B1F00001F030FC01468146284601F0D7FE0028C8
:10B200007FF739AD0398079F3123804600F8013B53
:10B21000013703904946204601F012FC7B1CDDF803
:10B220000CA00793CDF80C80002E7FF494AE96E628
:10B2300031463A46204601F041FE0646DEE60D9BC9
:10B24000CDF83480A8EB03039B444FF000088BE556
:10B25000DDE90A234FF0020ACDE91023FFF7F1BB25
:10B26000012323930893FFF7BBBB03D1049BDB07A8
:10B270003FF553AEDA461BF8013D302BFAD05EE6BF
:10B28000079B039A013307933123137057E60F9AF4
:10B29000002A00F0268103F23343069ADDF8348059
:10B2A0001A440692099A17461A44099267E54FF024
:10B2B00000094E46DFE429460D9A204601F09EFD26
:10B2C0000546B3E50E9067E500F00F81079A504BF5
:10B2D000564206F00F0203EBC203D3E90023DDE977
:10B2E0000A01F6F76DF936118046894600F0718142
:10B2F000484F00234FF0020AF20706D5D7E9002392
:10B30000F6F75EF90AF1010A0123761007F1080742
:10B31000F2D1002B3FF4B4AB80468946FFF7B0BBB7
:10B32000049B002B7FF449AEDDE90412C2F3130342
:10B33000002B3FF418AF40E6002A12DD2946012217
:10B340002046049301F0BAFD4946054601F02EFE61
:10B350000028049B40F31881392B00F0F9800BF191
:10B360003103BA460AF8013B079B0133374607937E
:10B370004646E4E50995069C049D02460B46F4F713
:10B38000C5FF52465B4680468946F5F7F3F960B93A
:10B3900052465B4640464946F5F7C4F900283FF45B
:10B3A000CEAC099BD9077FF5CAAC039A02E4716859
:10B3B000204601F01FFB0746002800F00E8133698C
:10B3C00002339A0006F10C010C30F5F71BFE3946EA
:10B3D0000122204601F072FD804614E629462046EF
:10B3E00001F00CFD054621E5DDE908239F1AC6E4BE
:10B3F000392B00F0AD80BA460133B3E7079A01322A
:10B400003746079246467BE5C4EC00080000F07F13
:10B41000B8EF000890EF0008DDF84CA0844901EB7C
:10B42000CA01DDE9102351E90201F6F7C9F8CDE9B7
:10B43000100149464046F5F7BDF90646F5F7B2F862
:10B440000B46024649464046F4F75EFF039F5346CB
:10B450003036012B07F8016B8046894600F0AE803C
:10B46000139E039B1E44734B002240464946F6F749
:10B47000A7F889468046F5F79DF98246F5F792F8D8
:10B480000AF1300A02460B4640464946F4F73CFFB3
:10B4900007F801ABB74280468946E4D1664B0022EB
:10B4A000DDE91001F4F732FF42464B46F5F744F967
:10B4B000002864D1DDE910235F490020F4F724FF60
:10B4C00042464B46F5F756F900283FF4ADABB2467D
:10B4D000013E1AF8013C302BF9D0149B013307933D
:10B4E0003DE5169BC3F13603D7E6DDE90A894FF047
:10B4F000020AFFF7C5BA089B002B3FF467AB129B0B
:10B50000002B7FF791AB079A013ACDE91332404601
:10B51000484B00224946F6F753F8804689460AF11F
:10B520000100F5F73FF842464B46F6F749F8434B22
:10B530000022F4F7EBFEA1F15073CDE91001119355
:10B54000FFF7C1BA079B013307933123FFF739BBDC
:10B55000079BBB4601330793392337460BF8013B62
:10B560004646DCE44FF000094E464BE69A466CE452
:10B57000109D139C149B01330793B246EFE4149B78
:10B58000039A0793FFF716BB7FF4EBAEDA077FF55C
:10B59000E8AEE1E6DDF854B0109D139CFFF744BB24
:10B5A000392BD5D0BAF1000F3FF7D9AED9E6229B9F
:10B5B000022B3FF712AECDF81C809BE53E466DE7AF
:10B5C000229B022B3FF709AE129BCDF81C800893FB
:10B5D00011E54FF0020AFFF753BA194B19483A46E2
:10B5E00040F2EA2102F050FF002666643146204610
:10B5F00001F000FA039078B9114B124800224FF481
:10B60000D57102F041FF104B0393FFF7F8B83FF4F8
:10B6100034ACC0F13C00B7E4039B236401224FF03B
:10B62000FF33239612930C920893FFF7FDBA00BFE5
:10B63000B8EF0008000024400000E03F00001C407C
:10B64000D4EC0008E8EC0008C8EC0008B1F90C20C4
:10B65000F8B50C461107074642D4636842F400620D
:10B66000002BA28159DDA56A002D54D000233E682D
:10B670003B6093B212F4805253D1E1690123384602
:10B68000A847421C63D0A389A56A5B0705D56368F8
:10B69000C01A236B0BB1E36BC01AE16902460023A9
:10B6A0003846A847411C3ED13B68002B3BD01D2BA0
:10B6B00001D0162B52D1A3892269226023F40063A2
:10B6C00000216160A381216B3E6021B304F140033E
:10B6D000994202D0384600F075F900202063F8BD89
:10B6E0002669C6B193B2256826609A070CBF6369C4
:10B6F0000023AD1BA3600CE0D4F824C0E1692B4605
:10B7000032463846E047B0F1000CA5EB0C05664424
:10B7100016DD002DF0DC0020F8BDE36B002BA2DC71
:10B72000F9E7206DB1E7B4F90C302269226023F407
:10B730000063A3810022DB046260C4D52065C2E7F8
:10B74000A38943F040034FF0FF30A381F8BD3B686D
:10B75000002B98D01D2B06D0162B04D0A38943F0C4
:10B760004003A381F8BD3E60D5E700BF38B50C4665
:10B77000054608B1836BA3B1B4F90C00B8B1636E90
:10B78000DB0701D4810515D528462146FFF75EFF6A
:10B79000636EDA07054602D4A3899B050ED52846B9
:10B7A00038BD00F017F8B4F90C000028E7D10546C1
:10B7B000284638BDA06D00F0D1FFE5E7A06D00F090
:10B7C000CFFF284638BD00BF014900F075BB00BF60
:10B7D00041E500082DE9F0478246394800F0BEFFF8
:10B7E000DAF83840002C66D1DAF80450354ACAF845
:10B7F0003C200323CAE9B843DFF8CC90DFF8CC80C3
:10B80000334F344E04230AF53B72CAF8E82221462E
:10B81000C5E90243C5E90044C5E904446C66082251
:10B82000AC6105F15C00FBF7F9FCC5E90759C5E916
:10B830000987EE6205F1580000F08CFFDAF8085035
:10B84000254BEB602146C5E90044C5E904446C661C
:10B85000AC60AC61082205F15C00FBF7DFFCC5E9D8
:10B860000759C5E90987EE6205F1580000F072FF3B
:10B87000DAF80C50194BEB602146C5E90044C5E9E4
:10B8800004446C66AC60AC61082205F15C00FBF717
:10B89000C5FC05F15800C5E90759C5E90A76C5F8A0
:10B8A000248000F057FF0123CAF838300448BDE86F
:10B8B000F04700F055BFBDE8F047014800F050BF29
:10B8C000800C0024C9B70008717900089579000838
:10B8D000D5790008F579000809000100120002007E
:10B8E000014800F03BBF00BF7C0C0024014800F081
:10B8F00037BF00BF7C0C002438B5084B084D5B1BDC
:10B900009C1007D0043B1D44013C55F8043998476E
:10B91000002CF9D1BDE8384003F006B800F100086A
:10B92000FCF00008F8B5244F0C460646FBF7C8FCAF
:10B93000BA685568C4F57E630F3325F003052B44C0
:10B9400023F47F6323F00F03A3F58054B4F5805FE5
:10B9500007DB00213046FBF721FFBB682B449842F0
:10B9600004D03046FBF7B2FC0020F8BD61423046FF
:10B97000FBF714FF01300DD0104ABB682D1B45F0BA
:10B9800001055D60136830461B1B1360FBF79EFCCE
:10B990000120F8BD00213046FBF700FFBA68831A8A
:10B9A0000F2BDEDD43F001035360054B03491B6899
:10B9B000C01A0860D5E700BF48040024400C0024EA
:10B9C00050080024002961D0F8B50C460646FBF764
:10B9D00077FC54F8042C7B4FA4F1080522F00101F8
:10B9E00005EB010CB868DCF80430604523F0030374
:10B9F00000F08B80D207CCF8043032D454F8082CF5
:10BA0000AD1A1144AA6807F1080082426AD00CEB13
:10BA10000304D4F804E0EC68D4601EF0010FA260C7
:10BA200000F0978041F001036B60CCF80010B1F595
:10BA3000007F35D27A68CB08480901210133814063
:10BA40001143796007EBC30257F83310083AC5E990
:10BA5000021247F83350CD603046BDE8F840FBF79E
:10BA600035BC0CEB03025268D00710D4194407F11F
:10BA70000800DCF80830834273D0DCF80C20DA6070
:10BA8000936041F001036B606950D0E7704741F06B
:10BA90000103B1F5007F44F8043CCCF80010C9D391
:10BAA000B1F5206F4FEA512348D28B0903F13900D9
:10BAB00003F13802C300F818FB580838984259D0EF
:10BAC0005A6822F003028A4202D99B689842F7D151
:10BAD000D868C5E902308560DD603046BDE8F840D1
:10BAE000FBF7F4BB0CEB03025268D20763D40B44A0
:10BAF000DCE90212CA60916043F001026A603046DC
:10BB0000EB50BDE8F840FBF7E1BB0B44D10707D48D
:10BB100054F8082CAD1A1344D5E90212CA6091609A
:10BB200043F001026A60284ABD6012689A4293D8C5
:10BB3000264B30461968FFF7F5FE8DE7142B0AD91E
:10BB4000542B1FD80B0B03F16F0003F16E02C300DF
:10BB5000B1E719448DE703F15C0003F15B02C30018
:10BB6000A9E741F00103C7E90455C5E902006B608C
:10BB7000695071E779689210012404FA02F20A43CD
:10BB80007A60A6E7B3F5AA7F06D8CB0B03F178005D
:10BB900003F17702C3008EE740F25452934206D875
:10BBA0008B0C03F17D0003F17C02C30083E74FF4AB
:10BBB0007E737E227FE741F001036B60CCF80010BA
:10BBC0004AE700BF4804002454080024700C0024F5
:10BBD0009368002B00F081802DE9F04FB1F90C3013
:10BBE0000C461907804683B0174698B223D52369BF
:10BBF0000BB310F002033D682BD04FF0000ADFF8C2
:10BC0000B4B256465E453346524628BF5B46404670
:10BC1000002E4FD0E169D4F824C0E047002852DD5F
:10BC2000BB681B1A8244361ABB60002BEAD1002085
:10BC300003B0BDE8F08F21464046FEF787FC0028A0
:10BC400040F03481B4F90C303D6898B210F0020332
:10BC5000D3D110F0010942D14E463EB38205D4F84B
:10BC600008B040F18180B3455A4600F2B18010F42B
:10BC7000906F40F0BE8020680192494600F03EFE81
:10BC8000A3682168019AA3EB0B030A44B246A360A0
:10BC900022600026B868A0EB0A00D144B8600028F2
:10BCA000C5D0B4F90C0080B2002ED7D1D5E90096EA
:10BCB0000835D2E7D5E900A60835A3E72146404676
:10BCC000FFF754FD80B3B4F90C3043F040034FF05C
:10BCD000FF30A38103B0BDE8F08F002070471E46FF
:10BCE000AA46994618461D4656B388B34A46D4E933
:10BCF00004132068B24228BF3246884205D9A168A1
:10BD000003EB010B5A4500F3A780934264DCE16921
:10BD1000D4F824C02A464046E047B0F1000BD2DDFB
:10BD2000B9EB0B09CAD00120BB68A3EB0B035D4440
:10BD3000A6EB0B06BB60002B3FF479AF002ED4D1ED
:10BD40000AF1080353E902569A460833002EF9D047
:10BD500032460A212846F5F7E3FB002800F09D80D3
:10BD60000130A0EB0509C1E720682369984217D884
:10BD70006369B34214D86FF00042B24228BF324622
:10BD8000E16992FBF3F2D4F824C002FB03F34046CE
:10BD90004A46E047B0F1000A95DDA6EB0A0679E7CE
:10BDA000B345DA4628BFB2465246494600F0A6FDE2
:10BDB000A3682268A3EB0A035244A3602260002B0D
:10BDC000EBD121464046FFF7D1FC0028E5D07AE7C9
:10BDD0002068B34632464FE72946019200F08EFDB7
:10BDE000019AA3689B1AA3602368134423609346B7
:10BDF00096E723682169A3EB010B636903EB430A10
:10BE00000AEBDA7A0BF101034FEA6A0A334453452D
:10BE1000524684BF9A46524643052CD511464046A9
:10BE2000FAF74CFF00283BD05A4621690190F5F7FC
:10BE3000E9F8A289019B22F4906242F08002A2817B
:10BE400003EB0B002361AAEB0B03C4F814A0A3605F
:10BE50002060B34632460FE729465A4600F04EFDB1
:10BE600023685B44236021464046FFF77FFC00289F
:10BE70003FF456AF27E74046FBF7A4FA03460028F5
:10BE8000DED121694046FFF79DFDB4F90C300C224C
:10BE900023F08003C8F8002017E7721C914626E7BC
:10BEA0000C22B4F90C30C8F800200EE74FF0FF3038
:10BEB000BEE600BF00FCFF7F2DE9F8430746884639
:10BEC00000F538764FF00009D6E90154013D11D450
:10BED000A389012B05F1FF3508D9B4F90E300133E0
:10BEE000214603D03846C04749EA00096B1C04F1DB
:10BEF0006804EDD13668002EE6D14846BDE8F883E7
:10BF00002DE9F0410469B4EB611F2FDD00F1140E3F
:10BF10004E1111F01F0C0EEB84050EEB86032BD097
:10BF20005EF8262004339D4222FA0CF1CCF1200861
:10BF300018D977461A6802FA08F20A4347F8042B20
:10BF400053F8041B9D4221FA0CF1F3D8A41BA30063
:10BF5000053B9B0801330EEB83044EF82310C9B157
:10BF6000043417E0416174460029F9D100230361CC
:10BF700000234361BDE8F0819D4288BF00F11002BB
:10BF8000F4D953F8041B42F8041F9D42F9D8A41BAE
:10BF90000EEB8404A4EB0E039B1074450361E7D001
:10BFA000BDE8F0812DE9F04FA84C8BB024680590D6
:10BFB00020468946029207930394F5F741FA2146F9
:10BFC0000144D9F8003011F801BC997830290246B3
:10BFD00040F0DA816FF00100C01A033300EB030A6E
:10BFE0001C4613F8011B3029F8D0DFF8648218F8DA
:10BFF0000130002B00F0F0802378002718F8033080
:10C000003D4626462BB116F8013F18F80330002BA9
:10C01000F9D1039901923046FBF7F0FC019A0090A8
:10C02000002800F09180002D40F091803378009539
:10C0300003F0DF03502B354600F09380C9F8006011
:10C04000002F40F0AB802B1B013B072B394604DD52
:10C050005B10072B01F10101FADC0598049200F056
:10C06000C9FC049A0190002800F06782019BAC4251
:10C0700003F11406069680F0DC810027C2F101036B
:10C08000B946049310E0202F00F091803946043720
:10C0900015F8013C18F80330554603F00F038B40A8
:10C0A000A54249EA030916D915F8013C5B4505F19B
:10C0B000FF3AE8D1049B5344A342E4D318460399C2
:10C0C00009920893FBF79AFCDDE908320028DAD1DF
:10C0D0001D46A542E8D846F8049B069BF61A019B2C
:10C0E000B6101E61484600F05FFD029B76011C6899
:10C0F000301AA04200F3AE80C0F226810027029BD6
:10C10000009A9B689342C0F289810299009A4B6819
:10C1100093427EDD9D1AAC4200F3BC80CA68022ABD
:10C1200000F0BC81032A00F0B481012A00F098815C
:10C130000598019900F084FC5025149A00232846A4
:10C1400013600BB0BDE8F08F002D00F00B81AD1B2C
:10C15000AB000093337803F0DF03502B35467FF4B8
:10C160006DAF6B782B2B00F0ED802D2B6AD06E1C01
:10C17000002018F803104B1E182B61D8737818F89C
:10C1800003301039013623BB00B14942009BC9F886
:10C1900000600B440093002F3FF455AFBAF1000F3D
:10C1A00014BF0025062528460BB0BDE8F08F0021FE
:10C1B00046F8049B042789466AE701EB810103EBFB
:10C1C0004103A3F1100116F8013F18F80330002BCA
:10C1D000DAD0192BF1DDD7E7039900922046FBF75F
:10C1E0000DFC009A002873D1A15C18F80130A51845
:10C1F000002B6FD030292C4605D114F8013F302B8D
:10C20000FBD018F80330B3FA83F77F094FF0010A27
:10C21000F7E6012557B1029BDB68022B62D0032BA6
:10C2200064D0012B00F0858045F01005149B019A25
:10C230001A60079B009A1A6028460BB0BDE8F08F81
:10C240002E46FBE60120AB78AE1C92E7F4EE000828
:10C25000F0ED0008019D061B3146284601F0B4F8B8
:10C26000074678B1721E53110699012751F8231021
:10C2700002F01F0307FA03F30B4203D0BA4200F3A4
:10C28000E2800227009B0198334431460093FFF778
:10C2900037FE34E76E1E002F40F0C980002E40F0BC
:10C2A000CC807311069A019852F8232006F01F06DD
:10C2B000012303FA06F61642294618BF47F0020783
:10C2C000FFF71EFE029B5B680093641B0225A1E73B
:10C2D0002178254601F0DF01502900F0BD80C9F822
:10C2E00000505BE7159BC3F101031593159B002BD1
:10C2F0009AD0019BDDF818901E6900214B464FEA49
:10C30000860809EB860003E0984243F8041C3FD9F5
:10C310001F4653F8042BB2F1FF3FF5D00132022D36
:10C320003A6000F0C08014F01F0440F0E080212546
:10C330007CE7BA077FF578AF069B1B681F43FB07B6
:10C34000D7D471E700207EE7DDE90031221A9B1A7D
:10C350000598009300F0B2FD034614330190069354
:10C360000027CCE6B35C18F80310B0180646002985
:10C370003FF45EAE16F8013F18F803100029F9D11A
:10C38000801B8100009153E69C1C4FF0000A2CE6B4
:10C39000019B9B689E4280F28D803346019901EBA0
:10C3A000830201330B61022D4FF0010151617AD0FC
:10C3B0009E42B8DA002B40F3A780019A09EB830371
:10C3C000516902F1180083424FEA510140F2AF80F7
:10C3D0004C46026841EAC27144F8041B50F8041B41
:10C3E00083424FEA5101F4D8019A9B1A193B9B08EA
:10C3F000013349F8231009EB8303002940F09B80A7
:10C400000199A3EB090292104B450A617FD0029B70
:10C41000009A9B6801329342009288DA019905984C
:10C4200000F00EFB149A00231360A325BBE601273E
:10C4300037E7069E4FF000094DE60198314600F0BF
:10C44000C3FF07462DE7B11E284600F0BDFF0028B8
:10C450003FF417AF032715E700230093012780E679
:10C46000AC427FF465AE012C08D00198611E00F04B
:10C47000ABFF00283FF45CAE029B5B6807990B6042
:10C48000019B069901221A610A60149A62251360C1
:10C4900089E6159A002A3FF44BAEEFE7159A002A79
:10C4A0007FF446AEEAE7029B1B68013BA34232D011
:10C4B0002225BBE6019B05985968013100F09AFAE4
:10C4C000074600283FD0DDF80490D9F810304946DF
:10C4D00002339A000C310C30F4F794FD494605986C
:10C4E00000F0AEFA07F114093B69019756E7C8441A
:10C4F000C4F1200458F8040C00F056FBA042BFF62B
:10C5000016AF019B1B6955E7019A00231361019A3D
:10C51000002353617BE7631104F01F0459F82320C3
:10C520000123A34013420CBF222521257EE6C9F832
:10C5300000104B4669B1043362E7074B0748019A84
:10C54000DE2101F0A1FF044B04483A46842101F0AA
:10C550009BFF019B1961DAE7D4EC000868ED000845
:10C5600010B4046809E014F8013FA3F1410CBCF1D8
:10C57000190F98BF2033934208D111F8012B002ADC
:10C58000F1D101340460012010BC7047002010BCC0
:10C59000704700BF2DE9F04F096885B04B1111F0CD
:10C5A0001F01029002EB8303039140F08E801D1F58
:10C5B0000193029B01991C68002341F8043C6178B7
:10C5C0000134002900F09780DFF87091A846AC464E
:10C5D0009A461E460EE0202900F28B80B24506DA0C
:10C5E000C44501D2072B5BDD624551D3082314F803
:10C5F000011FA1B119F801000028ECD00133082B6C
:10C6000006F101063ADCDCF80010090100F00F0029
:10C610000843CCF8000014F8011F0029EAD1002ECD
:10C6200069D0E04501D9072B73DD624551D2111F56
:10C63000634653F8040B41F8040F9D42F9D2A5EB71
:10C640000C0323F00303691C04330CF1010C614556
:10C6500038BF04231344002143F8041B9D42FBD23E
:10C66000019B53F8043C2BB9AA4248D055F8043D2D
:10C67000002BF9D0052005B0BDE8F08F6245B6D299
:10C6800000234CF8043C1946ACF1040C0123BDE72F
:10C690000023ACF104084CF8043CB246C446A6E7BB
:10C6A000C3F108018900DCF80030C1F1200E6046BA
:10C6B0008B46416801FA0EF73B43036021FA0BF306
:10C6C00040F8043F4045F4D38EE7191D01911D4603
:10C6D0006FE7039B002BC3D0039B0198C3F120019C
:10C6E0004FF0FF33CB4050F8041C0B4040F8043CA3
:10C6F000B9E7292909D0042005B0BDE8F08F01234E
:10C7000005202B6005B0BDE8F08F029901340C6064
:10C7100085E7C3F108039B00DCF80010C3F1200794
:10C720006446666806FA07F00143216026FA03F1C1
:10C7300044F8041FA045F4D877E700BFF0ED0008E7
:10C74000014B93F8280170476008002400487047A7
:10C7500050090024704700BF704700BF704700BFFA
:10C76000704700BF38B50C46084D84461146204638
:10C770001A4600232B606446F6F720F9431C00D0CC
:10C7800038BD2B68002BFBD0236038BD840C0024FF
:10C790002DE9F0418B890C46990796B008D504F134
:10C7A00043030122C4E90432236016B0BDE8F081DE
:10C7B000B4F90E100029064627DB6A4601F0C2FFD5
:10C7C000002821DB019D05F47045A5F50055B5FA5B
:10C7D00085F54FF480686D094FF400674146304697
:10C7E000FAF76CFAB4F90C30F0B1204AF26343F076
:10C7F0008003C4F81480A3812060206135BB3B43D3
:10C80000A38116B0BDE8F081A38913F0800519D08B
:10C810004FF0400841463046FAF750FA0025B4F987
:10C820000C302F460028E0D19A05BED423F0030334
:10C8300004F1430243F002030121C4E90421A3816E
:10C840002260B2E74FF480682F46C7E7B4F90E10B4
:10C85000304601F08DFF10B9B4F90C30CFE7A38951
:10C8600023F0030343F001031BB2C8E7C9B7000874
:10C8700070B50C46B1F90E10002996B015461E464B
:10C8800014DB6A4601F05EFF00280FDB019A02F418
:10C890007042A2F50052B2FA82F24FF4806352095C
:10C8A0004FF4006032602B6016B070BDB4F90C100C
:10C8B000002311F08000336004D0402218462A6023
:10C8C00016B070BD4FF480632B6016B070BD00BF12
:10C8D00082B049B15AB16BB113780B601278101E57
:10C8E00018BF012002B0704701A9002AF3D11046F9
:10C8F00002B070476FF00100F4E700BF88420DD925
:10C900008B1883420AD900EB020CBAB1624613F8C5
:10C9100001CD02F801CD9942F9D170470F2A0ED806
:10C92000034602F1FF3C4AB10CF1010C013B8C447F
:10C9300011F8012B03F8012F6145F9D1704740EA46
:10C9400001039B0750D1A2F1100370B501F1200C37
:10C9500023F00F0501F1100E00F11004AC441B0987
:10C960005EF8105C44F8105C5EF80C5C44F80C5CFB
:10C970005EF8085C44F8085C5EF8045C44F8045C0B
:10C980000EF1100EE64504F11004E9D1013312F066
:10C990000C0F01EB031102F00F0400EB031327D07F
:10C9A000043C24F003064FEA940C1E441C1F8E46E0
:10C9B0005EF8045B44F8045FB442F9D10CF1010461
:10C9C00002F0030203EB840301EB840102F1FF3C5C
:10C9D0004AB10CF1010C013B8C4411F8012B03F816
:10C9E000012F6145F9D170BD02F1FF3C03469BE781
:10C9F0002246EBE7C36C70B505460C464BB153F8C5
:10CA0000240080B1026843F824200023C0E90333E6
:10CA100070BD2122042101F057FD0346E86400287F
:10CA2000EDD1002070BD012101FA04F6721D9200C3
:10CA3000284601F049FD0028F3D0C0E90146E4E7AB
:10CA400031B1C36C4A6853F82200086043F82210E1
:10CA5000704700BF2DE9F0410D6907460E461C46A0
:10CA600001F1140E0020DEF800108BB202FB03432C
:10CA70004FEA134C090C02FB01CC01309BB203EBD3
:10CA80000C4385424EF8043B4FEA1C44EBDC3CB1BE
:10CA9000B368AB4207DD06EB850301355C613561A8
:10CAA0003046BDE8F081716838460131FFF7A2FFDA
:10CAB0008046A8B13269023206F10C0192000C30B6
:10CAC000F4F7A0FAFB6C726853F82210316043F857
:10CAD0002260464606EB850301355C613561DFE780
:10CAE000024B03484246B52101F0CEFCD4EC0008CD
:10CAF0000CEF00082DE9F8430C4628491E4617465E
:10CB000003F1080281FB0231092E4FEAE273054668
:10CB1000C3EB610339DD4FF0010C00214FEA4C0CEF
:10CB2000634501F10101F9DC2846FFF763FF014687
:10CB300068B3089B4361092F4FF00103036112DCC6
:10CB40000A340927BE420BDDF61B264414F8013BCC
:10CB50000A22303B2846FFF77DFFA6420146F5D169
:10CB60000846BDE8F88304F10909C8463C4418F8B2
:10CB7000013B0A22303B2846FFF76CFFA0450146E7
:10CB8000F5D1A7F108044C44DCE70021CCE70A46C4
:10CB9000034B0448CE2101F077FC00BF398EE33807
:10CBA000D4EC00080CEF0008020C12040346CAB9CA
:10CBB0000304102013F07F4F04BF1B02083013F052
:10CBC000704F04BF1B01043013F0404F04BF9B00A3
:10CBD0000230002B05DB13F0804F00F1010008BF8D
:10CBE000202070470020E5E70368024613F00700A5
:10CBF00007D0D9071DD498071FD55B081360012003
:10CC0000704799B209B91B0C1020D9B209B9083084
:10CC10001B0A190704BF1B090430990704BF9B08AE
:10CC20000230D90703D45B0800F1010003D0136080
:10CC3000704700207047202070479B081360022037
:10CC4000704700BF38B5C36C04460D464BB15868F9
:10CC5000B0B102685A6000220123C0E90435C26005
:10CC600038BD2122042101F02FFC0346E064002896
:10CC7000EDD1094B094800224FF4A07101F004FCEA
:10CC80001C220121204601F01FFC0028F1D00122C6
:10CC90000223C0E90123DEE7D4EC00080CEF000812
:10CCA0002DE9F04F0E691569AE4285B088461446ED
:10CCB00005DB2A46234635460C4616469846A368A9
:10CCC0006168AF19BB42B8BF0131FFF793FE019015
:10CCD000002800F08780019B03F1140909EB870A03
:10CCE000D14505D24B46002243F8042B9A45FBD888
:10CCF00008F1140808EB860B04F11403D8451A4612
:10CD000003EB85055FD22B1B153B23F00303043394
:10CD10001534A54238BF0423CDE902A7AC461F460F
:10CD2000924605E0000C29D1C34509F1040948D910
:10CD300058F8040B85B2002DF4D056464C4600231B
:10CD400056F8040B216882B21FFA81FE05FB02EE41
:10CD5000000C0A0C734405FB002202EB13429BB249
:10CD600043EA0243B44544F8043B4FEA1243E7D890
:10CD700049F8073058F8040C000CD5D0D9F8003029
:10CD8000544619464D4600222688090C00FB061120
:10CD90000A449BB243EA024345F8043B54F8046B4F
:10CDA0002968360C8BB200FB063303EB1243A44513
:10CDB0004FEA1342E8D8C34549F8073009F104099E
:10CDC000B6D8DDE902A7002F02DC05E0013F03D061
:10CDD0005AF8043D002BF9D0019B18461F6105B09D
:10CDE000BDE8F08F034B0448019A40F25D1101F059
:10CDF0004BFB00BFD4EC00080CEF000812F003035B
:10CE00002DE9F0411446064632D10D46A41020D03B
:10CE1000D6F84880B8F1000F33D0E3074FF0000791
:10CE200007D4641015D0D8F80000A8B18046E307F5
:10CE3000F7D5424629463046FFF732FFB5B169685B
:10CE4000F36C641053F821202A6043F82150054602
:10CE5000E9D12846BDE8F081424641463046FFF719
:10CE60001FFFC8F8000007608046E0E70546D8E7E6
:10CE7000013B0F4A52F823200023FFF7EBFD054644
:10CE8000C4E701213046FFF7B5FD804640B10123DC
:10CE900040F27122C0E904320023B0640360BCE7B1
:10CEA000044B054842464FF4A07101F0EDFA00BF73
:10CEB00080F00008D4EC00080CEF00082DE9F047E2
:10CEC0000C4690462669A368496806EB6216751CF5
:10CED0009D4207464FEA621904DD5B009D4201F165
:10CEE0000101FADC3846FFF785FD8446002851D061
:10CEF000B9F1000F00F114000EDD09F105024FEA4F
:10CF0000820E03460CEB8202002143F8041B93427D
:10CF1000FBD1AEF114031844216904F1140318F095
:10CF20001F0803EB81012DD0C8F1200986464FF080
:10CF3000000A1A6802FA08F242EA0A024EF8042BC2
:10CF400053F8042B994222FA09FAF2D80B1B153B2D
:10CF500023F00303043304F11502914238BF042384
:10CF6000BAF1000F18BF2E4640F803A0FB6C6268B0
:10CF7000CCF8106053F822102160604643F822403C
:10CF8000BDE8F087043853F8042B40F8042F994289
:10CF9000F9D8EBE7034B0448624640F2D91101F09F
:10CFA00073FA00BFD4EC00080CEF00080B6984464C
:10CFB0000069C01A15D10CF1140C14310CEB83026A
:10CFC00010B401EB830301E0944508D252F8044DFC
:10CFD00053F8041D8C42F7D004D24FF0FF3010BC40
:10CFE00070477047012010BC704700BF2DE9F84F13
:10CFF0000F691369FF1A002F0E4690467AD101F18E
:10D000001405143202EB830205EB830301E09D4219
:10D0100073D253F8041D52F8044DA142F7D064D3E3
:10D020007168FFF7E7FC8146002872D03569D8F8AF
:10D030001020C76008F1140E06F1140009F1140A5B
:10D0400006F1100C0EEB820200EB8507564600211C
:10D050005EF8044B5CF804BFA3B211FA8BF1CB1A53
:10D06000210CC1EB1B4101EB23419BB243EA01437D
:10D07000724546F8043B4FEA2141E9D8A2EB080487
:10D08000153C08F11508424524F0030606F1040694
:10D0900038BF0426304424F0030238BF0022874200
:10D0A0005244B24416D95646044654F8043B11FA89
:10D0B00083F10A1402EB134289B241EA0243A74208
:10D0C00046F8043B4FEA2241EFD87A1E101A20F0AE
:10D0D0000302524423B952F8043D013D002BFAD01B
:10D0E000C9F810504846BDE8F88F33460127464638
:10D0F000984695E7F9DB002792E70021FFF77AFCD5
:10D10000814668B101220023C9E904234846BDE8ED
:10D11000F88F074B07484A464FF4107101F0B4F9F5
:10D12000034B04484A4640F2322101F0ADF900BFFA
:10D13000D4EC00080CEF00080F4B0B40A3F1507328
:10D14000002B02DD0020194670475B42B3F1A07F3F
:10D150004FEA235205DA4FF40023002043FA02F18C
:10D160007047143A1E2ADABF4FF0004323FA02F246
:10D1700001220021104670470000F07F2DE9F8439E
:10D18000066900F1140808EB8606A6F1040956F8B2
:10D19000047C3846FFF708FDC0F120030A280B6025
:10D1A00036DDC8451ED2B0F10B0356F8082C26D048
:10D1B000C3F1200C22FA0CF19F400F43A6F10801A5
:10D1C00047F07F55884545F440153AD202FA03F0FE
:10D1D00056F80C3C23FA0CF303431C462046294620
:10D1E000BDE8F883B0F10B0308D007FA03F343F06E
:10D1F0007F55002345F440151C46EFE71A4647F0DB
:10D200007F5545F44015144620462946BDE8F8836D
:10D21000C0F10B0327FA03F2C84542F07F553CBF2B
:10D2200056F8082CDA4000F1150328BF002207FA4F
:10D2300003F345F4401543EA020420462946BDE8BD
:10D24000F88302FA03F31C46C8E700BF70B501215A
:10D2500082B016461D46FFF7CDFB044600284BD092
:10D260002B46C5F30A55C3F313030DB143F48013E2
:10D27000002E019322D068460096FFF7B5FC0028E7
:10D2800036D0019B0099C0F1200203FA02F20A4352
:10D29000C34001936261002B14BF02210121A361ED
:10D2A0002161ADB1069AA5F2334303441360079B95
:10D2B000C0F135001860204602B070BD01A8FFF72C
:10D2C00093FC019B0121C4E904132030002DE9D116
:10D2D00004EB8102A0F232431069069A1360FFF753
:10D2E00063FC079BC0EB41112046196002B070BD82
:10D2F000DDE900236261CEE7034B0448224640F299
:10D300000A3101F0C1F800BFD4EC00080CEF0008AE
:10D310002DE9F04383B00F4669468046FFF72EFFA4
:10D3200004460D46384601A9FFF728FFD8F810300B
:10D330003A690F469A1ADDE90013CB1A03EB421340
:10D34000002B06460BDD05EB03594D4632463B46A6
:10D3500020462946F4F75EFA03B0BDE8F083C3EB3C
:10D36000033307EB03510F46F0E700BF01394911C2
:10D3700001F1010C116902F1140303EB81018B42ED
:10D3800000EB8C0C16D210B5A0F1040E53F8044B30
:10D390004EF8044F9942F9D88B1A153B23F003033A
:10D3A00004331844844504D9002340F8043B8445E1
:10D3B000FBD810BD844505D9002340F8043B8445C3
:10D3C000FBD87047704700BF03694A11934200F1D0
:10D3D000140009DA00EB830302E053F8042DC2B90C
:10D3E0008342FAD80020704710DD11F01F010DD0E4
:10D3F00010B450F8224000EB820324FA01F202FA42
:10D4000001F18C420BD0012010BC704700EB82036D
:10D41000E6E70120704753F8042D002AF3D1834238
:10D42000F9D8002010BC704738B50C46084D84462A
:10D43000114620461A4600232B606446F5F7C6FACB
:10D44000431C00D038BD2B68002BFBD0236038BDB7
:10D45000840C0024DFF860C0F8B521F000430027F9
:10D46000634504460D461646176022DC844653EA9F
:10D470000C0C1ED0DFF844C001EA0C0C0A46BCF1CB
:10D48000000F09D10E4B0022F4F79AF86FF0350720
:10D4900004460A4621F0004322F0FF421B1522F405
:10D4A000E002A3F2FE3342F07F553B4445F4001501
:10D4B000336020462946F8BDFFFFEF7F0000F07F74
:10D4C0000000504301490020704700BF0000F87F72
:10D4D00030B540EA0104A30701D1032A0FD88446DE
:10D4E00001F1FF3E07E01EF8011F03F8011B541E67
:10D4F000C1B19C4622466346002AF4D130BD0B469A
:10D500008446194653F8045BA5F1013424EA050466
:10D5100014F0803FE4D1043A032A4CF8045B194626
:10D52000EFD8DDE76244002CE8D003F8011B9342FA
:10D53000FBD130BD2DE9F84F4B6E9C0490462DD5A4
:10D540009368126843B38B46064602F1080959E90D
:10D55000025A5FEA9A0715D0043D002401E0A74271
:10D560000ED055F8041F5A46304601F0B7F8431C58
:10D5700004F10104F3D10023C8E90133BDE8F88FB9
:10D58000D8F808302AF0030AA3EB0A03C8F80830D9
:10D5900009F10809002BDAD10020ECE7FEF718FBAF
:10D5A0000023C8E90133BDE8F88F00BF10B49468C8
:10D5B00014B110BCFFF7BEBF2046546010BC7047CA
:10D5C0002DE9F04FBDB0CDE904301C46019117465E
:10D5D00018B1836B002B00F08682019A536EDE0730
:10D5E00040F18F81B2F90C108AB2900408D441F452
:10D5F000005201994B6E8A8123F4005392B24B661C
:10D60000110740F1F780019B1B69002B00F0F280AD
:10D6100002F01A030A2B00F0FB8013AB10930023D7
:10D62000CDE91133CDE90A3308930DF14C09099383
:10D6300003933B78002B00F051813C4604E014F842
:10D64000013F002B00F02C81252BF8D1E51B40F089
:10D6500029812378002B00F041814FF00003002541
:10D660008DF83B30671C637802954FF0FF3B2B240D
:10D670000137A3F120025A2A00F25281DFE812F0AA
:10D6800098025001500194025001500150016A006B
:10D690005001500136026B0250014102A6025001B6
:10D6A000A2025B005B005B005B005B005B005B0059
:10D6B0005B005B00500150015001500150015001CE
:10D6C00050015001500123028400500150015001CB
:10D6D0005001500150015001500150015001DD0036
:10D6E00050015001500107025001590250015001F0
:10D6F0001E055001500150015001500150015001D0
:10D700005001500150012302860050015001500188
:10D710004F02860080005001450250018102DF0067
:10D720006F028000500107027E003E05500150014B
:10D73000400550017E00A3F13002002117F8013BA3
:10D7400001EB810102EB4101A3F13002092AF5D975
:10D7500002918EE7DDF814804046FEF7F7FF43683C
:10D760000A931846F3F76CFE0B9006464046FEF708
:10D77000EDFF83680993002E40F07B843B7877E7C8
:10D780003B7845F0200573E745F01005AC06049E94
:10D7900040F16F81073626F007063246736852F86B
:10D7A000086B04929846002BC0F22D84BBF1FF3F1A
:10D7B00000F0108556EA080325F0800A00F008847E
:10D7C0000A2E78F1000380F0BD84303601238DF8F5
:10D7D000EF60554600930DF1EF04DDF800809DF8F1
:10D7E0003B30D845B8BFD846002B00F0A88008F1E0
:10D7F0000108A4E0019D05982946FCF7A7FE002832
:10D8000040F08885AA8902F01A030A2B7FF405AF3D
:10D810000199B1F90E30002BFFF6FFAE4B6EDE071B
:10D8200002D4950540F156850199059823463A465C
:10D830003DB0BDE8F04F00F093BD45F0100515F088
:10D84000200800F00781049E073626F007063346BD
:10D85000D6F8048053F8086B049325F4806A0023FB
:10D860004FF000028DF83B20BBF1FF3F00F0C88174
:10D8700056EA08022AF0800540F0C181BBF1000F92
:10D8800040F0AB84002B40F0A8831AF00103009312
:10D8900000F0D68330238DF8EF300DF1EF049CE7D4
:10D8A000E51B1BD0119B129A01332A44072BC9E9AF
:10D8B00000751292119305DC09F10809039B2B44B2
:10D8C0000393C6E6002A00F07F830199059810AA09
:10D8D000FFF730FE40B90DF14C09EFE7129B002B2A
:10D8E00040F0098500231193019A536ED90740F146
:10D8F000A68093895B0600F1198503983DB0BDE8C9
:10D90000F08F019BB3F90C108D058AB23FF56DAE17
:10D910001D46986DFEF722FFB5F90C108AB264E639
:10D92000002BDBD08DF88C304FF001084FF0000356
:10D930008DF83B30CDF8008023AC4FF0000B15F094
:10D940000203069318BF08F1020815F08403079339
:10D9500005D1029BA3EB0806002E00F36C82DDE9E3
:10D960001121501C9DF83B608EB10DF13B0201313D
:10D97000C9F8002007284FF00102CDE91101C9F8CC
:10D98000042000F33B82024609F108090130069B9E
:10D99000DBB10FAB0231C9F8003007284FF00203AA
:10D9A000CDE91101C9F8043040F34082002900F0AC
:10D9B00006830199059810AAFFF7BCFD002893D1B2
:10D9C000DDE911210DF14C09501C079B802B00F063
:10D9D0005881009BABEB0306002E00F3B681009B41
:10D9E000C9F8004019440728CDE91101C9F80430ED
:10D9F00040F34481002900F072820199059810AA31
:10DA0000FFF798FD00287FF46FAF12990DF14C09D4
:10DA1000680705D5029BA3EB0804002C00F369827C
:10DA2000DDE902234245ACBF9B1843440393002920
:10DA300040F0D581002311930DF14C09F9E5019BCC
:10DA40009B899A053FF556AF019CA06DFEF788FEB5
:10DA5000A3894FE715F0100340F0238315F040022F
:10DA600000F0EB83049A52F8046B04929846B6B225
:10DA7000F3E656F8043B0496E80600F1ED826906E9
:10DA800040F1E78243F3C0381EB243468BE6049E62
:10DA900056F8044B4FF000038DF83B30002C00F09B
:10DAA000B183BBF1FF3F00F02E835A460021204690
:10DAB000F3F736FD002800F01284031B0093049650
:10DAC0004FF0000B89E6049E4FF000038DF83B30C9
:10DAD0004FF0010856F8043B8DF88C300496CDF8D1
:10DAE000008023AC29E7FDF775FE76E5049B53F82B
:10DAF000042B0292002A80F29F82029A04935242DF
:10DB000002923B7845F00405B2E53B786C2B03BFED
:10DB10007B7845F02005013745F01005A8E53B78F6
:10DB2000682B03BF7B7845F40075013745F040054D
:10DB30009EE545F0100A1AF0200800F05582049E78
:10DB4000073626F007063346D6F8048053F8086BEC
:10DB50000493012384E63B788DF83B4088E5049BE1
:10DB600053F8046B049330238DF83C3078238DF800
:10DB70003D30B94B089345F0020A4FF000080223EC
:10DB80006EE6AE0600F18382EC0600F13383680690
:10DB900000F19283A90540F12D83049E039A56F863
:10DBA000043B04961A7044E53B7845F001055FE5B7
:10DBB0009DF83B30002B7FF4E1AD20238DF83B3006
:10DBC0003B7855E53B7845F0800551E5394611F83D
:10DBD000013B2A2B00F0B383A3F13002092A0F4640
:10DBE0004FF0000B3FF645AD17F8013B0BEB8B0BED
:10DBF00002EB4B0BA3F13002092AF5D939E5AA460D
:10DC0000012B3FF4DDAD022B3CAC12D1089A06F09B
:10DC10000F033609D35C04F8013D46EA08764FEA63
:10DC2000181856EA0803F2D13CAB1B1B554600936B
:10DC3000D3E506F00703F60846EA48764FEAD80827
:10DC4000303356EA0801224604F8013DF1D11AF0BA
:10DC5000010FE9D0302BE7D03023023A04F8013C21
:10DC60003CAB9B1A554600931446B6E500991394B5
:10DC700001231491129111930DF14C0909F1080936
:10DC8000C6E6029BA3EB0806002E7FF7A2AE102E7D
:10DC900040F35183DFF8C4A15346CDE906B4BA4638
:10DCA000DDF814B0019C2F461D4607E002F1020C7E
:10DCB00009F108090246103E102E1EDD501C1031DD
:10DCC00010230728CDE91101C9F80050C9F8043024
:10DCD000ECDD10AA002900F08B80214658460DF19A
:10DCE0004C09FFF727FC00287FF4FEADDDE9112188
:10DCF000103E102E02F1010CE0DCDDE906B42B46EB
:10DD00003D4657469A463144BCF1070FCDE911C153
:10DD1000C9F800A0C9F8046040F39581002900F01B
:10DD2000BB820199059810AAFFF704FC00287FF434
:10DD3000DBAD009BDDE91121ABEB0306002E02F108
:10DD400001000DF14C097FF74AAE102EDFF80CA14F
:10DD500031DD5346CDE90645BA46059C019D4FF09D
:10DD6000100B1F4607E002F1020C09F108090246F8
:10DD7000103E102E19DD501C10310728C9E9007B18
:10DD8000CDE91101EFDD10AA19B3294620460DF1A6
:10DD90004C09FFF7CFFB00287FF4A6ADDDE9112188
:10DDA000103E102E02F1010CE5DCDDE906453B4694
:10DDB000604657469A4631440728CDE91101C9F813
:10DDC00000A0C9F8046000F3E68009F108090130F9
:10DDD00005E64FF0010C0A460DF14C09C8E7019920
:10DDE000059810AAFFF7A6FB00283FF423AE7BE5B9
:10DDF0004FF0010C0A460DF14C095CE7002900F0D8
:10DE0000DB800199059810AAFFF794FB00287FF4A6
:10DE10006BADDDE911210DF14C09501CB7E5022174
:10DE20000FAB1491139301200DF14C09024609F137
:10DE30000809501CC9E5102E40F35782DDE911C1D5
:10DE4000DFF81CA0CDE90CB410235446DDF804B073
:10DE5000DDF814A062460DE070EC00089CF00008AC
:10DE60008CF0000802F1020C09F108090246103E8C
:10DE7000102E1BDD501C10310728C9E90043CDE9E5
:10DE80001101EFDD10AA21B3594650460DF14C099E
:10DE9000FFF750FB00287FF427ADDDE91121103E8C
:10DEA000102E02F1010C4FF01003E3DCA246DDF866
:10DEB00030B00D9C62463144072ACDE91121C9F8E2
:10DEC00000A0C9F8046000F3A78009F10809501CFC
:10DED00048E50A464FF0010C0DF14C09C7E76C0705
:10DEE000119150D5029BA3EB0804002C4BDD0DF1E2
:10DEF0004C09102C40F30982DFF8ECA2119A059E20
:10DF0000DDF804B053461025BA461F4606E0901CC3
:10DF100009F108091A46103C102C19DD531C103168
:10DF2000072BC9E90075CDE91131F0DD10AA29B33D
:10DF300059463046FFF7FEFA00287FF4D5ACDDE9FC
:10DF40001121103C102C02F101000DF14C09E5DC0F
:10DF50003B4657469A4621440728C9E900A4CDE923
:10DF600011017FF75DAD71B10199059810AAFFF716
:10DF7000E1FA00287FF4B8AC129951E501200A4675
:10DF80000DF14C09C7E7DDE902234245ACBF9B1800
:10DF9000434403934EE500293FF468AE0199059888
:10DFA00010AAFFF7C7FA00287FF49EAC11981299C7
:10DFB00001300DF14C0912E5069B002B77D10120B1
:10DFC0000A460DF14C0900E511920DF14C0975E47A
:10DFD000BBF1000F7FF4F9AB55464FF0000BCDF8C5
:10DFE00000B03CACFFF7F9BB1AF010033AD11AF0BD
:10DFF000400200F01381049A52F8046B0492984690
:10E00000B6B201232CE42D2376428DF83B3068EB29
:10E010004808AA46012327E400297DD001990598E4
:10E0200010AAFFF787FA00287FF45EACDDE9112122
:10E030000DF14C09501C95E404933B78FFF718BB95
:10E040003CACFFF7CABB09F108090CF101006246BC
:10E05000BFE4AA0500F138814FEAE3781E46434643
:10E06000FFF7A1BB049B53F8046B04930123FFF754
:10E07000F7BB099B002B3FF481AB099B1B78002B5E
:10E080003FF47CAB3B7845F48065FFF7F1BADDE9FE
:10E09000031656F8042B0496CB17C2E90013FFF7BA
:10E0A000C8BA049B53F8046B0493FFF7D6BB022154
:10E0B0000FAB149113930DF14C09B8E64B4A08923B
:10E0C00015F0200836D0049E073626F007063246A3
:10E0D000D6F8048052F8086B0492EA0709D556EA8C
:10E0E000080206D08DF83D30302345F002058DF84A
:10E0F0003C3025F4806A0223FFF7B2BBAA461AE53A
:10E100003B4A0892DCE720460496F3F799F94FF072
:10E11000000B0090FFF761BB9DF83B20002A00F048
:10E12000C18001200DF13B02149013920DF14C09B6
:10E13000014628E415F0100242D0049A52F8046B0C
:10E140000492CAE70AF48063CDF800B0CDF81890C5
:10E15000BB46DDF8249000253CAC1F4609E0304664
:10E160004146F2F7CDFD0A2E78F100031BD3064697
:10E170008846304641460A220023F2F7C1FD114687
:10E18000303104F8011C0A220023013C0135002F24
:10E19000E5D099F80010A942E1D1FF2DDFD00A2E79
:10E1A00078F1000364D23CAB1B1BCDF824905F4692
:10E1B000DDF81890DDF800B000935546FFF70DBB71
:10E1C00015F0400147D0049951F8046B0491904632
:10E1D000B6B282E7AA46FFF7F3BA012BAA467FF44C
:10E1E00012ADFFF7F2BA00BF8CF0000884EC000813
:10E1F00070EC0008049E039A56F8043B1A600496DB
:10E20000FFF717BABBF1060FD84628BF4FF0060834
:10E21000504CCDF800800496FFF78FBB049B1AF496
:10E22000007814BF53F8046B53F8046B04931CBFBD
:10E230009046F6B20123FFF713BB049B15F4007858
:10E2400014BF53F8046B53F8046B04931CBF90463F
:10E25000F6B2FFF702BB049A15F4007814BF52F827
:10E26000046B52F8046B04921CBF8846F6B234E784
:10E270000B9B0A99E41A1A462046FFF729F999F8E8
:10E2800001300BB109F10109304641460A22002351
:10E290000025F2F735FD6AE701200A460DF14C0929
:10E2A000FFF797BB069B002B7FF4B9AD0A46012010
:10E2B0000DF14C09FFF78DBB049E039A56F8043B01
:10E2C00004961A80FFF7B5B943F3C0185EB243460F
:10E2D000FFF769BA886DFEF743FAFFF7A5BACDF8E4
:10E2E00000B004968346FFF778BA119A1299DFF8C6
:10E2F00068A00132DFE50199059810AAFFF71AF925
:10E3000000283FF4EFAAFFF7EFBA1198DFF848A012
:10E31000013020E6019B5B6EDB0707D4019B9B89E4
:10E320009F0503D4019B986DFEF71AFA4FF0FF3357
:10E330000393FFF7E2BADFF824A08446E3E4049AEB
:10E340007B780F4652F8041B049241EAE17BFFF709
:10E350008FB900BF98EC00088CF000089CF0000812
:10E36000F0B51F468B89ADF26C4D23F00203ADF87A
:10E370000C304B6E1993CB89ADF80E30CB690793F7
:10E380004B6A09931AAB009304934FF480631546CC
:10E3900006460293059316A800230C460693FEF743
:10E3A000D9F92A463B4669463046FFF709F9051E6A
:10E3B00007DB69463046FDF7D9F9002818BF4FF052
:10E3C000FF35BDF80C305B0603D5A38943F040034D
:10E3D000A3811698FEF7C0F928460DF26C4DF0BDEA
:10E3E00049B1FF2A02D80A70012070478A230360CE
:10E3F0004FF0FF3070470846704700BF2DE9F047E7
:10E40000DFF87CA00646DAF8000098460F469146F1
:10E41000FEF7A4F91B4B1B68D3F8484124B3656889
:10E420001F2D26DC5EB96B1C0235DAF80000636034
:10E4300044F82570FEF794F90020BDE8F08704EB5E
:10E4400085010123C1F88890D4F88821AB401A4394
:10E45000022EC4F88821C1F80881E4D1D4F88C21B7
:10E460001343C4F88C31DEE703F5A674C3F84841C2
:10E47000D5E7DAF80000FEF773F94FF0FF30DCE77C
:10E4800058080024FCEB000800B50B4C2568144626
:10E49000EE681A4685B003460D464CB10749009513
:10E4A000CDE901143046064900F0B0F800F0E8F973
:10E4B00004490C46F3E700BF1C000024ACF0000840
:10E4C000BCF0000828EA000838B5A1FB02148CBB98
:10E4D000F8F7F4FB0546E0B150F8042C22F00302F3
:10E4E000043A242A17D8132A1AD91B2AC0E900444F
:10E4F0001DD9242A14BF00F1100200F118024FF0B8
:10E500000003C0E9024404BF04614461C2E900336E
:10E510009360284638BD2146F8F780FE284638BD6E
:10E5200002460023C2E900339360284638BD00F15B
:10E530000802F6E7F8F788FB0C2300250360E8E7FC
:10E5400070B500294BD006460C4610B1836B002BEA
:10E5500048D0636ED80734D5B4F90C30002B3ED0C8
:10E5600021463046FDF772F8E36A054633B1E169AA
:10E57000304698470028B8BF4FF0FF35A3891A06E8
:10E580003BD4216B41B104F14003994202D03046A3
:10E59000FDF718FA00232363616C21B13046FDF7C3
:10E5A00011FA00236364FDF79BF9636E0022DB0719
:10E5B000A28127D5A06DFEF7CFF8FDF797F9284681
:10E5C00070BDA3899905CBD4A06DFEF7C7F8B4F947
:10E5D0000C30002BC4D1656E15F0010508D0002564
:10E5E000284670BDFDF7F6F8636ED807B4D4E8E7A7
:10E5F000A06DFEF7B5F8284670BD21693046FDF7DD
:10E60000E1F9BEE7A06DFEF7ABF8D3E70EB410B5A5
:10E6100083B005AB064C53F8042B019301462068E8
:10E62000FEF7CEFF03B0BDE8104003B0704700BF57
:10E630001C0000242DE9F04383B0074688461446A9
:10E64000FEF77EF8012803D108F1FF33FE2B37D9FE
:10E65000424604F15C0301A9384600F0F3F8421C7D
:10E66000064633D038B39DF804C00DF105090025E6
:10E6700009E023685A1C226083F800C00135B542C6
:10E6800019D219F801CBA368013B002BA360F0DA83
:10E69000D4F818E0734561462246384602DBBCF1E7
:10E6A0000A0FE6D100F076F8431CE7D10646304663
:10E6B00003B0BDE8F0834646304603B0BDE8F083C2
:10E6C0005FFA88FC8DF804C00646CEE7A389304681
:10E6D00043F04003A38103B0BDE8F08330B5536E2F
:10E6E00013F0010FB2F90C30144683B005469AB20C
:10E6F00001D198051CD5900406D4626E43F40053F2
:10E7000042F40052A381626622462846FFF792FF38
:10E71000636EDA07054602D4A3899B0502D5284615
:10E7200003B030BDA06DFEF71BF8284603B030BD26
:10E73000A06D0191FEF712F8B4F90C3001999AB26C
:10E74000D9E700BF70B50C46084D034600262046A9
:10E7500011461C462E60F4F751F9431C00D070BDE1
:10E760002B68002BFBD0236070BD00BF840C0024FD
:10E7700038B5074D0022044608462A60F4F7ECF845
:10E78000431C00D038BD2B68002BFBD0236038BD64
:10E79000840C0024F8B50D461446064610B1836B70
:10E7A000002B43D0B4F90C20A369A360170790B2E3
:10E7B0001BD52369CBB1EDB281042F4622D5226847
:10E7C0006169D31A994229DD0133A1680139A16039
:10E7D000511C2160157062699A422AD0A389DB0717
:10E7E00001D50A2D25D03846F8BD21463046FBF725
:10E7F000ADFE20BBB4F90C20236990B2EDB28104C8
:10E800002F46DCD442F40052A281626E616922F488
:10E81000005262662268D31A9942D5DC21463046FE
:10E82000FCF7A4FF58B922680123CEE7FCF7D2FF1A
:10E83000B8E721463046FCF799FF0028D3D04FF0C7
:10E84000FF37D0E770B5054684B01C4639B10B4E92
:10E85000D6F8E060B047431C09D004B070BD0A464A
:10E860000649D1F8E06001A9B047431CF5D1002268
:10E870008A2322602B6004B070BD00BF60080024B2
:10E8800008B5062000F004F80120F4F7FDF800BFF9
:10E8900038B5154B1F281D6820D8D5F8DC22044652
:10E8A00062B152F820304BB1012B15D0591C0FD05A
:10E8B000002542F820509847284638BD284600F0E9
:10E8C0002BF8224601462846BDE8384000F00EB835
:10E8D00016232B60012038BD002038BD16232B6085
:10E8E0004FF0FF3038BD00BF1C00002470B50C464F
:10E8F000084D03460026204611461C462E60F4F7BC
:10E90000BBF8431C00D070BD2B68002BFBD02360EC
:10E9100070BD00BF840C0024F4F7ACB8F8B500BF9C
:10E92000F8BC08BC9E467047F8B500BFF8BC08BCF0
:04E930009E46704748
:10E938007374203D2025640A00000000313233340E
:10E9480035363738393031003132333435363738A7
:10E958000000000032303234303133310000000022
:10E968004972697300000000EFBBBF006E756C6CE4
:10E97800000000002564000025312E3135670000B5
:10E98800256C670025312E313767000066616C738E
:10E998006500000074727565000000004A534F4E10
:10E9A80020737472696E673A2025730D0A0000009F
:10E9B80074656D706572617475726500706E0000C3
:10E9C800736E000070726F64756374696F6E5F6454
:10E9D800617465006D616E756661637475726572E8
:10E9E800000000006465766963655F706978656C2E
:10E9F8005F6C656E677468007365745F696E7465D3
:10EA080067726174696F6E5F74696D6500000000FC
:10EA180054656D70657261747572653A2025640A73
:10EA280000000000506E3A25640A0000536E3A2533
:10EA3800640A000050726F64756374696F6E5F6476
:10EA48006174653A25640A004D616E756661637488
:10EA5800757265723A25640A00000000446576699B
:10EA680063655F506978656C5F4C656E6774683A7A
:10EA780025640A005365745F496E74656772617432
:10EA8800696F6E5F54696D653A25640A000000007D
:10EA98004A534F4E2070617273696E6720657272B7
:10EAA8006F722E0054656D70657261747572653A87
:10EAB800252E31660D0A0000000000000102030443
:10EAC8000102030406070809010002000400060009
:10EAD80008000A000C00100020004000800000011F
:10EAE80008040204080101010101010307010000F3
:10EAF8000020202020202020202028282828282006
:10EB080020202020202020202020202020202020FD
:10EB18002088101010101010101010101010101065
:10EB28001004040404040404040404101010101055
:10EB3800101041414141414101010101010101011F
:10EB48000101010101010101010101011010101071
:10EB580010104242424242420202020202020202F1
:10EB68000202020202020202020202021010101045
:10EB7800200000000000000000000000000000006D
:10EB8800000000000000000000000000000000007D
:10EB9800000000000000000000000000000000006D
:10EBA800000000000000000000000000000000005D
:10EBB800000000000000000000000000000000004D
:10EBC800000000000000000000000000000000003D
:10EBD800000000000000000000000000000000002D
:10EBE800000000000000000000000000000000001D
:10EBF80000000000200000246E660000696E697441
:10EC080079000000616E000035000000CEFBFFFFB8
:10EC1800CB030000010000000000000034000000E9
:10EC2800CEFBFFFFCB030000010000000000000046
:10EC3800BC89D897B2D29C3C33A7A8D523F64939CA
:10EC48003DA7F444FD0FA5329D978CCF08BA5B25EC
:10EC5800436FAC6428066811494E4600696E660029
:10EC68004E414E006E616E003031323334353637E6
:10EC78003839616263646566000000003031323300
:10EC880034353637383941424344454600000000A0
:10EC9800286E756C6C2900003000000020202020B0
:10ECA800202020202020202020202020303030301C
:10ECB8003030303030303030303030304E614E000F
:10ECC800496E66696E6974790000000042616C6C77
:10ECD8006F63207375636365656465640000000095
:10ECE8002F6D6E742F776F726B73706163652F77FA
:10ECF8006F726B73706163652F4743432D31302DFD
:10ED0800706970656C696E652F6A656E6B696E7384
:10ED18002D4743432D31302D706970656C696E65E0
:10ED28002D3333385F32303231313031385F31365C
:10ED380033343531363230332F7372632F6E657743
:10ED48006C69622F6E65776C69622F6C6962632FDC
:10ED58007374646C69622F64746F612E63000000C1
:10ED68002F6D6E742F776F726B73706163652F7779
:10ED78006F726B73706163652F4743432D31302D7C
:10ED8800706970656C696E652F6A656E6B696E7304
:10ED98002D4743432D31302D706970656C696E6560
:10EDA8002D3333385F32303231313031385F3136DC
:10EDB80033343531363230332F7372632F6E6577C3
:10EDC8006C69622F6E65776C69622F6C6962632F5C
:10EDD8007374646C69622F6764746F612D676574FE
:10EDE8006865782E63000000000000000000000045
:10EDF800000000000000000000000000000000000B
:10EE080000000000000000000000000000000000FA
:10EE1800000000000000000010111213141516174E
:10EE28001819000000000000001A1B1C1D1E1F00FE
:10EE380000000000000000000000000000000000CA
:10EE48000000000000000000001A1B1C1D1E1F000F
:10EE580000000000000000000000000000000000AA
:10EE6800000000000000000000000000000000009A
:10EE7800000000000000000000000000000000008A
:10EE8800000000000000000000000000000000007A
:10EE9800000000000000000000000000000000006A
:10EEA800000000000000000000000000000000005A
:10EEB800000000000000000000000000000000004A
:10EEC800000000000000000000000000000000003A
:10EED800000000000000000000000000000000002A
:10EEE80000000000000000002E000000F0EE000806
:10EEF80028EA00085C08002443000000504F5349EA
:10EF0800580000002F6D6E742F776F726B737061ED
:10EF180063652F776F726B73706163652F47434327
:10EF28002D31302D706970656C696E652F6A656E5C
:10EF38006B696E732D4743432D31302D70697065B1
:10EF48006C696E652D3333385F3230323131303190
:10EF5800385F313633343531363230332F7372639C
:10EF68002F6E65776C69622F6E65776C69622F6C9E
:10EF78006962632F7374646C69622F6D7072656364
:10EF88002E630000000000000080E03779C3414391
:10EF9800176E05B5B5B89346F5F93FE9034F384DF7
:10EFA800321D30F94877825A3CBF737FDD4F1575A3
:10EFB800000000000000F03F0000000000002440B6
:10EFC80000000000000059400000000000408F4091
:10EFD800000000000088C34000000000006AF840FC
:10EFE8000000000080842E4100000000D012634120
:10EFF8000000000084D797410000000065CDCD4196
:10F00800000000205FA00242000000E87648374276
:10F01800000000A2941A6D42000040E59C30A24214
:10F028000000901EC4BCD64200003426F56B0C4389
:10F038000080E03779C3414300A0D8855734764330
:10F0480000C84E676DC1AB43003D9160E458E14391
:10F05800408CB5781DAF154450EFE2D6E41A4B4406
:10F0680092D54D06CFF08044F64AE1C7022DB5444B
:10F07800B49DD9794378EA440500000019000000DE
:10F088007D0000002020202020202020202020207B
:10F0980020202020303030303030303030303030A8
:10F0A800303030302C2066756E6374696F6E3A208C
:10F0B80000000000617373657274696F6E20222509
:10F0C8007322206661696C65643A2066696C652004
:10F0D800222573222C206C696E65202564257325F2
:04F0E800730A0000A7
:08F0EC00441CFF7F010000003D
:08F0F40021A60008E502000856
:04F0FC00C102000845
:10F100009D6C0008AD6C0008AD7300080090D00342
:10F110000090D00301000000100000002000002437
:10F12000000000000C03002474030024DC0300240E
:10F1300000000000000000000000000000000000CF
:10F1400000000000000000000000000000000000BF
:10F1500000000000000000000000000000000000AF
:10F16000000000000000000000000000000000009F
:10F17000000000000000000000000000000000008F
:10F18000000000000000000000000000000000007F
:10F19000000000000000000000000000000000006F
:10F1A000000000000000000000000000000000005F
:10F1B000000000000000000000000000000000004F
:10F1C000000000000000000001000000000000003E
:10F1D0000E33CDAB34126DE6ECDE05000B00000003
:10F1E000000000000000000000000000000000001F
:10F1F000000000000000000000000000000000000F
:10F2000000000000000000000000000000000000FE
:10F2100000000000000000000000000000000000EE
:10F5500048040024480400245004002450040024DB
:10F56000580400245804002460040024600400248B
:10F57000680400246804002470040024700400243B
:10F5800078040024780400248004002480040024EB
:10F59000880400248804002490040024900400249B
:10F5A0009804002498040024A0040024A00400244B
:10F5B000A8040024A8040024B0040024B0040024FB
:10F5C000B8040024B8040024C0040024C0040024AB
:10F5D000C8040024C8040024D0040024D00400245B
:10F5E000D8040024D8040024E0040024E00400240B
:10F5F000E8040024E8040024F0040024F0040024BB
:10F60000F8040024F8040024000500240005002468
:10F610000805002408050024100500241005002416
:10F6200018050024180500242005002420050024C6
:10F630002805002428050024300500243005002476
:10F640003805002438050024400500244005002426
:10F6500048050024480500245005002450050024D6
:10F660005805002458050024600500246005002486
:10F670006805002468050024700500247005002436
:10F6800078050024780500248005002480050024E6
:10F690008805002488050024900500249005002496
:10F6A0009805002498050024A0050024A005002446
:10F6B000A8050024A8050024B0050024B0050024F6
:10F6C000B8050024B8050024C0050024C0050024A6
:10F6D000C8050024C8050024D0050024D005002456
:10F6E000D8050024D8050024E0050024E005002406
:10F6F000E8050024E8050024F0050024F0050024B6
:10F70000F8050024F8050024000600240006002463
:10F710000806002408060024100600241006002411
:10F7200018060024180600242006002420060024C1
:10F730002806002428060024300600243006002471
:10F740003806002438060024400600244006002421
:10F7500048060024480600245006002450060024D1
:10F760005806002458060024600600246006002481
:10F770006806002468060024700600247006002431
:10F7800078060024780600248006002480060024E1
:10F790008806002488060024900600249006002491
:10F7A0009806002498060024A0060024A006002441
:10F7B000A8060024A8060024B0060024B0060024F1
:10F7C000B8060024B8060024C0060024C0060024A1
:10F7D000C8060024C8060024D0060024D006002451
:10F7E000D8060024D8060024E0060024E006002401
:10F7F000E8060024E8060024F0060024F0060024B1
:10F80000F8060024F806002400070024000700245E
:10F81000080700240807002410070024100700240C
:10F8200018070024180700242007002420070024BC
:10F83000280700242807002430070024300700246C
:10F84000380700243807002440070024400700241C
:10F8500048070024480700245007002450070024CC
:10F86000580700245807002460070024600700247C
:10F87000680700246807002470070024700700242C
:10F8800078070024780700248007002480070024DC
:10F89000880700248807002490070024900700248C
:10F8A0009807002498070024A0070024A00700243C
:10F8B000A8070024A8070024B0070024B0070024EC
:10F8C000B8070024B8070024C0070024C00700249C
:10F8D000C8070024C8070024D0070024D00700244C
:10F8E000D8070024D8070024E0070024E0070024FC
:10F8F000E8070024E8070024F0070024F0070024AC
:10F90000F8070024F8070024000800240008002459
:10F910000808002408080024100800241008002407
:10F9200018080024180800242008002420080024B7
:10F930002808002428080024300800243008002467
:10F940003808002438080024400800244008002417
:10F95000FFFFFFFF00000200740C0024FF00000006
:10F960004300000000000000000000000000000054
:10F970000000000000000000000000000000000087
:10F980004300000000000000000000000000000034
:10F990000000000000000000000000000000000067
:10F9A0004300000000000000000000000000000014
:10F9B0000000000000000000000000000000000047
:10F9C00043000000000000000000000000000000F4
:10F9D0000000000000000000000000000000000027
:10F9E00043000000000000000000000000000000D4
:10F9F0000000000000000000000000000000000007
:10FA000043000000000000000000000000000000B3
:10FA100000000000000000000000000000000000E6
:10FA20004300000000000000000000000000000093
:10FA300000000000000000000000000000000000C6
:10FA4000E1E30008D1C8000800000000F8EA00085F
:10FA5000F0EE000828EA000828EA000828EA000872
:10FA600028EA000828EA000828EA000828EA00082E
:10FA700028EA000828EA0008FFFFFFFFFFFFFFFF5A
:10FA8000FFFFFFFFFFFF0000010041534349490012
:10FA90000000000000000000000000000000000066
:10FAA00000000000000000000000415343494900ED
:10FAB0000000000000000000000000000000000046
:0CFAC0000000000000000000000000003A
:0400000508002E3D84
:00000001FF
